:10000000002000202523030879C002088DC00208C3
:10001000A1C00208B5C00208C9C002080000000063
:10002000000000000000000000000000DDC0020829
:10003000F1C00208000000003D4800086BA5000860
:1000400055260308592603085D26030897C60208AB
:100050006126030801C8020849C30208D9C402087E
:1000600065C5020865260308692603086D2603088E
:100070007126030875260308792603087D260308E0
:100080008126030885260308892603088D26030890
:100090009126030895260308992603089D26030840
:1000A000A1260308A5260308A9260308AD260308F0
:1000B000B1260308B5260308B9260308BD260308A0
:1000C000C1260308C5260308C926030809C102087A
:1000D000CD260308D1260308D5260308D926030810
:1000E00003C6020865C70208DD260308E1260308E7
:1000F000E5260308E9260308ED260308F126030890
:10010000F5260308F9260308FD260308012703083E
:1001100005270308092703080D27030811270308EB
:1001200015270308192703081D270308212703089B
:1001300025270308292703082D270308312703084B
:1001400035270308392703083D27030841270308FB
:1001500045270308492703084D27030851270308AB
:1001600055270308592703085D270308612703085B
:1001700065270308692703086D270308712703080B
:10018000752703087927030838B5DFF8CC4C002021
:10019000E06120626062A062E062A081DFF8BC0CD6
:1001A000E063DFF8BC0C206460643220E0824FF42E
:1001B00096702083DFF8AC5C4FF42072002105F1CB
:1001C000400002F04BF84FF42072002105F530702A
:1001D00002F044F89022002105F5B86002F03EF8E4
:1001E00040220021284602F039F840220021DFF8A1
:1001F0003C0D02F033F840220021DFF8340D02F00C
:100200002DF840220021DFF82C0D02F027F84022C3
:10021000002105F5A86002F021F84022002105F533
:10022000B06002F01BF840220021DFF80C0D02F054
:1002300015F840220021DFF8040D02F00FF8052226
:100240000021204602F00AF805220021DFF8F00C18
:1002500002F004F805220021DFF8D40D01F0FEFFC2
:100260000020A0822063A0632061A0606063E0643E
:100270000220A07331BD80B50FF2100002F093F898
:10028000DFF8D40B0021017301BD00004C54205352
:10029000746F70007047DFF8C01B4FF47A725043E0
:1002A000C86301460FF2040002F07DB84C5420539D
:1002B0005044202564000000DFF89C2B4FF47A7135
:1002C00048431064014651640FF2040002F06BB819
:1002D0004C5420575044202564000000DFF8781B60
:1002E000C88201460FF2040002F05DB84C5420535E
:1002F0005220256400000000DFF85C1B08830146E3
:100300000FF2040002F04FB84C5420534152202504
:10031000640000000EB410B587B0DFF8184DBDF8CA
:100320006E0000281ED1DFF8100DD0E90023CDE9C2
:100330000223D4E90001CDE90001DDE9022300F048
:1003400088FFDFF8141BC96B4FF47A724243914265
:1003500006D201460FF2280002F025F801200AE03B
:10036000002008E004A802F0BBFA204604A90522F8
:1003700002F05EFB002007B010BC5DF810FB00002F
:100380004C542053544F5020436865636B696E672B
:1003900020256400DFF8C00A01210162C16100214B
:1003A0008162C1627047DFF8B00A01214162C16118
:1003B0007047DFF8A40AC0697047DFF89C0A002183
:1003C000C1610FF2080001F0EEBF00004C54205252
:1003D000455345545F434D4452440000DFF8780ACA
:1003E000002101620FF2040001F0DDBF4C542052E5
:1003F000455345545F504F5352455100DFF8580A5A
:10040000002141620FF2040001F0CDBF4C54205294
:10041000455345545F504F4941434B00DFF8380A7C
:10042000012181620021C16201727047DFF8280A50
:100430000121C16270472DE9FC4106460F469046F6
:10044000DFF8E84ADFF81C5A20462946402202F02D
:10045000FFFA85ED000B85ED021B85ED042B85F879
:10046000296085F82A7085F82B80D4E904230020C0
:10047000014602F029FB0ED1D4E9002302F024FB4F
:1004800009D1D4E9022302F01FFB04D120462946FA
:10049000402202F0DDFA95ED020B8DED000BD5E95F
:1004A00000230FF20C0001F07EFFBDE8F381000095
:1004B0004C54205550504F5320256620256600008F
:1004C00030B583B0DFF89049A06A012815D1DFF874
:1004D000605A2846DFF88C19402202F0B9FA95EDEF
:1004E000020B8DED000BD5E900230FF2140001F093
:1004F0005AFF0020A06201203EBD00203EBD00004A
:100500004C54203173742025662C20256600000091
:1005100030B583B0DFF84049A06A012815D1DFF873
:10052000145A2846DFF83C19402202F091FA95ED62
:10053000020B8DED000BD5E900230FF2140001F042
:1005400032FF0020A06201203EBD0020A0623EBD1F
:100550004C5420326E642025662C20256600000055
:100560000020DFF8F418CA6A012A01D1C86201200C
:1005700070470FB400B59DB0DDE92E2302F0B4FA48
:10058000CDE90C01DDE92001DDE9302302F0ACFA10
:10059000CDE90E010CA984B06846402202F058FA59
:1005A0000FBC00F05DFD53EC102B0020DFF81C1E8B
:1005B00002F05AFB41EC100B1DB05DF814FB00007B
:1005C0000FB470B52DED048B9CB0DFF88C58687AB1
:1005D000002801D1002043E00A2801DB0A2600E0C0
:1005E000AE7A9FED998B002422E0DFF8781801EBBA
:1005F000801000F530710CA8402202F029FA24A9DD
:1006000084B06846402202F023FA0FBCFFF7B1FF26
:10061000B0EE409AF0EE609A51EC190B53EC182BA7
:1006200002F000FC03D2B0EE498AF0EE698A641C45
:10063000E4B22046B042D8DB288B02F019FC024617
:100640000B4651EC180B02F0EDFB01D2002007E045
:1006500053EC182B0FF2140001F0A5FE0120E86402
:100660001CB0BDEC048B70BC5DF814FB4C542053E3
:1006700041204F55542025660000000030B585B05C
:10068000DFF8E04794F969058DF8000004F269503D
:1006900090F901108DF8011090F902008DF8020018
:1006A000B4F86C05ADF80300DFF88C59D5E900010A
:1006B000CDE90201DDE90223DDE9000100F0C9FD19
:1006C000C4F87805DFF89007D5E90023C0E90023D6
:1006D00005B030BD0FB42DE9F0412DED088B84B08D
:1006E000DFF87447DFF87C57A07A05EB80109DEDAA
:1006F000120B80EDA00B00F520709DED140B80ED2A
:10070000020B9DED160B80ED040B2099816394F88C
:100710000980B8F10A0F01DB4FF00A089FEDBF8B8B
:10072000B0EE489AF0EE689AB0EE48AAF0EE68AAE9
:1007300000261DE005EB861753EC182BD7E9B00116
:1007400002F0A4FB41EC180B07F5307753EC192BA2
:10075000D7E9020102F09AFB41EC190B51EC1A0B9C
:10076000D7E9042302F092FB41EC1A0B761CF6B297
:100770004645DFDB404602F07BFB41EC1B0B51ECB6
:10078000180B53EC1B2B02F0F5FB05F5A862C2E930
:10079000000105F2405651EC190B53EC1B2B02F0F3
:1007A000E9FBC6E9020151EC1A0B53EC1B2B02F0DA
:1007B000E1FBC6E9040195F969058DF8000005F231
:1007C000695797F901008DF8010097F902008DF83B
:1007D0000200B5F86C05ADF80300DFF85C88D8E9D5
:1007E0000001CDE90201DDE90223DDE9000100F0AD
:1007F00030FD0246C5F87825D8E90001C4E90001BA
:100800000192B87800907B7895F86925617A0FF2AB
:10081000142001F0C8FD96ED020B8DED000B05F5DF
:10082000A860D0E900230FF2606001F0BCFD032056
:10083000A0730FF2044001F0B6FD04B0BDEC088BCC
:10084000BDE8F0015DF814FB00000000006AF8400C
:100850000FB42DE9F0472DED088B86B0DFF8D047B7
:10086000DFF8D4A7DAE90001CDE90401D4E90001F9
:10087000CDE90201DDE9042300F0EBFCDFF8D855F7
:10088000A97ADFF8E06506EB81129DED160B82ED8B
:10089000B00B02F530739DED188B83ED028B9DED4F
:1008A0001A9B83ED049B237882F8E93202F2E92354
:1008B00067785F70A7789F7000B2C2F8F802481C92
:1008C000A872C0B20A2801D10020A872687A00F18B
:1008D000010885F809805FFA88F8A8F1010002F0A4
:1008E000BDFA41EC1A0B06F2405953EC1A2BD9E928
:1008F000020102F0B9F953EC182B02F0C7FA41ECEF
:10090000180B53EC1A2BD9E9040102F0ADF953ECA2
:10091000192B02F0BBFA41EC190B404602F0A8FA81
:1009200041EC1B0B53EC1A2B06F5A86041680068DC
:1009300002F09AF9DDE9162302F0A8FA53EC1B2B1A
:1009400002F018FB06F5A862C2E9000151EC180B91
:1009500053EC1B2B02F00EFBC9E9020151EC190B01
:1009600053EC1B2B02F006FBC9E9040106F26957A0
:10097000B8F1010F0AD1207886F86905607878709F
:10098000A078B870B4F80300A6F86C0596F969056C
:100990008DF8000097F901008DF8010097F9020029
:1009A0008DF80200B6F86C05ADF80300DAE9000135
:1009B000CDE90201DDE90223DDE9000100F049FC97
:1009C0000246C6F87825DAE90001C5E9000101927E
:1009D000B87800907B7896F86925697A0FF2440020
:1009E00001F0E1FC99ED020B8DED000B06F5A8601E
:1009F000D0E900230FF2904001F0D5FC687A01287D
:100A000005D10120A8730FF28C4001F0CCFC06B098
:100A1000BDEC088BBDE8F0075DF814FB000000009A
:100A2000000000004C542025642053502025643AD7
:100A300025643A25642C2025640000000FB42DE9BC
:100A4000F0472DED0A8B86B0DFF8ECA5DAE900015E
:100A5000CDE90401DFF8E804D0E90023CDE9022361
:100A6000DDE90423DDE9020100F0F3FB8046DFF855
:100A7000E843A07A461E36B2002E01D50A3636B2B9
:100A8000607A02F0F5F941EC180BF64D05EB86168D
:100A900053EC182B05F5A8604168006802F0E4F8F3
:100AA000D6E9B02302F020F841EC190B06F53077B7
:100AB00005F2405953EC182BD9E9020102F0D4F8A1
:100AC000D7E9022302F010F841EC1A0B53EC182B73
:100AD000D9E9040102F0C8F8D7E9042302F004F8C8
:100AE00041EC1B0B9FEDE0CBD6E9B023DDE918010B
:100AF00002F0CCF953EC1C2B02F0B6F8C6E9B001B9
:100B0000D7E90223DDE91A0102F0C0F953EC1C2BEE
:100B100002F0AAF8C7E90201D7E90423DDE91C01C4
:100B200002F0B4F953EC1C2B02F09EF8C7E9040163
:100B3000C7F8388053EC1A2BD7E9020102F0A6F966
:100B400041EC1A0B51EC1B0BD7E9042302F09EF980
:100B500041EC1B0B51EC190BD6E9B02302F096F9CE
:100B600053EC182B02F006FA05F5A862C2E9000161
:100B700051EC1A0B53EC182B02F0FCF9C9E90201F5
:100B800051EC1B0B53EC182B02F0F4F9C9E90401EA
:100B900095F969058DF8000005F2695696F901008E
:100BA0008DF8010096F902008DF80200B5F86C0589
:100BB000ADF80300DAE90001CDE90201DDE9022325
:100BC000DDE9000100F045FB0246C5F87825DAE9C9
:100BD0000001C4E900010192B0780090737895F8A3
:100BE0006925617A0FF2380001F0DDFB99ED020B07
:100BF0008DED000B05F5A860D0E900230FF28820E9
:100C000001F0D1FB0320A0730FF22C0001F0CBFB0D
:100C100006B0BDEC0A8BBDE8F0075DF814FB0000E0
:100C20004C5420256420552D53502025643A2564CA
:100C30003A25642C202564004C5420415245412023
:100C400053544159000000000FB42DE9F0472DED39
:100C50000A8B86B09FED848BDDE91823DDE928013E
:100C600002F014F953EC182B01F0FEFF41EC190BC4
:100C7000DDE91A23DDE92A0102F008F953EC182B0B
:100C800001F0F2FF41EC1A0BDDE91C23DDE92C0138
:100C900002F0FCF853EC182B01F0E6FF41EC180BC6
:100CA000A74CDFF894A3DAE90001CDE90401D4E907
:100CB0000001CDE90201DDE9042300F0CAFA664D26
:100CC000A97ADFF8AC6C06EB811282EDB09B02F5DD
:100CD000307383ED02AB83ED048B237882F8E93225
:100CE00002F2E92367785F70A7789F70B4F8033049
:100CF000A2F8EC32C2F8F802481CA872C0B20A2866
:100D000001D10020A872687A00F1010885F80980F5
:100D10005FFA88F8A8F1010002F0A0F841EC1B0B83
:100D200006F2405953EC1B2BD9E9020101F09CFF5C
:100D300053EC1A2B02F0AAF841EC1A0B53EC1B2BC4
:100D4000D9E9040101F090FF53EC182B02F09EF852
:100D500041EC180B404602F08BF841EC1C0B53ECB5
:100D60001B2B06F5A8604168006801F07DFF53EC7D
:100D7000192B02F08BF853EC1C2B02F0FBF806F554
:100D8000A862C2E9000151EC1A0B53EC1C2B02F0D3
:100D9000F1F8C9E9020151EC180B53EC1C2B02F0DD
:100DA000E9F8C9E9040106F26957B8F1010F0AD15F
:100DB000207886F8690560787870A078B870B4F803
:100DC0000300A6F86C0596F969058DF8000097F9FF
:100DD00001008DF8010097F902008DF80200B6F8C5
:100DE0006C05ADF80300DAE90001CDE90201DDE9A7
:100DF0000223DDE9000100F02CFA0246C6F878254E
:100E0000DAE90001C5E900010192B87800907B7829
:100E100096F86925697A0FF2580001F0C4FA99ED45
:100E2000020B8DED000B06F5A860D0E900230FF250
:100E3000580001F0B8FA687A012805D10120A8739A
:100E40000FF2500001F0AFFA06B0BDEC0A8BBDE81E
:100E5000F0075DF814FB0000D8240120E0930400A3
:100E600060E31600F8C50020000000000000E03F2D
:100E70004C5420256420532D53502025643A25647A
:100E80003A25642C202564004C54202566202566D4
:100E9000000000004C54204152454120494E0000C2
:100EA0000FB410B584B0DFF8CC0A016B01EBC102BE
:100EB000DFF8BC3A03EBC20202F5B8639DED060B06
:100EC00083ED000B9DED080B83ED020B08AC94ED58
:100ED000021B83ED041B9DF8413082F8E93502F2D4
:100EE000E9530DF1410464785C700DF14104A4787C
:100EF0009C70BDF84430A2F8EC3502F2EC5211AB14
:100F0000DB685361C48A1483048B5483002901D1A4
:100F10000121016302938DED000BDDE906230FF241
:100F2000240001F040FA1FBC5DF814FBF0250120FD
:100F30003026012070260120B0260120F026012055
:100F4000582E01204C5420555341202566202566FB
:100F5000202564000FB4F0B585B0DFF8184A4825A5
:100F6000DFF80C6A206B05FB006000F5B8619DEDB1
:100F70000A0B81ED000B9DED0C0B81ED020B0CAA11
:100F800092ED020B81ED040B9DF8511080F8E915EC
:100F900000F2E9520DF151035B7853700DF15107E6
:100FA000BF789770BDF95420A0F8EC258DF8041097
:100FB0008DF805308DF80670ADF8072094F9000023
:100FC0008DF80C0060788DF80D00A0788DF80E007B
:100FD000B4F80300ADF80F00DDE90323DDE90101FA
:100FE00000F037F9074600979DF906309DF9052076
:100FF0009DF904100FF2440001F0D5F9206B05FBB8
:101000000061C1F8007601F20061E28A8A80228BD9
:10101000CA80022801D2401C20630220A0730FF274
:10102000340001F0C0F905B0F0BC5DF814FB00001D
:10103000602E0120682E0120502E01204C54205398
:101040005341312025643A25643A25642C202564D7
:10105000000000004C542041524541204F5554009F
:101060000FB438B52DED048B8CB006AA08A90AA8D8
:101070009DED140B00F06EF8DDE90A230020DFF887
:10108000F81801F0F1FD04460D46DDE90823DFF80C
:10109000EC08DFF8EC1801F0E7FD22462B4601F0E2
:1010A000F5FE04460D46DDE90623DFF8D808DFF833
:1010B000D81801F0D9FD22462B4601F0E7FE41EC9D
:1010C000180B00AA02A904A89DED160B00F042F827
:1010D000DDE904234FF03330DFF8B01801F0C4FD30
:1010E00004460D46DDE90223DFF8A408DFF8A41862
:1010F00001F0BAFD22462B4601F0C8FE04460D461B
:10110000DDE90023DFF87408DFF88C1801F0ACFD8E
:1011100022462B4601F0BAFE41EC190B53EC182B7A
:1011200051EC180B01F0A0FD04460D4653EC192BB1
:1011300051EC190B01F098FD22462B4601F0A6FE5A
:1011400041EC100B02F03AF80CB0BDEC048B31BC52
:101150005DF814FB70B52DED048BB0EE408AF0EE17
:10116000608A04460D46164651EC180B53EC182BBA
:1011700001F0BAFC41EC190B53EC192B0020DFF8FD
:101180001C1801F071FD41EC100B84ED008B85ED16
:10119000000B0022DFF8043801F0ECFE02460B469B
:1011A00051EC190B01F0A0FC0022DFF8F43701F03C
:1011B0005BFDC6E90001BDEC048B70BDDFF8B40730
:1011C000006A7047DFF8AC07406A704780B540227C
:1011D0000021DFF8D00701F041F840220021DFF8BC
:1011E000C80701F03BF8DFF8D40D0021417281728D
:1011F000016181820FF20C00BDE8024001F0D3B81A
:10120000000000004C542052455345545F41535058
:1012100000000000DFF8A40D006B704780B5DFF818
:10122000501701F5B06001F5A861402201F010FCF3
:10123000DFF8880D0021016301BDC9B201EBC102D5
:10124000DFF82C1701EBC20101F5B861482201F06B
:10125000FFBB3FB581B04FF47A704EF66022DFF8E5
:10126000603D9DF904109DF90540544303FB014185
:101270009DF9064014FB0011BDF9074001FA84F105
:101280009DF90C409DF90D506A4303FB04229DF922
:101290000E3013FB0020BDF90F2000FA82F0441A33
:1012A00042F20F721319934205D200240FF23C0050
:1012B00001F079F807E0DFF80C2D944203DADFF84B
:1012C000082D1018441ADFF8040D844200DB044690
:1012D000204601F0C3FDDFF8F82CDFF8F83C01F000
:1012E000C3FC05B0BDE8304001F0E8BF41542D4CCF
:1012F0005420646966662054696D65205265736583
:10130000740000002DE9F64383B08146BDF90F401B
:101310004EF66025DFF8A86C9DF90C009DF90D10C4
:10132000694306FB00109DF90E104FF47A7211FB11
:10133000020000FA84F10C98412808D15F18DFF808
:10134000980C87420BD3DFF8940CC71907E0994239
:1013500004D2DFF8740C4018C71A00E0CF1A3846E0
:1013600001F086FD0022DFF8783C01F003FE01F079
:10137000A5FF80465FFA88F806FB1876304601F034
:1013800077FD0022DFF85C3C01F0F4FD01F096FFF0
:10139000C0B28DF8008001468DF8011005FB106089
:1013A00001F066FDDFF8282CDFF8283C01F05CFC3A
:1013B00001F084FF8DF80200ADF80340484600A913
:1013C000052201F035FB05B0BDE8F08300408F40F9
:1013D00010B50024DFF89C05C16C012907D1012458
:1013E0000021C1640FF2540000F0DDFF23E0DFF8BC
:1013F0008005D0F87815D0F8B825914216D190F82C
:10140000691590F8A925914210D100F2A95100F276
:10141000695042784B789A4208D18078897888421E
:1014200004D10FF6EC3000F0BEFF04E001240FF60B
:10143000E83000F0B8FF204610BD00004C542046B4
:101440005500000000B58DB0DFF82805407A00286F
:101450000AD0DFF8941B84B06846402201F0F8FA05
:101460000FBCFFF71DFD06E00FF6B4300DB05DF8C0
:1014700004EB00F098BF0DB000BD00001CB5DFF814
:10148000F444217B61732073401E05284DD8DFE8AA
:1014900000F0034C16222C4100A801F021FADFF8DD
:1014A0004C0B00A9052201F0C3FA616C21640020F5
:1014B000E0720FF67830BDE81C4000F074BF00A861
:1014C00001F00EFADFF8240B00A9052201F0B0FAB2
:1014D000A06BA06413BD00A801F002FADFF80C0BAA
:1014E00000A9052201F0A4FA13BD00202061A0820A
:1014F00040220146DFF8B00400F0B0FE00A801F081
:10150000EFF9DFF8E80A00A9052201F091FAA06BD3
:10151000A06413BD00A801F0E3F9DFF8D00A00A928
:10152000052201F085FAA06BA06413BD0CB400B5D0
:1015300083B09DF939108DF800100DF1390191F942
:1015400001108DF801100DF1390191F902108DF89B
:1015500002100021ADF8031000A9052201F068FA7D
:101560000EBC5DF80CFB00002DE9F84F2DED0A8B49
:101570009CB082469FED558BDFF8F883B8F81000D9
:10158000B8F81290814502D25FFA89F901E0C0B241
:101590008146B8F91400461E00D50A36DFF8D0B3EC
:1015A0000BEB861797ED109B97ED12AB97ED14BBE5
:1015B00001243CE0301A00D50A300BEB801505F110
:1015C00040010CA8402201F043FA07F1400184B029
:1015D0006846402201F03CFA0FBCFEF7CAFFB0EEAD
:1015E00040CAF0EE60CA51EC180B53EC1C2B01F012
:1015F00019FC03D2B0EE4C8AF0EE6C8A53EC1B2B34
:10160000D5E9140101F042FC41EC1B0B53EC192B02
:10161000D5E9100101F03AFC41EC190B51EC1A0B21
:10162000D5E9122301F032FC41EC1A0B641CE4B240
:1016300020464845BEDB484601F01AFC41EC1C0B35
:1016400051EC1B0B53EC1C2B01F094FCCAE9040178
:1016500051EC190B53EC1C2B01F08CFCCAE9000176
:1016600051EC1A0B53EC1C2B01F084FCCAE902016B
:10167000B8F81000B8F8121088421ED207F14001E5
:101680000CA8402201F0E4F9DFF8641984B0684640
:10169000402201F0DDF90FBCFEF76BFFB0EE40CA4F
:1016A000F0EE60CA51EC180B53EC1C2B01F0BAFBA6
:1016B00003D2B0EE4C8AF0EE6C8AB0EE480AF0EE3F
:1016C000680A1CB0BDEC0A8BBDE8F18F0000000079
:1016D000000000000FB42DE9F0412DED068BA0B005
:1016E0002CA984B06846402201F0B2F90FBCFEF785
:1016F00067FFA04D68639E4E012812D100206863E9
:1017000006F5A86184B06846402201F0A1F90FBC3B
:10171000FFF720FCFFF75AFD0FF6201000F043FE04
:1017200019E1B5F9144006EB841040302CA9402291
:1017300001F08EF9601CA88200B20A2801D10020B5
:10174000A882288A0A2801DA401C2882688A401C5C
:101750006882314682B06846402201F079F90CBCBB
:101760000EA8FFF7E3FE288A0A2801DA002700E026
:101770002F7D8D4CD4E900010022134601F0A4F91D
:101780002FD1D4E9020101F09FF92AD1D4E9040153
:1017900001F09AF925D106EB8716DFF8588896F9FB
:1017A000690088F8000006F2690090F9011088F8D5
:1017B000011090F9020088F80200B6F86C00A8F851
:1017C0000300DFF82C0806F14001402201F040F947
:1017D000204606F14001402201F03AF90020A063C2
:1017E000B9E010A8FFF7C0FEB0EE408AF0EE608AC4
:1017F000DFF80088288B400801F03AFB53EC182BE7
:1018000001F010FB28D206EB871696F9690088F8DC
:10181000000006F2690090F9011088F8011090F9B3
:10182000020088F80200B6F86C00A8F80300DFF8A0
:10183000C00706F14001402201F00AF9204606F1F6
:101840004001402201F004F90020A06368820FF2F9
:10185000FC7000F0A8FD7EE0D8E90001CDE90001B0
:10186000DDE90E23FFF7F5FC064631460FF2EC707A
:1018700000F099FD286C4FF47A71714388426AD266
:101880006F8A3846042866DBA16B002916D19DEDCE
:10189000100B84ED000B9DED120B84ED020B9DED02
:1018A000140B84ED040BA663214684B068464022E5
:1018B00001F0CEF80FBCFEF7CBFF43E0401E01F075
:1018C000CDFA41EC190B384601F0D2FA41EC1A0B73
:1018D00051EC190BD4E9002301F0C6F9DDE92C2302
:1018E00001F0D4FA53EC1A2B01F044FBC4E90001D7
:1018F00051EC190BD4E9022301F0B6F9DDE92E23EE
:1019000001F0C4FA53EC1A2B01F034FBC4E90201D4
:1019100051EC190BD4E9042301F0A6F9DDE93023D9
:1019200001F0B4FA53EC1A2B01F024FBC4E90401D2
:10193000A663214684B06846402201F089F80FBCB6
:10194000FEF7C8FEA06B009053EC182B698A0FF2CB
:101950001C7000F028FD20B0BDEC068BBDE8F00146
:101960005DF814FB7047DFF85406807B7047000079
:10197000F8C50020D824012000C05B409A999999AD
:101980009999FD3F5839B4C876BE9F3F33335640CE
:10199000AE47E17A14AEF73F9999993F00004E4067
:1019A0000020AC4038CB0020B02601200EB478B522
:1019B0002DED028B9EB00646DFF80046A06B08189E
:1019C000A06300A800F08CFFDFF82C56284600A981
:1019D000052201F02DF8207B062800F2E782DFE8DF
:1019E00010F0070012007400C1006A011402C00266
:1019F000FFF7ECFB0120FFF741FD217B0FF2846034
:101A000000F0D1FCD2E225A983B06846582201F04B
:101A10001FF80EBC304680B2FEF77CFC002843D095
:101A2000D5E90001CDE903014D200090E36BDDE92C
:101A300003010A46014601A8FFF764FCDFF8BC0574
:101A400001A9052200F0F4FFDFF8B41582B0684662
:101A5000402200F0FDFF0CBC1CA8FFF767FDD5E994
:101A60000001CDE90001DDE90023DDE91C01FFF7FC
:101A7000F0FB05463D2D07DB29460FF2186000F00C
:101A800092FCFEF787FC06E00120A06229460FF2D7
:101A9000146000F088FC0220FFF7F0FC217B0FF2BD
:101AA000146000F080FC81E2A06A012840F07E8290
:101AB0000020A062DFF8481584B06846402200F09C
:101AC000C7FF0FBCFFF706FE70E2FEF7F9FC002827
:101AD00034D00320FFF7D2FC0FF2E85000F063FC93
:101AE000607A00281FD0DFF81C55294684B068466C
:101AF000402200F0ADFF0FBCFEF762FD60630128DD
:101B000011D100206063DFF8E01484B06846402201
:101B100000F09EFF0FBCFFF71DFAFFF757FB0FF217
:101B2000B85000F040FCDFF8D81484B0684640227A
:101B300000F08EFF0FBCFFF7CDFD37E2FEF710FD82
:101B4000002800F03382207A401C2072C0B20328A3
:101B500080F243810120FFF791FC0FF2985000F0D2
:101B600022FC23E2A06A012851D10020A062DFF804
:101B70009064607A00281DD0314684B068464022C7
:101B800000F066FF0FBCFEF71BFD6063012811D15A
:101B90000020606306F5A86184B06846402200F02A
:101BA00057FF0FBCFFF7D6F9FFF710FB0FF25C50A1
:101BB00000F0F9FB314684B06846402200F048FF4F
:101BC0000FBCFFF787FD31460CA8402200F040FF14
:101BD000DFF8301484B06846402200F039FF0FBCB3
:101BE000FEF7C7FCB0EE408AF0EE608AE08A01F0B2
:101BF0003FF953EC182B01F015F908D20120FFF73B
:101C00003DFC53EC182B0FF2105000F0CCFBD5E943
:101C10000001CDE90201DFF8D403D0E90023CDE9CA
:101C20000023DDE90223DDE90001FFF712FBA16BD0
:101C3000A26C8E1A332E08D30120FFF71FFC314609
:101C40000FF2EC4000F0AFFBB0E1216C4FF47A7280
:101C50005043814280F0AA81DFF8A41382B0684625
:101C6000402200F0F5FE0CBC1CA8FFF75FFCD5E994
:101C70000001CDE90001DDE90023DDE91C01FFF7EA
:101C8000E8FA05463D2D07DBFEF784FB29460FF2F7
:101C9000B84000F088FB06E00120A06229460FF260
:101CA000044000F080FB0420FFF7E8FB0FF2A8409F
:101CB00000F079FB7AE1FEF72BFC002800F082802F
:101CC000D14E314684B06846402200F0C1FE0FBCC0
:101CD000FEF776FC6063012818D100206063C249DA
:101CE00084B06846402200F0B3FE0FBCFFF732F923
:101CF000FFF76CFA0FF2704000F055FB607B05288F
:101D000040F054810120FFF7B9FB4FE1BD4D314652
:101D10000CA8402200F09CFE294684B06846402270
:101D200000F096FE0FBCFEF724FCB0EE408AF0EE09
:101D3000608AE08A01F09CF802460B4651EC180BD1
:101D400001F070F82BD2607B052831460CD184B0AD
:101D50006846402200F07CFE0FBCFEF76FFE0FF2DB
:101D6000144000F020FB10E00CA8402200F070FEB0
:101D7000294684B06846402200F06AFE0FBCFEF798
:101D800063FF0FF2FC3000F00EFBFEF70CFB0520AA
:101D9000FFF774FB0FF2F03000F005FB06E10120C5
:101DA000FFF76CFB53EC182B0FF2F03000F0FBFA4E
:101DB000934984B06846402200F04AFE0FBCFFF70A
:101DC00089FCF3E0FEF7CCFB002800F0EF80207ADE
:101DD000401C2072C0B2032807DB0620FFF74EFB31
:101DE0000FF2003000F0DFFAE0E0884820640320C2
:101DF000FFF744FB217A0FF2B83000F0D4FA216CDF
:101E00000FF2282000F0CFFAD0E0A06A012846D1D6
:101E10000020A0627A4E607A00281DD0314684B03E
:101E20006846402200F014FE0FBCFEF7C9FB606359
:101E3000012811D10020606306F5A86184B06846CE
:101E4000402200F005FE0FBCFFF784F8FFF7BEF953
:101E50000FF2743000F0A7FA31460CA8402200F0CF
:101E6000F7FD684984B06846402200F0F1FD0FBCE0
:101E7000FEF77FFBB0EE408AF0EE608AE08A00F069
:101E8000F7FF53EC182B00F0CDFF08D20120FFF72D
:101E9000F5FA53EC182B0FF23C3000F084FAD5E938
:101EA0000001CDE902015148D0E90023CDE900232A
:101EB000DDE90223DDE90001FFF7CBF9A16BA26C9C
:101EC0008E1A332E08D30120FFF7D8FA31460FF2CD
:101ED0001C3000F068FA69E0216C4FF47A725043CC
:101EE00081423BD2464E96F929008DF8700006F2E9
:101EF000290090F901108DF8711090F902008DF809
:101F00007200D5E90001CDE90001DDE90023DDE93A
:101F10001C01FFF79EF905463D2D07DBFEF73AFA57
:101F200029460FF2E02000F03EFA06E00120A06210
:101F300029460FF2E02000F036FA0420FFF79EFA5F
:101F4000E07A401CE072C0B203282FDB606C4100D5
:101F500021640FF2D80000F026FA27E0FEF78EFB8E
:101F600024E0A06BA16C401A33280BD30120FFF7AB
:101F700085FA0FF2B42000F016FA0FF2C02000F03C
:101F800012FA13E0A06A01280BD10120FFF776FABC
:101F90000FF2B42000F007FA0FF2A02000F003FACD
:101FA00004E0607B042801D1FEF768FB207B1EB0B3
:101FB000BDEC028B72BC5DF810FB0000D824012040
:101FC00080EE3600F1D8FFFF005C2605C0E40A056C
:101FD000FCA9F1D24D62503F015C260500A4D9FA5C
:101FE00040774B41004CED4038CB0020682E01205B
:101FF000F0260120602E0120502E0120582E0120B5
:10200000F8C500203026012070260120E09304004E
:102010004C542053410000004C542044490000001F
:102020004C54204E6F20504F530000004C542D57FD
:1020300050204348414E4745202564004C542053CE
:10204000617665205341554D000000004C542052EC
:10205000455345545F474150000000004C54204711
:1020600041204D546D202564000000004C54205345
:102070005020534741522025642C2025662C2025D2
:10208000640000004C542D434B5F53544F502025A7
:10209000640000004C5420524551504F532D4620AF
:1020A000256400004C54204E2D524551504F532072
:1020B000256400004C542D4745545F315F504F5309
:1020C000202564004C542D434B5F555345525F4DC2
:1020D0004F564554000000004C54205353412D46A8
:1020E000500000004C542D53535F50415553455FF1
:1020F000535300004C542053535F475053204E4FCE
:1021000054204F4B20317374000000004C54205376
:1021100053412D554D0000004C542D434B5F5354FB
:102120004F502D554D2D64697374202566000000B5
:102130004C542D434B5F53544F502D554D2D7374BC
:1021400065702025640000004C5420524551504FCA
:10215000532D5320256400004C542D4745545F32C5
:102160005F504F53000000004C54205353412D53F7
:10217000500000004C54205544542053500000009F
:102180004C542053535000004C542D434B5F555337
:1021900045525F4C454156494E4700004C542D4333
:1021A0004845434B5F53544F502D535020256600F4
:1021B0004C542D475053204E4F54204F4B20326EDD
:1021C00064202564000000004C54205353412D55D9
:1021D0004C0000004C542D434B5F53544F502D5531
:1021E0004C20646973742025660000004C542D4314
:1021F0004B5F53544F5020554C207374657020250D
:10220000640000004C5420524551504F532D554C02
:10221000202564004C54204E2D524551504F532DD3
:10222000554C2025640000004C5420535320414756
:1022300041494E2042592053544550004C542D439F
:102240004B5F53544F5000004C5420535320414790
:1022500041494E20425920504F53000010B50446CA
:1022600010460A460146204601F054F8204610BDAB
:10227000BFF34F8FDFF81C07016801F4E061DFF85E
:10228000442711430160BFF34F8FFEE710B5DFF81D
:1022900038474FF48E7200212046FFF7DFFF2046BB
:1022A00010BDDFF82407704710B5FFF7EFFF0446B5
:1022B00000231A461146084600F06FFAC046C04691
:1022C00001F05CF8204600F019F801F0AEFA204663
:1022D00000F0D0F9204600F015F8204600F01FF875
:1022E00000F093F900206072A072E0722073012068
:1022F00060730020E075A073012010BD0021C17142
:10230000017231E010B50446DFF88C0601F0E2F806
:10231000DFF8B80601F0DEF80120607110BD10B5DD
:10232000044601F042F90120A07110BD38B5044601
:10233000012501F0EDF9012804D12846E0700020C4
:10234000A0700AE0022804D10020E0702846A070A6
:1023500003E00020E070A0700546284632BD80B53D
:1023600001F054FB012002BD10B50446E07901F0F4
:102370008BFC0121217010BD70B504460025E67963
:10238000E171FFF7F1FF002807D02046FFF7BAFF01
:102390002046FFF7C4FF012503E0E6712046FFF762
:1023A000E3FF284670BD0EB470B5C1B0054600A865
:1023B0004FF4807102F0F2F9FFF773FF044645AB6A
:1023C0002A464FF4807100A802F0ECF900A802F050
:1023D00007FA451C00A82818002100F8011CDFF8A6
:1023E000F0653078401C30707078F021084202D0DF
:1023F000992002F011FA02F07CFA7078401C70709B
:10240000207E2818FF2810DA207E002803D0207EA6
:1024100000190A2101762A4600A9207E00191930E8
:1024200002F07EFA207E2818207600A802F0D0FC68
:102430007078F021084202D0992002F0EDF970780E
:10244000401E7070C0B2002801D102F04CFA03F0B7
:10245000AAF841B070BC5DF810FB0428DFF83C0519
:1024600003D8DFF8341501607047DFF860150160AC
:102470007047DFF82C1551F82000007F002807D0A6
:10248000DFF8500501784A1C0270032900DBEFE6F3
:1024900070472DE9F84305460E4617464FF00208EF
:1024A000DFF82C456078F021084202D0992002F034
:1024B000B3F902F01EFA6078401C60709DF80000CD
:1024C000401E8DF8000017F8019B2846FFF7C5FF56
:1024D00000AB4A463946304601F0EEFC002810D0E9
:1024E0006078F021084202D0992002F095F96078D6
:1024F000401E6070C0B2002801D102F0F4F9012042
:102500001FE05FFA88F8424629460FF2D440FFF7F1
:102510004AFF4046A0F101080028D9D16078F02197
:10252000084202D0992002F077F96078401E60706E
:10253000C0B2002801D102F0D6F92846FFF799FF72
:102540000020BDE8F2832DE9F04704460D4616460B
:102550001F46DFF85084089888F80000DFF8709470
:1025600099F80100F021084202D0992002F054F9B4
:1025700002F0BFF999F80100401C89F801002046DB
:10258000FFF76BFF4FF0020A4346324639462846B2
:1025900001F042FD002813D099F80100F021084213
:1025A00002D0992002F038F999F80100401E89F80C
:1025B0000100C0B2002801D102F095F9012022E00B
:1025C0005FFA8AFA524621460FF22040FFF7EBFEEF
:1025D0005046A0F1010A0028D6D199F80100F02157
:1025E000084202D0992002F017F999F80100401E24
:1025F00089F80100C0B2002801D102F074F9204628
:10260000FFF737FF0020BDE8F08703F029BDF8B5DC
:10261000044602270025DFF888630DE039464F1E87
:10262000C9B200290AD1002804D120690121A9409A
:102630008843206102276D1C162D10DA56F82500FC
:10264000006E006880470128E8D121690122AA4074
:102650001143216156F8251001220A77E3E720692A
:10266000032803D0022801D0012802D140F4805071
:102670002061F1BD01F018BE01F071BE81B00022F1
:10268000ADF80220ADF80020C079042808D0062853
:1026900009D008280AD009280BD00A280CD00EE04F
:1026A0004FF4C8600DE04FF448600AE04FF4C850A2
:1026B00007E04FF4FA5004E042F2107001E041F2FA
:1026C0007070ADF802200DE0BDF80020521CADF88E
:1026D0000020BDF800208242F6DBBDF80220521C2B
:1026E000ADF80220BDF802208A4203D20022ADF8E4
:1026F0000020EEE701B07047417230B589B003F0B9
:1027000083FD0446FFF7CDFD054600A8242102F015
:1027100045F80020ADF8220001900A208DF808004D
:1027200000208DF809008DF80A00687A00280DD085
:10273000002C18D000208DF80000052001900B20FF
:102740008DF8080000A805F0CFFC0CE0002C0AD0A2
:1027500001208DF80000052001900B208DF8080065
:1027600000A805F0C1FC09B030BD01F014BE01F0B5
:102770001CBE01210846F8E701210846F7E70221BF
:102780000120F2E702210120F1E701F019BE10B5A6
:102790000446FFF786FD447510BD2DE9F04782B071
:1027A0000C4615462F46264680464FF47A714FF068
:1027B0003C0C4FF4616918FB09F216FB0C22BA18A5
:1027C00001FB0232DFF8E0E19EF900A01AFB09F9F3
:1027D0009EF901A01AFB0C9C9EF902904CFA89FC10
:1027E000BEF9039001FB0C919EF808C0BCF1000FEC
:1027F00022D144EA00012943194302D001218EF875
:1028000008108EF80000B8F1000F04D59EF8000003
:1028100018308EF800008EF801408EF80250AEF8A5
:10282000033000933B4632469EF900100FF2EC1045
:10283000FFF7B9FDBDE8F38791420DD3A1EB020C80
:10284000ACF2D17CDFF89091CC45DAD30FF2A8102E
:1028500002B0BDE8F047A6E5D3D2A2EB010CACF282
:10286000D179DFF874A1D145CBD363460FF298102C
:1028700002B0BDE8F04796E510B504002FD003F094
:1028800079FD4949CA68002A00D0841AB1F80320AA
:10289000A218A1F8032012B2B2F57A7F06DBA2F5E6
:1028A0007A72A1F803208A78521C8A7091F902206A
:1028B0003C2A04DB3C3A8A704A78521C4A7091F9EF
:1028C00001203C2A04DB3C3A4A700A78521C0A7008
:1028D00091F90020182A01DB00220A70C86010BD9F
:1028E0003149052200F0A4B80FB410B52DED028BCC
:1028F0002E4C104600F0BCFA2D4A2E4B00F0B4F9D5
:10290000206161619FED2C8B049800F0B1FA53ECCB
:10291000182B00F0A9F920606160059800F0A8FA72
:1029200053EC182B00F0A0F9A060E1609DF81C00AA
:10293000207604F118009DF81D1041709DF81E10BE
:1029400081709DF81F10C1709DF820100171BDF8B5
:10295000210000EE100AB8EE400A10EE100A05F051
:10296000EBFC174A1D4B00F07FF905F00DFDC4F894
:102970001D00BDF82300A4F821009DF8250084F86F
:102980002300BDEC028B10BC5DF814FB0749242228
:1029900000F04EB80CED00E0005400403468002018
:1029A00008400020F02E01205C2C0120A8290120E5
:1029B000FCA9F1D24D62503F8DEDB5A0F7C6B03EF7
:1029C0003BDF4F8D0400FA05AC0A0120005800409F
:1029D0002C670020EF2E01205F4C2605976EA23F4A
:1029E00049574520256420256400000049524520B0
:1029F000256420256400000041542D536574545310
:102A0000312025642025640041542D5365745453AE
:102A100032202564202564202564000041542D5374
:102A20006574542025643A25643A25642E25640093
:102A300062B38B0708D0521E11F8013B00F8013B2E
:102A400000F024808B07F6D1830740F0208000BF80
:102A5000103A07D330B4B1E83810103AA0E8381073
:102A6000F9D230BC530724BFB1E80810A0E8081021
:102A700044BF51F8043B40F8043BD20724BF31F86F
:102A8000022B20F8022B44BF0B7803707047083AE2
:102A900007D3B1E80810083A40F8043B40F804CBEB
:102AA000F7D25307E4E750F8041B61B150F8042B48
:102AB000D30744BFA9F101039A18002342F8043B4D
:102AC000091FFAD1EFE7704790420CD141EA030C9D
:102AD00050EA4C0C07D0994205D14FF4001C1CEB76
:102AE000410F38BF8942704770B44FF0004591EAFA
:102AF000030F44BF6B4000F0D3B900BF841A71EBE1
:102B0000030604D26E40001BB141121973414FF409
:102B1000001C1CEB410F34BF7CEB430684E00C0D22
:102B2000A4EB1356362E7DDC012E43DC45EAC3238D
:102B300043EA525312BFD20292025B08240545EACF
:102B4000C12141EA5051D2EBC020994125D407D18F
:102B5000B0FA80F610FA06F164D00020203608E0C2
:102B6000B1FA81F6B140C6F1200220FA02F2114317
:102B7000B0404FEAF474B4EB465434F001064FEA27
:102B800074040AD8D6F50016760D04F00044F0401F
:102B900061FA06F25040F1404840C00A40EA415014
:102BA00021F0004128BF5FEA500550F1000044EBDE
:102BB000D12137E045EAC323DB0A45EAC121C90A2E
:102BC000B6F120050EDD42EA0242120CC5F12006E4
:102BD00003FA06F6EB4042EA06056D42984161F1C0
:102BE00000010DE062FA06F5F240554063FA06FC7A
:102BF00082EA0C02F3405A406D42904161EB0301BE
:102C000011F4801F05D1641E620502D06D004041A1
:102C1000494121F48011430875F1004350F100004F
:102C200041EB045170BC70471CEB410F15D223F0EF
:102C3000004352EA43060BD04FEA4C0CBCEB410F69
:102C400004D80C0D661E342EB7DDEBE7801A9941CF
:102C500050EA410608BF0021E4E708BF1CEB430F20
:102C600028BF6FF00001DDE7B0B581EA030C0CF07E
:102C7000004C40F2FF7515EA11541DBF15EA1357B9
:102C8000AC42AF4239E0E41923EA455343F48013E0
:102C9000C90241F0004141EA505EC7021100A7FBA2
:102CA000020200284FF00000EEFB01204FF000016F
:102CB000E3FB072118BF42F00102401800214941FF
:102CC000E3FB0E01A4F580640F0302D252004041E1
:102CD000494154F101046CDD470872F1004250F1A2
:102CE000000051EB0451A1F580115CBF41EA0C01D9
:102CF000B0BD4CEA05510020B0BD05EA1357AC4207
:102D000014BFAF4241E050EA410E1CBF52EA430EED
:102D100002E061460020B0BD24423C441BD15FEA82
:102D2000070EF6D0090302BF01460020AEF1140ED3
:102D3000B1FA81F7AEEB070401FA07FE0C37C7F1D1
:102D4000200100FA07F7C8404EEA000E23EA455377
:102D500043F48013A2E733F00043B3FA83F704BFD0
:102D6000B2FA82FE77440B3FE41BB7F1200E2FBF6F
:102D700002FA0EF3BB40C7F1200E22FA0EFE38BF56
:102D800043EA0E03BA40641C82E750EA410E14BFC6
:102D900052EA430E6FF000014FF4001717EB430F98
:102DA0008ABF194617EB410FB5E74CEA05510020E1
:102DB000B0BDD4F10104B4F120070FDAC4F120074B
:102DC000520828BF42F0010210FA07F501FA07F78E
:102DD000E1BF2A43E0403843E1400FE0352C98DC66
:102DE000C7F1200452EA400220FA07F218BF42F06D
:102DF000010231FA07F0A1400A43002172F10042BA
:102E000050F1000051EB0C01B0BD8268521C826091
:102E1000426832B10268531C036011704168491E58
:102E2000416070474FF4001C1CEB410F94BF1CEB3A
:102E3000430F09E041EA030C50EA4C0C52EA0C0C37
:102E400003D2994208BF9042704714BF8B4282421E
:102E500070470268531C036011707047010040F115
:102E60000980F446404200F005F851F00041604707
:102E7000010000BF09D0B0FA80F18840C91CC1F53B
:102E80008461090501EBD0214005704770B44FF013
:102E9000004591EA030C44BF6B40FFF72FBE00BF13
:102EA000841A71EB030603D2001BB141121973415E
:102EB0004FF4001C1CEB410F34BF7CEB430443E098
:102EC0000C0DA4EB1356352E50DC45EAC323DB0A68
:102ED00045EAC121C912B6F120050DDD63FA05F6F8
:102EE000EB4086EA0305124218BF45F00105C01801
:102EF00051F100010CD213E062FA06F5F2405540A0
:102F0000F3415A40B340F3405A408018594107D327
:102F100049085FEA30005FEA350528BF45F0010542
:102F200001F58011420875F1004250F1000041EBBB
:102F3000045170BC4FF4001C1CEB410F38BF7047AC
:102F40000020090D090570471CEB410F10D252EA11
:102F500043060BD0BCEB410F05D80C0DAB43661EEE
:102F6000342EB5DD02E0AB438018594170BC704788
:102F700070BC7047F0B540F2FF7581EA030C0CF0AD
:102F8000004C15EA11541DBF15EA1357AC42AF426D
:102F9000E5E0BC41C1F31301C3F31303801A994167
:102FA00043F4801304D2641E400049418018594103
:102FB000C90241EA5051B1FBF3F603FB1611A2FB23
:102FC0000675D7EBC020A94102D2761E8018594160
:102FD000C90241EA5051B1FBF3FE03FB1E11A2FBF3
:102FE0000E75D7EBC020A94103D2AEF1010E8018B7
:102FF0005941890241EA9051760546EA8E2EB1FB8D
:10300000F3F603FB1611A2FB0675D7EB8020A9414E
:1030100002D2761E80185941C90241EA50514EEA47
:10302000060EB1FBF3F603FB1611A2FB0675D7EBF8
:10303000C020A94102D2761E80185941C90241EA36
:103040005051B1FBF3F703FB1711A2FB0735D3EB8C
:10305000C020A94167F100070CBF004247F00107FB
:1030600066F3D5274FEA1E31B80814F5806412DDE7
:10307000BD0775F1004250EB0E5051EB045111F5B4
:10308000801F5CBF41EA0C01F0BD4CF07F6141F054
:10309000E0410020F0BDBD076D0840EA0E5041F44C
:1030A0008011D4F10104B4F120060ADAC4F120063B
:1030B0000200E04001FA06F3E1401843B240154334
:1030C0000EE0342C13DCC6F1200445EA40056D08FF
:1030D00020FA06F2154321FA06F0A1400D43002123
:1030E00075F1004250F1000051EB0C01F0BD0020E1
:1030F0005FEA0C01F0BDCFB992185B41B3FA83F7D8
:1031000004BFB2FA82F6BF190B3FB7F120062FBFFA
:1031100002FA06F3BB40C7F1200622FA06F638BFD2
:103120003343BA401CB1E419641E33E77F4231F0E7
:103130000041B1FA81F404BFB0FA80F6A4190B3C47
:10314000B4F120062FBF00FA06F1A140C4F1200619
:1031500020FA06F638BF3143A0403C1B1AE7AC42C8
:103160001ABF05EA1357AF4212E050EA41061CBFEE
:1031700052EA4306BFE750EA4107304661461CBFAA
:1031800041EA0551F0BD52EA430C08BFC143F0BD0E
:1031900000204FF4001616EB410F98BF16EB430FBB
:1031A00008BF16EB410F24BFC14305E016EB430FE8
:1031B0000CBF61464CEA0551F0BD000051EC100B0C
:1031C00000B500F003F841EC100B00BD40F2FF7CAD
:1031D0000B0D4DD0634566D230B421EA035141F462
:1031E000801103F2FD3C5FEA5C0C01D300184941F9
:1031F000890041EA907180004FF440140023E202FC
:10320000D50AB1F5100107D46D081DD2091B641948
:1032100000184941491BF7D56D080AD20919641BEA
:1032200000184941491BEFD56D08F7D301E052085A
:1032300017D0C01861419B1AAC4100184941801A4F
:10324000A941F4D452080AD0C01AA1419B186C417C
:1032500000184941801AA941E9D45208F4D15B1CF5
:103260006C4161084FEA330001EB0C5130BC7047F0
:1032700050EA0103FBD030B4B1FA81F311B9B0FACE
:1032800080F41B190B3BB3F120042FBF00FA04F1AB
:103290009940C3F1200420FA04F438BF2143984038
:1032A000D3F101039DE76345E1D011F5801FDED81E
:1032B00050EA4101DBD0D94305F0AEB8F446400DE9
:1032C00040EAC120490006D200F014F8004248BF8D
:1032D0006FF00040604700F00DF84FF00041884269
:1032E0008CBF084640426047400D40EAC12049007B
:1032F00080F00D8040F00040490DA1F58061491C2F
:1033000005D4D1F11F0154BFC840C01770474FF01A
:103310000000704762F30F2262F31F42401810F062
:10332000030308D0C91A1FD3DB0748BF00F8012DDB
:1033300028BF20F8022D130030B41446154610396A
:1033400028BF20E93C00FAD8490728BF20E90C0033
:1033500048BF40F8042D890028BF20F8022D48BF3F
:1033600000F8012D30BC7047C91818BF00F8012DB6
:10337000CB0728BF00F8012D7047000030B583B09F
:103380000121032005F0B3F8DFF8804C204605F05A
:1033900047F9DFF87C5C284605F042F901208DF8FA
:1033A000040000208DF8050001208DF806000020A3
:1033B0008DF80700012128460183C04601200090B6
:1033C00000A9284605F088F9022128460183C04655
:1033D0000220009000A9284605F07EF901208DF812
:1033E000040000208DF80500ADF806004FF4807051
:1033F000009000A9284605F06FF94FF48071284627
:103400004183C04601208DF8040000208DF805009E
:1034100001208DF8060000208DF807004FF4805041
:10342000009000A9204605F057F94FF4805120463E
:103430004183C04604220621284605F09BF9042258
:103440000721284605F096F902208DF80400012096
:103450008DF805008DF8060000208DF8070040204B
:10346000009000A9284605F037F98020009000A9B7
:10347000284605F031F904220A21284605F07AF998
:1034800009220321284605F075F902208DF8040071
:1034900001208DF805008DF8060000208DF807004A
:1034A0004FF48060009000A9284605F015F9082027
:1034B000009000A9284605F00FF9286820F0300098
:1034C00040F010002860206820F0300040F010002C
:1034D000206037BD1FB5DFF83C4BA04230D1012141
:1034E0004FF4001005F00EF80121022004F0FFFF58
:1034F00001214FF4001005F026F800214FF40010D0
:1035000005F021F80020ADF804004BF6FF70ADF88F
:1035100006004FF48060ADF80A004FF48040ADF82B
:103520000C000A20ADF80800DFF8CC0C009000A9D0
:10353000204605F062F90121204605F0C1F91FBDC2
:10354000DFF8B84CA0422FD101214FF4800004F0E5
:10355000D9FF0121022004F0CAFF01214FF48000AD
:1035600004F0F1FF00214FF4800004F0ECFF002094
:10357000ADF804004BF6FF70ADF806004FF4806024
:10358000ADF80A004FF48040ADF80C000A20ADF809
:103590000800DFF8640C009000A9204605F02DF922
:1035A0000121204605F08CF91FBD2DE9F04192B0B4
:1035B00001214FF4805004F0B0FF0121084604F0CF
:1035C00096FF01214FF4800004F091FFDFF83C4AA0
:1035D00005221146204605F0CDF805220721204698
:1035E00005F0C8F805220621204605F0C3F805229B
:1035F0000421204605F0BEF802208DF804000120C9
:103600008DF805000020ADF806002020009000A9EC
:10361000204605F061F88020009000A9204605F0C2
:103620005BF84020009000A9204605F055F81020D6
:10363000009000A9204605F04FF8DFF8C44B204663
:1036400005F0A0F9DFF8BC5B00202880686001204D
:10365000288100206881E860072028820020688097
:10366000DFF8A46B304605F0FDF9DFF8A07B3846A3
:1036700005F0F8F94FF48060069000210D910321C8
:103680000E9100210F910A910890DFF8180C039019
:1036900008461090099007904FF400300C900846AF
:1036A0000B904FF0C068CDF8088040200590084688
:1036B000049002A9304605F059FA00200B90CDF88D
:1036C0000880059005F11400049002A9384605F021
:1036D0004DFA002068802946204605F082F9012233
:1036E0000221204605F0ACF901221146204605F0E2
:1036F000A7F90121204605F097F90021304605F091
:103700005CFA0021384605F058FA12B0BDE8F081A5
:1037100030B589B001214FF0805004F0F3FE012054
:1037200005F0B4FA01214FF4802004F0E0FE0F20F0
:1037300005F05CFC0446102005F058FC054601200D
:1037400004F0D2FE002004F0CFFE21460F2005F049
:1037500040FC2946102005F03CFC00214FF480205D
:1037600004F0C5FE012004F05DFE412004F00CFFD2
:103770000028FAD04FF4807004F0A0FE012004F07D
:10378000B0FE05F0D6FA3F20069040F2FF100790F9
:103790000020059005A805F083FA0020029002A9F8
:1037A00005F0E8FA00208DF8070001208DF80400EC
:1037B0008DF805008DF8060001A9002005F053FBE7
:1037C0004FF4800005F0F2FC4FF4800003900020DD
:1037D0008DF8100008208DF8110001208DF81200DE
:1037E00003A805F0A1FC03208DF800000D208DF842
:1037F000010000208DF8020001208DF8030000A8D0
:1038000005F0E1FC032005F0A2FB4FF4804005F039
:1038100058FC4FF4800005F0C9FC01214FF48040B2
:1038200005F015FC012009B030BD10B586B00121AE
:10383000084604F05CFE01214FF4804004F06DFE68
:1038400000208DF810008DF8130001200390DFF8A0
:10385000BC4703A9204604F03FFF0420039003A9BE
:10386000204604F039FF0021084605F0E5FC02215E
:10387000002005F0E1FC00208DF8080001208DF803
:103880000A0001900C208DF8090001A805F04CFCFD
:10389000042001900C208DF8090001A805F044FCDB
:1038A000042005F083FC28208DF800000F208DF8FF
:1038B000010000208DF8020001208DF8030000A80F
:1038C00005F081FC06B010BD10B586B00121084698
:1038D00004F00DFE01214FF4804004F01EFE002094
:1038E0008DF810008DF813004FF40064039403A9C1
:1038F000DFF8180704F0F0FE0B21002005F09CFC17
:1039000000208DF8080001208DF80A0001940C2099
:103910008DF8090001A805F007FC204605F046FCDB
:1039200028208DF800000F208DF8010000208DF870
:10393000020001208DF8030000A805F044FC06B049
:1039400010BD30B58DB0044601214FF4807004F0F5
:10395000E4FD00A804F0FAFE0A20009003208DF890
:10396000040000208DF8070000A9DFF8A00604F08D
:10397000B3FE05F075FC02A805F0B7FC4FF48030EB
:10398000039002A805F0A3FC06A805F096FCDFF85A
:10399000DC5A06A9284605F070FC072301222146BF
:1039A000284605F0B3FC0121284605F0F2FC012170
:1039B000284605F0A0FC0DB030BD38B5DFF8AC4AA4
:1039C000204605F0E1FC4FF47A750221204605F00F
:1039D000F7FC002803D12846451E0128F5DA2046C9
:1039E000BDE8324005F0E0BC80B50021DFF87C0A7C
:1039F00005F081FC00214FF48070BDE8044004F024
:103A00008CBDDFF8280B00687047000038B5040053
:103A100040D0012005F03AF9002005F0B2FA4FF449
:103A20000055042005F02EFB012804D12846451E30
:103A300080B20028F5D100EE104AB8EE400ADFED62
:103A4000800A80EE800AF0EE000A20EE200ADFED08
:103A50007D0A80EE800ABDEEC00A10EE100A401EFC
:103A600080B205F084FA4FF4804005F02AFB4FF451
:103A7000800005F09BFB012005F083FADFF8AC0A1B
:103A800001218160046021460FF22000BDE834402E
:103A9000FEF789BCDFF8940A00210160012005F0DF
:103AA000F5F80020BDE8324005F06BBA536574525A
:103AB0005443203D2025640030B4014601200023FA
:103AC000DFF86C2A1C469460946814F00C0FFBD14C
:103AD0000C460B2C55D8DFE804F02054545406193A
:103AE0002031383F464D946844F080049460DFF8FC
:103AF000444A4FF4C0652560146824F08074146053
:103B0000DFF8B44ADFF8305A25603BE00346DFF8BF
:103B1000A84ADFF8A85A256034E094689460DFF87A
:103B2000144A4FF4C0652560146824F08074146052
:103B3000DFF8844ADFF8885A256023E00223DFF8A3
:103B4000784ADFF8805A25601CE00323DFF8684AD2
:103B5000DFF8745A256015E00423DFF85C4ADFF8CB
:103B6000C45A25600EE00523DFF84C4ADFF8B85A46
:103B7000256007E00623DFF8404ADFF8B05A2560E9
:103B800000E01846002B4AD003EBC3030FF2B80441
:103B90001B1994689460146824F08074146014688D
:103BA00024F0806414609C781D8844EA8514DD78D4
:103BB0006D086D1E44EA05441D7944EA05645460AD
:103BC000DC881D7A2D0745EA8414DFF8BC5A2C6086
:103BD000146844F0807414601468A401FCD55B7907
:103BE00043F4C063DFF84C492360936893609368A3
:103BF0009360052904D1916841F09001916005E03E
:103C00000A2903D1916841F480519160916841F093
:103C100002019160916801F00C010829FAD1DFF8E6
:103C200098190968DFF8642A914207D2DFF8F01A80
:103C30000A6822F4404242F480420A6030BC704775
:103C400000007A4400000047200110040F03020125
:103C500003F00010060F01020103C00010080F015D
:103C6000020103C00010060F01020103F00010065C
:103C70000F01020103C80010040F02020103A80093
:103C800010020F030201030016E7002800E0401EA7
:103C9000FDD170477CB50726DE4988426BD10120F3
:103CA0008DF804008DF805008DF8060000208DF8D1
:103CB000070040200090DFF8885A00A9284604F049
:103CC0000BFD8020009000A9284604F005FD40214E
:103CD00028464183C0460F20FFF7D7FF40212846E2
:103CE0000183C0460F20FFF7D0FF3046461E80B24A
:103CF0000028ECD18020009000A9284604F0ECFCBC
:103D0000402128464183C0460520FFF7BEFF8021A1
:103D100028460183C0460520FFF7B7FF402128460B
:103D20000183C0460A20FFF7B0FF402128464183A7
:103D3000C0460520FFF7A9FF802128464183C046E1
:103D40000520FFF7A2FF02208DF8040001208DF866
:103D500005008DF8060000208DF807004020009037
:103D600000A9284604F0B8FC8020009000A928464D
:103D700004F0B2FC73BDDFF8841488426AD10120DC
:103D80008DF804008DF805008DF8060000208DF8F0
:103D900007004FF480640094DFF8A45900A9284676
:103DA00004F09AFC0820009000A9284604F094FC36
:103DB000214628464183C0460A20FFF766FF214678
:103DC00028460183C0460A20FFF75FFF3046461EA3
:103DD00080B20028ECD10820009000A9284604F009
:103DE0007BFC214628464183C0460520FFF74DFF56
:103DF000082128460183C0460520FFF746FF2146DB
:103E000028460183C0460A20FFF73FFF2146284687
:103E10004183C0460520FFF738FF0821284641832B
:103E2000C0460520FFF731FF02208DF80400012075
:103E30008DF805008DF8060000208DF8070000942D
:103E400000A9284604F048FC0820009000A9284654
:103E500004F042FC73BD10B5DFF8E848012120688A
:103E600004F067FD206804F099FC2068FFF732FB3E
:103E700005E02068FFF70EFF2068FFF72BFB4FF4EB
:103E80000031206804F060FD0028F2D110BD30B48C
:103E90000022838A008BDFF8AC48656843EA004063
:103EA0000840000255EA102060600840884200D1B6
:103EB0000122104630BC70472DE9F84F04460D46EC
:103EC00016464FF420491F78DFF878884FF4003108
:103ED000D8F8000004F038FD002808D04846A0F1CA
:103EE00001090028F2D1FFF7B6FF00208CE0D8F8D6
:103EF000000001884FF6FF52114001800121D8F8DF
:103F0000000004F0E9FC4FF4805AD1460020C8F8C4
:103F10000400D8F800B0DFF830185846FFF7B7FFB4
:103F2000002805D14846A0F101090028F1D163E03D
:103F3000D14600222146584604F0E6FC0020C8F88D
:103F40000400D8F80040DFF804182046FFF79FFF70
:103F5000002805D14846A0F101090028F1D14BE025
:103F60003146C9B220460182C046D1460020C8F879
:103F70000400D8F80040DFF8D8172046FFF787FF85
:103F8000002805D14846A0F101090028F1D133E00D
:103F9000012F15D1297820460182C046D146002044
:103FA000C8F80400DFF8AC17D8F80000FFF76FFF7F
:103FB000002823D14846A0F101090028F2D11BE0D6
:103FC0003846471EC0B2002818D015F8011BD8F893
:103FD00000000182C046D1460020C8F80400DFF886
:103FE0007417D8F80000FFF752FF0028E8D14846C0
:103FF000A0F101090028F2D1002005E00121D8F844
:10400000000004F075FC0120BDE8F28F00000240C2
:1040100000040240005400402DE9F54F81B00D46E8
:104020001E464FF420483778DFF818474FF4003128
:10403000206804F089FC002808D04046A0F101085F
:104040000028F3D1FFF707FF0020D3E020680188A4
:104050004FF6FF52114001800121206804F03CFC22
:104060004FF48059C84600206060DFF8DCA6D4F821
:1040700000B051465846FFF70AFF002805D14046D8
:10408000A0F101080028F2D191E000229DF804106F
:10409000584604F039FCC84600206060D4F800B0EF
:1040A000DFF8A8165846FFF7F2FE002805D1404673
:1040B000A0F101080028F1D179E0BDF80810C9B2DB
:1040C00058460182C046C846DFF88C16206804F0C6
:1040D0003BFC002805D14046A0F101080028F3D19F
:1040E00065E00121206804F0F7FBC846002060600D
:1040F000D4F800B051465846FFF7C9FE002805D154
:104100004046A0F101080028F2D150E001229DF8BC
:104110000410584604F0F8FB022FC84639DADFF8DD
:104120003C16206804F010FC002805D14046A0F1A0
:1041300001080028F3D13AE00021206804F0EDFBEB
:104140002068018B012104F0D3FBC846DFF810166C
:10415000206804F0F9FB002805D14046A0F10108D1
:104160000028F3D123E02068008AC0B2287030789C
:10417000401E3070C84620680188890505D5404634
:10418000A0F101080028F6D111E0012104F0C5FBDF
:104190002BE000206060DFF8CC152068FFF777FE89
:1041A000002806D14046A0F101080028F3D10020E4
:1041B00020E0012616E0012F0CD1012E0AD10026A5
:1041C0003146206804F0A9FB2068818A018B012117
:1041D00004F08EFB2068818A490603D5008A05F821
:1041E000010B7F1EFFB2002FE5D10121206804F0F2
:1041F00094FB0120BDE8FE8F801A060000580040A5
:10420000003001408429012088640240106402408B
:10421000DFF854050168082933D1DFF814130A6860
:1042200042F080720A604268B2F1806F03D10A687E
:1042300042F080620A600A689201FCD58A6842F006
:1042400002028A608A6802F00C02082AFAD14268E7
:10425000B2F1806F02D10A681201FCD5DFF8581361
:104260000968DFF82824914207D2DFF8B4140A68FD
:1042700022F4404242F480420A6000210160416021
:1042800070474168B1F1806F09D1A9490A6842F0CD
:1042900080620A600A681201FCD500214160704703
:1042A000000000000C300140DFF8C004016841F05C
:1042B00080510160DFF8680401688908890041F0D5
:1042C00001010160DFF8A8040FF2050141607047A9
:1042D00038B5DFF8A044208840F004002080FDF7C6
:1042E000E0FF807A012803D1012004F0D2FC02E033
:1042F000002004F0CEFCDFF880548021DFF87C043D
:1043000004F0A8FB002818D172B68948DFF85814C9
:10431000826802F00C020A60006800F08060486069
:10432000286840F00400286030BF62B6286820F09A
:1043300004002860FFF76CFF0CE0608840F0040088
:104340006080286820F00400286030BF286840F0B2
:1043500004002860608840F00400608031BDDFF810
:10436000100440680047DFF81814012806D010D365
:10437000032809D005D3042809D00AE0DFF8C013C8
:1043800007E0DFF8001404E0DFF8FC1301E0DFF8D9
:10439000FC130846704710B50C46FFF7E4FF2146B2
:1043A00089B2BDE8104004F0E1B910B50C46FFF742
:1043B000DAFF214689B2BDE8104004F0D9B9000007
:1043C000E0B500238DF8083001238DF80A30002A6B
:1043D00003D10C228DF8092002E008228DF8092073
:1043E00004283CD8DFE800F00315212A2A004FF406
:1043F0000060019028208DF800000F208DF801004A
:1044000000208DF80200012921D118468DF8030003
:104410001FE01846019010208DF8090006208DF845
:1044200000000E208DF80100EAE70220019007202D
:104430008DF800000F208DF80100E1E704200190C5
:1044400008208DF800000F208DF80100D8E78DF8C6
:10445000030001A804F068FE00A804F0B4FE07BD44
:104460004FF40061C64804F07AB900000020014012
:1044700010B5044601214FF4802004F038F821469D
:10448000102004F0A6FD00214FF48020BDE810406C
:1044900004F02DB810B501214FF4802004F027F866
:1044A000102004F0A3FD044600214FF4802004F006
:1044B0001EF87B2004F068F8002802D099A0FDF7D0
:1044C00072FF7A2004F060F8002802D096A0FDF771
:1044D0006AFF792004F058F8002802D093A0FDF775
:1044E00062FF7C2004F050F8002802D090A0FDF775
:1044F0005AFF7D2004F048F8002802D08DA0FDF777
:1045000052FF7E2004F040F8002802D08AA0FDF778
:104510004AFF7F2004F038F8002802D087A0FDF77A
:1045200042FF04F043F82046C0B210BDE82C012041
:1045300000380240003C024000127A003EB50C46B2
:1045400015460422014602A800F0EAF90422214699
:1045500001A800F0E5F90422294600A800F0E0F9DE
:1045600002A9002004F006FC01A9002004F07BFC55
:1045700004F074FC0446864A002300981946101A79
:1045800063EB0101490241EAD051400204F042FFCD
:104590000090844205D2011B4FF0004004F033FD2F
:1045A00037BDA04207D2C4F50070009909184FF03A
:1045B000004004F028FD37BDE06700208096980099
:1045C0000024F40000366E010048E8012DE9704334
:1045D00084B004460D46164602A9002004F019FCDA
:1045E00001A9002004F08FFC04F038FC0090684A18
:1045F000A2FB00894FEA582848EAC958A2EB0800F4
:104600000090042202A9204600F08AF9042201A9A0
:10461000284600F085F9042200A9304600F080F910
:10462000BDE87F83005A620280F0FA0200BD0105F6
:1046300070B48C1E012C01DA0C34401E3C21642520
:10464000B0FBF5F5C5EB90054FF4C876B0FBF6F678
:10465000751940F26F1674430C26B4FBF6F4641916
:10466000121940F26D1404FB00204A4A101800EBA6
:10467000400203EBC200039A01FB0020049A01FBF5
:10468000002070BC7047000084380240018793030B
:104690001CB50C4601680191416800918368C268AD
:1046A0000169491C406900F26C70FFF7C1FF20608E
:1046B000002016BD10B58EB037480068C405E40D63
:1046C00001A9002004F0A5FB00A9002004F01BFCB8
:1046D0009DF8040006909DF8050005909DF80600E1
:1046E00004909DF80100401E08909DF8020007907C
:1046F0009DF803006430099002A904A8FFF7C8FFE1
:104700004FF47A7010FB04F0400AC0F57A70039001
:10471000029A4FF47A73C117E3FB02010EB010BD89
:1047200000700040504F520050494E00424F52001E
:104730005346540049574400575744004C505700C3
:1047400000040240346800200100030082000700DA
:104750008000070084000700040000100200001021
:104760004000001002000300F42D012040380240F8
:10477000E82C01201800024010ED00E0003001405C
:104780000000024000080240000C024000100240FD
:1047900000CA9A3B7505F5FF28280040002204F066
:1047A000B1BE000008B584B00023029311B9009394
:1047B000019302E00090481E019004AB00A9074855
:1047C0007844183004F0B8FE009909B100220A704C
:1047D000002858BF029805B000BD00BF2FE6FFFFBC
:1047E00000F10103810704D010F8011B89B1810792
:1047F000FAD10268B2F10131914311F0803F04BF58
:1048000050F8042FF6E710F8011B11B110F8011B46
:10481000FBE7C01A7047000000B585B002460FF2F2
:10482000140100A805F054FD00A800F099FB05B0A4
:1048300000BD00004F45256400000000304881683D
:10484000002904BF08B008E0EFF30982A2F12802B2
:10485000036882E8F84F83685A6000F04BFD816876
:1048600059B14A6892E8F84F036002F1280282F3D6
:10487000098813F47F4F36D07047224822490968CF
:10488000401A80F308884FF08071C1611F4981612F
:104890007FF0060E704701BC2046DFF874E000BDD3
:1048A000FEE71C48006818490968401A203820F0C3
:1048B000070080F308884FF0000181F3118862B689
:1048C00000F00DF8FEE74FF0000181F31188124966
:1048D000124A0A604FF0800181F3118870470E4937
:1048E0000E4A0A6070474FF0000181F3118870474B
:1048F00000BF4FF0800181F31188704700BF0000B6
:104900002C670020E01F00205026030819A600088D
:10491000A14800080000000804ED00E000000010BD
:1049200010B50446FEF784F8204610BDEFF303806F
:104930007047BFF34F8FDFF86C06016801F4E06148
:10494000DFF8642611430160BFF34F8FFEE770B5B7
:1049500082B006460C462046FFF742FF0546202D52
:1049600005D10422314600A8FFF7DAFF06E0102D3A
:1049700016D10222314600A8FFF7D2FF002000E046
:10498000401CA8420EDA015D7829F9D0009A2B4626
:104990005B1E1B1ADA4002F0010230398A42EFD066
:1049A000002076BD012076BDDFF8001601600620EC
:1049B0007047A0F10060B0F53E3F01D8012070477C
:1049C00000207047F8B504460D460020009020688E
:1049D000FFF7EFFF00281AD000A8FFF7E5FF064613
:1049E000002700E07F1CB74211D2009850F8371022
:1049F00000EBC700406840422268520810EB4200BA
:104A0000FFF7A5FF0028EDD02F600120F2BD0020A8
:104A1000F2BDF8B50C46DFF898150A6D4B6D002510
:104A200059082E465F1B062F11D3482707FB012785
:104A30003F6C874200D20D46B84200D20B46E918BF
:104A4000490837467E1C1F2FECD300E06D1C9D42A9
:104A500011D2482707FB05210E6CB042F6D34E6CED
:104A60008642F3D34022204605F04CFC002084F817
:104A700040000120F2BD40220FF20061204605F007
:104A800041FC0020F2BDF0B591B0044600250EE0D7
:104A900032590FF2F45100A805F01AFC00A8FFF7F4
:104AA0009FFE024600A9381D05F02CFC6D1C05EB8D
:104AB000C500C600305900280BD0371900A9FFF7F0
:104AC000A8FF0028E4D0402200A9381D05F01AFCF8
:104AD000ECE711B0F0BDF8B507460C4615460026C8
:104AE00030460090002F1ED0002C09D1F2BD06EBFD
:104AF000C600C00057F8041B490849004151761C04
:104B00000C2E0FD200A93846FFF75CFF002807D112
:104B10003868FFF74EFF002802D13F1DBC42F1D29A
:104B2000BC42E4D23046F2BD70B5DFF888140A46C4
:104B30000B68D21A1368DFF88044A34201D000202A
:104B400070BDDFF86C44121D22650968091F4822F8
:104B5000B1FBF2F1616510F1030F02D010F1130FF8
:104B60000AD1DFF85854A86805F002FC0646A86888
:104B700005F00AFC811905E005F014FC054605F076
:104B800013FC4119DFF83854A069286005F1480288
:104B9000A06AFFF7A0FF2846FFF775FF012070BD50
:104BA0000EB430B5CCB0044600A84FF49671FFF7B0
:104BB000F5FD00254FAB22464FF4967100A8FFF794
:104BC000F1FD00A8FFF70CFE044609E0DFF8E01352
:104BD000C86D421CCA6500A9695C05F04DFC6D1CDE
:104BE000A542F3D34CB030BC5DF810FB38B50024BF
:104BF000DFF8BC53E8650FF29840FFF7D1FFDFF80C
:104C0000C40301680FF2AC40FFF7CAFFA86C009024
:104C1000AB6B6A6B296B0FF2B440FFF7C1FFE96C15
:104C20000FF2E040FFF7BCFF6A69A9690FF2E840A4
:104C3000FFF7B6FF0FF2F840FFF7B2FF06E01018DB
:104C4000021D0FF20450FFF7ABFF641C04EBC4001D
:104C5000C200DB4811580029F1D10FF2F840FFF7EC
:104C60009FFFA86D441E002505E00918BBA0FFF7B3
:104C700097FF641E6D1C3C2D09D2002C00D53B24EF
:104C8000322000FB04F1D0480A5C002AEDD131BD8E
:104C9000CE48CF490A6802604A6842608A688260EA
:104CA000CA68C2600A6902614A6942610A7E826119
:104CB000097F8161C7490A7882614A6842628A68CD
:104CC0008262CA68C2620A6902634A6942638A6987
:104CD0008263CA69C2638A6EC0F88820BE4A93693B
:104CE000C0F89830D368C0F88C301369C0F89030A1
:104CF0005369C0F894300B6FC0F89C304B6FC0F80C
:104D0000A0308B6FC0F8A430C96FC0F8A810B349A9
:104D10000968C0F8AC10B2490B68C0F8CC304B68D9
:104D2000C0F8D0308B68C0F8D430CB68C0F8D83029
:104D30000969C0F8DC105168C0F8E8101168C0F8C3
:104D4000E410704770B506460C46994D6FF01E0191
:104D5000401A14D0083812D0001F05D0001F0ED002
:104D600008380CD0001F10D104F120002862EFF3A6
:104D7000148040F00200E862286AA86205E004F1AD
:104D800020002862EFF31480E862EFF30880686285
:104D9000EFF305802863EFF300806863FFF7C6FD3B
:104DA000A863EFF31080E863EFF311802864EFF35A
:104DB00013806864F1EE100AA864EE64002004E039
:104DC00054F8201045F82010401C0828F8D370BD76
:104DD00070B5774CA16D3C2901D30021A165A56D6B
:104DE0003221794A01FB05260A4601463046FFF783
:104DF00097FD002086F83100681CA06570BD70B575
:104E0000014674462046FFF79DFFFFF741FF20460D
:104E1000FFF78AFE00F09AF8002832D100F034F84B
:104E200005F0CAFAF32005F041FB6E484FF000543C
:104E3000002505E02178641C05F01EFB30466D1C42
:104E4000461CB5F5C03FF5D3532105F015FB5221A3
:104E5000304605F011FB741C4121204605F00CFB87
:104E6000641C4D21204605F007FB5F48C046C04644
:104E700004F10D00FFF7BAFE05F0A7FA5B4800F059
:104E80001FF8BDE8704054E510B505F095FAF32021
:104E900005F00CFB564C3820206002E020680830FA
:104EA00020602068402807D2002105F094FA0928E4
:104EB000F4D0FFF73EFDFCE7BDE8104005F085BAF1
:104EC00038B5044605F078FAF32005F0EFFA3D48CE
:104ED0000168204605F0B4FA241DFF21204605F0A4
:104EE000CBFA641C404D6979204605F0C5FA641C74
:104EF000E978204605F0C0FA641C2979204605F0BF
:104F0000BBFA641C2978204605F0B6FA641C69785F
:104F1000204605F0B1FA641CA978204605F0ACFAE9
:104F2000F521601C05F0A8FABDE8314005F04DBA46
:104F300080B505F041FAF32005F0B8FAAA212D4812
:104F400005F09AFABDE8014005F03FBA0020294972
:104F50000978F52900D101207047000025730A0067
:104F600010B50446FFF73CFCC0B2142800DB132048
:104F7000024621462048FFF7D3FC4FF0AC300078C2
:104F800010BD80B500F049F8BDE80140D1E480B51E
:104F9000FFF7CEFF4FF4C83212490020BDE80840A9
:104FA00002F0EDB80CED00E00400FA05CC6600203C
:104FB000901E0120FC4F0508FECAFECA2C67002087
:104FC00064EB00205068002034B30020C40C0120A2
:104FD00000ED00E020ED00E004E000E0A0ED00E0E6
:104FE00034EF00E000000608EC2D0120F4FF070874
:104FF000802E0120FFFF0708842B012010B500F050
:105000001BF80FF270142046FFF7EAFB0246214618
:105010000020BDE8104002F0B2B880B501214FF485
:10502000802003F064FA012003F030FE94210F2069
:10503000BDE8044003F0CDBF80B501214FF48020CE
:1050400003F055FA012003F021FE00210F20BDE8F6
:10505000044003F0BEBF10B5002401214FF48020AE
:1050600003F045FA012003F011FE0F2003F0BEFF0C
:10507000942800D10124204610BD00004E6F20531B
:10508000796D626F6C000000307825303878000050
:105090000A0A0A0A3D3D2043726173682044756D17
:1050A0007020496E666F726D6174696F6E203D3D50
:1050B0000A0000004669726D77617265205665725C
:1050C00073696F6E203A2025640A00000A49505324
:1050D00052203D20307825782C2041505352203DDD
:1050E00020307825782C2078505352203D2030787D
:1050F00025782C205046534352203D203078257887
:105100000A0000000A6661756C74206D6F6465208A
:105110003D203078257800000A5043203D2030782B
:1051200025782C204C52203D20307825780A00002C
:105130000A3C43726173682043616C6C2053746154
:10514000636B3E0A0000000030782578202025732C
:105150000A0000000A0A3D3D20526563656E742016
:105160004C6F67204D65737361676573203D3D0A21
:1051700000000000534E414D5900000000000000A7
:1051800038B5FFF7B6FBDFF830068468DFF828068D
:1051900000210171FFF7A7FB002C2CD0206800280C
:1051A00029D0607C2168497CC0B2814223D1256826
:1051B00000E00D002968002903D04A7CC0B2824279
:1051C000F7D0FFF796FBDFF8F0050069A04203D1A6
:1051D000DFF8E40521680161E06921680160C861C8
:1051E000E56129682160002900D0CC612C6095F828
:1051F000410085F84000FFF776FB31BD10B5FFF7A1
:1052000078FBDFF8B8050468DFF8AC05006A201AFF
:10521000012832DADFF8A005046A04E0DFF8980517
:105220000462FFF760FBDFF898050078C00722D51D
:10523000FFF75FFBDFF8880500788007EED5DFF821
:105240008005007810F0FD00DFF874150870FFF796
:105250004AFBDFF86405006A8442FAD0DFF858059B
:105260000462DFF858050068401CDFF8501508603C
:10527000DFF844154862FFF73CFB10BD38B5040069
:105280000020A071206A10F57A606062E069002851
:1052900002D02000E1698847FFF725FBE56809E0B7
:1052A000E868616A401A002801D5E8686062FFF783
:1052B0001AFB2D68002D1AD0FFF71BFB2069002870
:1052C00004D0687C2169497C884212D3287C40073D
:1052D000EDD5E868216A401A0128E1DA280000F0DB
:1052E0009EF9FFF706FB287C0028D9D101E0FFF7E3
:1052F00000FB31BD70B504000020607001202070FB
:1053000005F050F80078C0B2CD2802D07D20FFF71C
:1053100083FAA06800280CD0A068406C002808D050
:10532000A068406C01680800002802D0A0684068AE
:10533000884794F8290000280BD0A06894F828101A
:1053400080F84010DFF870040079002801D0FFF7E2
:1053500017FFDFF870040078002823D0DFF8680416
:105360000068DFF85414096A401A002804D5DFF8F1
:1053700054040021017015E0FFF7BBFA05F05AF95B
:105380000500FFF7B0FAA068002808D0A068406BBD
:105390002818DFF838140968401AA1684863DFF854
:1053A0002C040560A068002808D0A068007C0028B4
:1053B00004D1A068006B401CA16808632069002824
:1053C0002BD003E030682061FFF78DFAFFF791FAE8
:1053D0002669002E27D0357CEDB2002D23D068073A
:1053E00010D5F068216A411A012906DA300000F070
:1053F00016F9307C002805D10FE0616A411A0029B6
:1054000000D56062EDB215F0FB001028DAD1B0686B
:1054100080684068007C0028D4D1FFF76AFA02E077
:105420002000FFF72BFFA0790028F9D1DFF89003C7
:105430000078C00701D5FFF7E1FE00206071206908
:10544000002839D02069007C002805D020698068B8
:1054500080684068A06001E02069A060A06890F8C2
:105460004C00642802D08020FFF7D6F9A068806A3B
:105470000078CD2802D07820FFF7CEF9A068406CE4
:10548000002808D0A068406C41680800002802D0BD
:10549000A06840688847A06890F8400084F8280019
:1054A00084F82900DFF810038068C06A401CDFF828
:1054B00008138968C8620BE0002084F829000020E6
:1054C00084F828000020A06000202070FFF70BFA6D
:1054D000200070BD80B505F0DBF8DFF8F412097824
:1054E000002806D0022810D009D3042815D010D3E4
:1054F00014E0002902D0A320FFF78EF911E0002963
:1055000002D1A420FFF788F90BE0A620FFF784F969
:1055100007E0A720FFF780F903E002E0A820FFF7EB
:105520007BF901BD10B505F0B3F80400DFF8A00267
:105530000078002802D0A020FFF76EF9002C05D0DB
:10554000022C08D003D3032C09D00CE00EE0A420D9
:10555000FFF762F90AE0A620FFF75EF906E0A72050
:10556000FFF75AF902E0A820FFF756F910BD80B501
:1055700005F08EF8002805D0022808D006D30328AD
:1055800009D00CE0A320FFF747F90BE00AE0A620C2
:10559000FFF742F906E0A720FFF73EF902E0A82056
:1055A000FFF73AF901BD80B5DFF80C02007800285A
:1055B00002D19720FFF730F9DFF8FC010078401E98
:1055C000DFF8F4110870C0B2002827D1DFF8E80135
:1055D0004068002822D0FFF78CF9DFF8DC01406832
:1055E00000280BD0DFF8D00101210170DFF8C801DD
:1055F000FFF769F9DFF8C00100210170DFF8B80199
:105600004078F021084202D09920FFF705F9DFF831
:10561000A8014078002801D1FFF765F901BD10B558
:10562000816800290CD0DFF89011096AC160816897
:105630000A684968002A00D051600A600021816030
:10564000017C11F003010174C9B2002945D1DFF8D2
:1056500068110969002929D1DFF85C110861DFF8B8
:105660005801007800280CD1DFF84C0101210170AD
:10567000DFF84401FFF727F9DFF83C010021017052
:1056800003E0DFF8340101214171DFF82C0140789B
:10569000F021084202D09920FFF7BEF8DFF8180188
:1056A0004078002801D1FFF71EF916E0427C4B7CC0
:1056B000D2B29342D0D38142D1D04B7CD2B29A4263
:1056C0000BD10300FFE71B68002BDED05C7CD2B25D
:1056D000A242DAD18B42F6D1BEE710BD10B504006C
:1056E000627C35480078401C33490870394800E036
:1056F00008000168002903D04B7CD2B29A42F7D34C
:105700002160E061046000290AD0CC61487CD2B2FB
:10571000904202D194F8410000E0002084F840005B
:10572000207C002812D1FFF7E4F82000FFF777FF74
:1057300021484078F021084202D09920FFF76CF808
:105740001D484078002801D1FFF7CDF8FFF72BFF67
:1057500010BD10B51848047817480078401C164949
:1057600008701548FFF7AFF81348047012484078E6
:10577000F021084202D09920FFF74EF80E484078F9
:10578000002801D1FFF7AFF810BD10B504F086FF77
:1057900009480121017004F005FE04006846C04676
:1057A000021B203A012A03DBCD212000FCF756FD25
:1057B00009480121017010BD2C670020C02E012076
:1057C000132F0120142F0120D82E0120C42E0120D8
:1057D000152F012038670020172F0120506002602C
:1057E0004160086070470A68F8E7486001607047E8
:1057F00001684068F9E7F8B50600DFF8C05802D53F
:1058000005F15800F2BD05F158040020296F00E0B1
:10581000096805F17002914204D00C46A2689642D4
:10582000F6D10120002840D1A86FD0F88070182050
:1058300004F058FF0446A660002F05D0B74203D2FB
:10584000B6FBF7F0784300E03046E060002F02D06E
:10585000B74200D23E46266100202075DFF860681E
:105860003078401C30707078F021084202D09920C6
:10587000FEF7D2FFFFF73DF87078401C707005F11D
:1058800070012046FFF7AFFF7078F021084202D088
:105890009920FEF7C1FF7078401E7070C0B20028DA
:1058A00001D1FFF720F8FFF77EFE2046F2BD38B5A4
:1058B000044694F91400002829D1DFF80458287808
:1058C000401C28706878F021084202D09920FEF729
:1058D000A3FFFFF70EF86878401C68702046FFF7BA
:1058E00087FF204604F016FF6878F021084202D0B6
:1058F0009920FEF791FF6878401E6870C0B20028BA
:1059000001D1FEF7F0FFBDE83140FFF74CBE31BDDD
:10591000F8B5044608466FF00045FFF76CFF0646F1
:1059200094F9050094F90410814214D1C01C800040
:1059300004F0D8FE074694F90500012807DB820031
:1059400021683846FEF7ECFF206804F0E3FE27608C
:105950006079C01C607194F90400411C21712168B8
:1059600041F82060DFF85C07864202D0307D401CA1
:105970003075002008E0216851F820108A689542AF
:1059800001DB1546A160401C94F904108842F2DB4B
:10599000F1BDF8B504466FF00046DFF8202702F1AC
:1059A000580502F158004FF0FF33002704E0664528
:1059B00001DB664675467F1C94F904C067450DDA25
:1059C000D4F800C05CF827E0DEF808C0002BEED564
:1059D0008C45ECD170463B465BB2ECE7002B11D412
:1059E000BCF1010F0EDB06E0216801EB830676684F
:1059F00041F823605B1C94F904104E1EB342F3DBA4
:105A0000491E217102F15801884204D0017D491ECE
:105A10000175FFF74CFFA560F1BD10B4C26A836B3E
:105A2000406C9C68002C02D56FF0004300E01B69BD
:105A30008468002C02D56FF0004000E000699842B5
:105A400000DD1846D2685143884201DB012000E0A6
:105A5000002010BC704738B5DFF860168A6FD36E2F
:105A6000012490F90850AC402343D36601F66C1131
:105A7000FFF7B9FE012032BD10B5DFF84016896F7F
:105A8000CA6E012390F90840A3409A43CA66FFF703
:105A9000AFFE012010BD012070472DE9FC410446F6
:105AA0000D4616461F4604F12400FFF731FF07EBB1
:105AB000470004EB8008314608F13000FFF728FF6B
:105AC000019598F9340000903B46627A94F90810E9
:105AD0000FF2F450FCF767FCBDE8F3812DE9FC41BF
:105AE00004460D4616461F4604F12400FFF751FFF9
:105AF00007EB470004EB8008314608F13000FFF760
:105B000048FF019598F9340000903B46627A94F979
:105B100008100FF2C850FCF746FCBDE8F381C16ADB
:105B20008A68012A09DB0969012906DA006D002863
:105B300001D500207047022070470020704701EB1C
:105B4000410200EB8201896B8A68012A09DB09693D
:105B5000012906DA006D002801D5002070470220D7
:105B6000704700207047002900D5D8E7E7E70129F2
:105B700000DA012113460A468FE7012900DA0121E4
:105B800013460A46AAE7DFF83405C06A417A481E80
:105B90008041C00F704713464FF0FF3211467CE73B
:105BA00013464FF0FF32114698E780B5DFF80C0539
:105BB0000068417A002902D1006E406880470120C8
:105BC00002BD80B5FFF758FFDFF8F0040068417AA6
:105BD000002902D1006E80688047012002BDB1F526
:105BE0007A7F01DC4FF47A7113460A464FF4FA715A
:105BF00053E7B1F57A7F01DC4FF47A7113460A4618
:105C00004FF4FA716AE710B50446002922D5E06A1C
:105C1000816801291CDB0069012819DA022120466C
:105C2000FFF7FBFE002813D194F9540010F1010F87
:105C300004D1002084F85400012010BD002807D1B1
:105C4000012060774FF0FF3084F85400022010BD2F
:105C5000002010BDBDE8104071E74FF0FF3280F822
:105C60005420F8E6DFF85424926FD2F88020A03256
:105C700052420265EFE600290AD5C06A816801290F
:105C800004DB0069012801DA022070470020704718
:105C900055E7B52900DAB42113460A463C21FCE653
:105CA000B52900DAB42113460A463C2116E710B59F
:105CB0000446002927D5E06A8168012921DB0069B3
:105CC00001281EDA03212046FFF7A7FE002818D17D
:105CD00094F95400014611F1010F04D1002084F819
:105CE0005400012010BD002803D1012084F8540085
:105CF00010BD012905D14FF0FF3084F85400022077
:105D000010BD002010BDBDE8104018E74FF0FF3275
:105D100080F85420DFF8A423926FD2F88020B432A8
:105D20005242026597E6DFF89423926FD2F8802002
:105D3000C832524202658EE613464FF0FF321146DA
:105D4000ABE613464FF0FF321146C7E680B5FFF7CA
:105D500082FEFCF7A6FA00210175012002BD80B584
:105D6000FFF78AFEFCF79DFA00210175012002BDB4
:105D70002DE9F0410C46D14D55F82060307206F106
:105D800054070FF26C313961152800F22F81DFE8DA
:105D900010F0160026003300530043006200730029
:105DA0008200B2009200A200C200D200E000EC002B
:105DB000F90007011401210121012101210106F14E
:105DC0000800062141760A21817605F674114160AA
:105DD00040F2DC5181600FF23430386106E106F1A7
:105DE0000800062141760A21817605F6507141604E
:105DF0004FF496718160F9E006F108000C214176BC
:105E00001021817605F5805190314160102181602B
:105E10000FF24C303861E9E006F1080007214176C5
:105E20000B21817605F58051843141600B21816021
:105E30000FF22C303861D9E006F1080006214176D6
:105E40000A21817605F5855141600A2181600FF2B2
:105E500010303861CAE006F10800062141760A21B7
:105E6000817605F58051AC3141604FF4FA71816063
:105E70000FF208303861B9E006F1080014214176CC
:105E80001821817605F595514160182181600FF246
:105E90005C303861AAE006F1080002214176062153
:105EA000817605F59051D4314160062181600FF271
:105EB000043038619AE006F108000A2141760E218B
:105EC000817605F59051C43141600E2181600FF259
:105ED000C82038618AE006F10800012141760521D9
:105EE000817605F59051DC314160052181600FF22A
:105EF000E02038617AE006F10800052141760921A9
:105F0000817605F59051B8314160092181600FF229
:105F1000342038616AE006F10800062141760A2142
:105F2000817605F59051E43141600A2181600FF2DC
:105F3000F81038615AE006F1080001214176052188
:105F4000817605F59051F031416040F286618160C3
:105F50004CE006F10800012141760521817605F526
:105F6000CC5141600521816040E006F108000C2120
:105F700041761021817605F5C851883141601021A4
:105F8000816033E006F10800112141761521817608
:105F900005F5C8519831416040F63401816025E033
:105FA00006F10800112141761521817605F504518D
:105FB000CC3141601521816018E006F10800042110
:105FC00041760821817605F5C85178314160082174
:105FD00081600BE006F10800012141760521817600
:105FE00005F580517C3141600521816006F1080092
:105FF00000210175417581750176C16001614170B3
:1060000006F128080846C8F828004FF0FF3086F847
:1060100054007880062206F15800FCF71FF9002092
:1060200010E000EB400106EB8101002281F83420F2
:1060300034314A7005F158024A6006EB80010022B3
:106040008A64401C0228ECDB002086F8280088F8CF
:10605000010005F15800C8F80400FC60BDE8F081BB
:1060600010B5164C04F066FBA067002006E068211E
:1060700011FB00417C3144F82010401C1628F6DB4F
:106080004FF0FF30206660660020A06605F0EAFD54
:1060900006F04AFC07F0DBF808F056F809F0FCF9C6
:1060A00008F04AFB08F0CDFD09F060FA09F0AFFDF9
:1060B00009F061FABDE8104009F06EBA084000200E
:1060C0002C67002060400020414420256420256486
:1060D0002025642025642C2025640000524D2025B5
:1060E00064202564202564202564202564000000A8
:1060F000975A0008575A0008975A0008795A00081A
:106100006F5B00087B5B0008675B0008875B00082B
:10611000575A0008875B0008795A00086F5B00082F
:106120007B5B0008675B0008AB5B0008575A000800
:10613000975A0008C35B0008975B0008A15B000842
:10614000675B0008975A00085B5C0008975A0008D4
:10615000795A0008DF5B0008F35B0008075C000861
:10616000975A0008655C0008975A0008795A000899
:106170006F5B00087B5B0008775C0008975A00089B
:106180000D5D0008975A0008795A0008935C0008D2
:10619000A15C0008AF5C0008975A0008275D000862
:1061A000975A0008795A00086F5B00087B5B00086B
:1061B000675B0008975A00084D5D0008975A000871
:1061C0005F5D0008395D0008435D0008675B0008FB
:1061D000975A0008575A0008975A0008795A000839
:1061E0006F5B00087B5B0008675B0008975A00083C
:1061F000575A0008975A0008795A0008395D000874
:10620000435D0008675B0008DFF8280E00787047E0
:106210002DE9F0418AB004F08DFA0446DFF8185EEB
:106220002E6842E096F9080007283DD00B283BDA9B
:10623000062839D006F10807B86C002803D5D4F831
:1062400080100818B8644FF0FF313046FA6D92693B
:1062500090478046B8F1010F04D197F84C00B96D12
:1062600009698847B8F1020F0BD1797E38697A68DD
:106270008018BA6D52699047002802D0304609F064
:1062800013FE00213046FA6D92699047022801D131
:106290000120B87501213046FA6D926990470228B5
:1062A00002D1304609F0ACFE3668AE42BAD1D4E92C
:1062B0001C01002901D100280CD00A208DF808000B
:1062C00002208DF80000D4F88000ADF8220000A86C
:1062D00001F00AFF01200AB0BDE8F08130B585B0B9
:1062E00004460D46CA208DF800002888ADF801004C
:1062F0000220ADF80300BDF80100001D04F0F2F922
:10630000CDF8090002220DF10301FEF709FB02227C
:106310002946DDF80900801CFEF702FB2A88214689
:10632000DDF80900001DFEF7FBFA0020288000A917
:10633000DFF8F00D0AF066F905B030BD42F2341115
:10634000081A322801DA012070470020704780B512
:10635000FBF7A7FF407B002804D009F0FDFCDFF825
:10636000C81D086001BD80B509F0F6FCDFF8BC1D52
:10637000086001BDDFF8B40D0068704710B582B049
:1063800000F10C03D96A89680091042200A95C7DA0
:10639000DB68C06818182018FEF7C2FA13BD30B4C5
:1063A0001488651C1580052565541488651C1580A6
:1063B000635413885C1C1480007A585430BC7047B6
:1063C00032B515461C4621884A1C228037224A5580
:1063D00021884A1C2280007A4855022200A9208880
:1063E0004019FEF79DFA2088801C208031BDF8B549
:1063F00017461D4600F10C06069CA4B2B27D62430E
:10640000C06809182888C019FEF78AFA2888B17D63
:10641000614311FA80F02880F1BD30B400F110031F
:106420009B7C914203D1006990FBF3F00DE00C4698
:10643000154603D2281B90FBF3F006E00069001B11
:1064400090FBF3F095FBF3F1081880B230BC704775
:1064500000F110018A688B7CD2188A600069824240
:1064600001D10020886000208873704770B582B029
:1064700004460D461E4692B289B2FFF7CEFF009049
:10648000069B324629462046FFF7B1FF73BDF8B59B
:10649000044615461E462269002D00D11546069F6A
:1064A0000097FFF7E3FF2069854206DA009733463D
:1064B0002A4600212046FFF7D9FFF1BD2DE9FC4116
:1064C00004460D461646A1696069002815D50027C7
:1064D0000A4692B289B22046FFF79FFF80463346B4
:1064E0002A4641462046FFF76BFFA26900962B46DD
:1064F00011462046FFF7CBFF2EE0814216DA012736
:106500000A4692B2014689B22046FFF786FF8046CE
:1065100033462A4641462046FFF752FF00962B4657
:10652000A26961692046FFF7B2FF15E002270A461B
:1065300092B2014689B22046FFF76FFF804633468C
:106540002A4641462046FFF73BFF00962B46A269AC
:1065500061692046FFF78AFFA06901906069009099
:106560003B46424694F908100FF20800FBF71BFF68
:10657000BDE8F3815061636B203D256420256420D4
:1065800025642025642025640000000070B582B0D9
:1065900004460D461646A06C012811DAA07F01289A
:1065A00011D133462A4601212046FFF709FF012079
:1065B000009033462A46A1692046FFF718FF02E003
:1065C0002046FFF77BFF0123324629462046FFF78E
:1065D000E6FEA0696061A36CE26C94F908100FF20A
:1065E0000C00FBF7E0FEA06CE06473BD666C757395
:1065F0006820256420256420256400002DE9F843E7
:1066000004460D46164604F095F88146FBF749FE10
:10661000804604F10807B87D002802D02046FFF725
:10662000ADFE386C0128C0F2888098F80E00002872
:1066300044D0B87D002800F0C280786CD9F8801072
:10664000401A7864B87E3969FA68531A834205D0D3
:10665000002A2FD1BA68511A81422BD194F908200F
:10666000397E0FF26010FBF79EFE397E00291ED0A6
:1066700094F908200FF26410FBF795FE3869B97E93
:10668000421892B2F96889B22046FFF7C6FE334637
:106690002A4601462046FFF793FE00962B463869AE
:1066A000B97E4218F9682046FFF7F1FE02E04FF08C
:1066B000FF30F8602046BDE8F243C9E698F80E00C6
:1066C00000287CD1786CD9F88010401A78640128B1
:1066D0002CDA386C7864386BD0F80C8094F9083078
:1066E0008268396C0FF21010FBF75DFEB868B97E56
:1066F00090FBF1F0396C91FBF8F1814202DB4FF035
:10670000FF30F860B87D00280AD02046FFF7A0FED1
:10671000324629462046FFF7D1FE3869F8604EE040
:10672000324629462046BDE8F843C7E6B87D002832
:1067300045D02046BDE8F2438AE6B87D00283ED029
:1067400094F9080098F80A10002919D0072801D0F8
:106750000D282FD133462A4601212046FFF730FE6F
:106760000120009033462A4639692046FFF73FFE54
:106770007A7894F908100FF29400FBF714FE19E0F0
:10678000092809D194F85E10012905D10FF28C0077
:10679000BDE8F443FBF707BE33462A4601212046F5
:1067A000FFF70EFE0120009033462A463969204645
:1067B000FFF71DFE2046FFF74BFE3869F860BDE885
:1067C000F183000073757370656E64206669666F8F
:1067D0002066756C6C2025642025640073757370C9
:1067E000656E64206669666F2066756C6C20322069
:1067F00025642025640000006669666F2066756C5C
:106800006C332025642025642025640041502053EA
:10681000757320256420256400000000233E6C75FC
:10682000785F73617420256400000000F8B50446A9
:106830000D46DFF80468376805E02A4621463846E9
:10684000FFF7DCFE3F68B742F7D1F1BD2DE9F0411B
:1068500004460D46DFF83C6CF76907F10C0898F820
:106860001510D8F80C00FA688018D8F8542052692E
:10687000904700280AD0012088F81200787A002872
:1068800004D02A4621463846FFF7B8FEB66906F11D
:106890000C07797DF868F26880187A6D5269904724
:1068A000002809D00120B874707A002804D02A4644
:1068B00021463046FFF7A2FE0120BDE8F0810288A4
:1068C000D21C02800A80704780B50B889B1AADF8F5
:1068D0000030BDF80030002B09D01018012100F85D
:1068E000031C022200A9801EFEF71AF801BD0888C9
:1068F000C01E088001BD2DE9F04FADF64C1D0446C9
:106900000D4603F017FF0746FBF7CBFC804610A8A7
:1069100040F60811FDF742FF00208DF8020006A89E
:106920002821FDF73BFF01A81421FDF737FF0020C8
:10693000ADF800000646D7E91C01002902D1002865
:1069400000F0748398F909000AF02FFB002800F08A
:106950006D8300A92846FFF7B2FFB0461CE0D7E9D7
:106960001C0142460AF030FD00F0010011F0000168
:1069700001D100280ED008EB8800DFF81C1B01EBCA
:10698000C00292F90900012804D10DF1020110A8FA
:10699000126A904708F10108B8F12D0FDFDB374686
:1069A0001AE02888411C298099F80210015528888E
:1069B000FFF7C4FC00280DD0BDF800202946204672
:1069C000FFF782FF29462046FFF788FC00A92846EA
:1069D000FFF775FF7F1C7FB29DF80200874280F2AF
:1069E0001D832988481C288040F2211010FB07F0E5
:1069F00010AA825C0A5529884A1C2A8010AA00EB3A
:106A0000020898F8010008552888411C298008F1DF
:106A1000010999F80110015599F8010003281ED0C9
:106A2000092800F049810C2800F023811A2800F081
:106A300042821B2800F056811C2800F070821D281D
:106A400000F063811E2800F05A82252800F0998208
:106A5000262800F0D382282800F0AE82A1E798F81B
:106A60000100032805D12888411C298099F80210CB
:106A700001552888411C298099F80310015599F87F
:106A80000300C0280DD1B8F83020D8F8321028887B
:106A90000019FDF745FF2888B8F83010081828803D
:106AA00085E7711C00064ED401A808F10402527853
:106AB0003254C9B298F806200A54491CC9B20022BF
:106AC0000A544A1C08F20601D2B24B781354521CE5
:106AD000B8F80E30D2B21E0A1654521CD2B2135459
:106AE000521C08F20E03D2B29E781654521CD2B237
:106AF000DB781354521CD2B298F812301354521C43
:106B0000D2B298F813301354521CD2B28B7813546B
:106B1000521CD2B2C9781154511CC9B298F80A203B
:106B20000A54491CC9B298F80B200A544E1CF6B2FC
:106B3000324601A928880019FDF7F2FE288850FA8C
:106B400086F0288033E7D8F8052006A8130C3354C4
:106B5000C9B2130A0B54491CC9B20A54491CD8F8CB
:106B60000920C9B2130C0B54491CC9B2130A0B54A7
:106B7000491CC9B20A54491CD8F80D20C9B2130CDB
:106B80000B54491CC9B2130A0B54491CC9B20A540C
:106B9000491CD8F81120C9B2130C0B54491CC9B2B6
:106BA000130A0B54491CC9B20A54491CD8F82720AF
:106BB000C9B2130C0B54491CC9B2130A0B54491C1B
:106BC000C9B20A544A1C08F22701D2B20B791354F5
:106BD000521CD2B24B791354521CCB88D2B21E0A2B
:106BE0001654521CD2B21354521CD2B2097A115408
:106BF000511CD8F81520C9B2130C0B54491CC9B24A
:106C0000130A0B54491CC9B20A54491CD8F819205C
:106C1000C9B2130C0B54491CC9B2130A0B54491CBA
:106C2000C9B20A54491CD8F81D20C9B2130C0B5420
:106C3000491CC9B2130A0B54491CC9B20A54491C55
:106C4000D8F82120C9B2130C0B54491CC9B2130A3D
:106C50000B54491CC9B20A544E1CF6B2324606A95E
:106C600028880019FDF75CFE288850FA86F02880F5
:106C70009DE608F10301B1F90300C0F3072242EADF
:106C80000020A1F80300B1F90700C0F3072242EA8F
:106C90000020A1F80700B1F90500C0F3072242EA7D
:106CA0000020A1F80500092228880019FDF738FE08
:106CB0002888093028807AE62888034698F8011049
:106CC000032909D1022208F103011819FDF728FE52
:106CD0002888801C28806AE6401C288099F80200D9
:106CE000185564E62888411C298099F8021001553E
:106CF00098F8010005287FF45AAE2888411C2980A5
:106D000008F104014978015551E608F1030998F8A2
:106D10000100012840F0BF802888411C298099F893
:106D2000041001554FF0000A9CE01B2010FB0A9B49
:106D3000DBF80C20DBF808100FF20030FBF733FB18
:106D4000DBF81800010221F0FF11000A00F0FF102B
:106D50000843CBF818004FEA3040CBF81800042263
:106D60000BF1180128880019FDF7DAFD2888001DAD
:106D70002880DBF80800010221F0FF11000A00F072
:106D8000FF100843CBF808004FEA3040CBF808006A
:106D900004220BF1080128880019FDF7C1FD28889D
:106DA000001D2880DBF80C00010221F0FF11000A11
:106DB00000F0FF100843CBF80C004FEA3040CBF84E
:106DC0000C0004220BF10C0128880019FDF7A8FD26
:106DD0002888001D2880DBF81000010221F0FF1137
:106DE000000A00F0FF100843CBF810004FEA3040D3
:106DF000CBF8100004220BF1100128880019FDF7D0
:106E00008FFD2888001D2880DBF81C00010221F07E
:106E1000FF11000A00F0FF100843CBF81C004FEAF6
:106E20003040CBF81C0004220BF11C01288800190B
:106E3000FDF776FD2888001D2880BBF81600010AA2
:106E400041EA0020ABF8160002220BF11601288857
:106E50000019FDF765FD2888801C28800AF1010AC9
:106E60005FFA8AFA99F804008245FFF65EAFB8F837
:106E70001B21D8F81D1128880019FDF751FD28881D
:106E8000B8F81B1108182880B8F81B110FF2BC10B5
:106E9000FBF789FA8BE505287FF489AD2888411C2A
:106EA000298099F8021001552888411C298099F8F9
:106EB000031001557BE508F1030198F80100032850
:106EC00005D12888421C2A8098F80A200255D1F85A
:106ED0000100020222F0FF12000A00F0FF1010432E
:106EE000C1F801004FEA3040C1F8010007222888AC
:106EF0000019FDF715FD2888C01D288057E508F109
:106F000003010888020A42EA002008800222288839
:106F10000019FDF705FD2888801C288047E508F149
:106F2000030098F8011001297FF441AD99F802108F
:106F3000012918D129884A1C2A8000780855B8F8F8
:106F40000420D8F8061028880019FDF7E9FC2888E5
:106F5000B8F8041008182880B8F804100FF20010D0
:106F6000FBF721FA23E502297FF421AD29884A1C89
:106F70002A8002780A5529884A1C2A80C079085537
:106F800015E52888411C2980B9F802100155288888
:106F9000411C2980B9F9021009120155B9F90220E2
:106FA000D8F8051028880019FDF7BAFC2888B9F927
:106FB000021008182880FAE42888411C2980B9F8B2
:106FC000021001552888411C2980B9F902100912C4
:106FD00001552888411C298008F104014978015590
:106FE000B9F90220D8F8061028880019FDF798FC96
:106FF0002888B9F9021008182880D8E408F103019C
:107000000888020A42EA0020088002222888001923
:10701000FDF786FC2888801C2880C8E4BDF8002085
:1070200029462046FFF750FC09F0EDFF0DF64C1DF8
:10703000BDE8F08F0F2F0120744900204C54204EE2
:107040004D47202564202564000000004F4A483A3F
:1070500020415442442073697A653A202564000037
:107060004F4A483A20415044522073697A653A2089
:10707000256400002DE9F04105460E46FBF711F9A5
:107080000746DFF818442078401C20706078F02113
:10709000084202D09920FDF7BFFBFDF72AFC60787B
:1070A000401C607097F81880B8F1000F26D0308827
:1070B000404480B2FFF742F9002803D03146284609
:1070C000FFF70CF93088411C31800321415530888D
:1070D000411C318000F80580424607F119013088D3
:1070E0004019FDF71DFC308840443080FF2200210C
:1070F00007F11900FBF7B2F8002038766078F0212C
:10710000084202D09920FDF787FB6078401E60702E
:10711000C0B2002801D1FDF7E6FBBDE8F041FEF763
:1071200042BA00008C6A0020B02E0120B42E01204B
:1071300038B504460D46FBF7B4F8817A002909D129
:10714000417B002906D129884A1C2A8006220A553B
:107150000121417331BD38B504460D462888002809
:107160000CD02046FFF786FF29462046FFF7E0FFB8
:1071700029462046BDE83440FFF7B0B831BD14B50C
:1071800085B0049101A90022134614461CC10A21AE
:10719000ADF8001004218DF804108DF805000A46A2
:1071A00005A90DF10600FDF7BBFB042204A90DF1B2
:1071B0000A00FDF7B5FB00A901A8FFF78FF806B09C
:1071C00010BD80B5FBF76DF84FF49671FBF756FADA
:1071D00007208DF802000120ADF8000000A90DF194
:1071E0000200FFF77BF801BD2DE9F041DFF8804C8C
:1071F0006068002828D0218888421FD003F072FAE6
:10720000054666682788A6EB07081FFA88F84246F5
:10721000381900F108012846FDF782FB3A4604F1CF
:10722000080108EB0500FDF77BFB3246294604F117
:107230000800FDF775FB284603F06CFA626804F15C
:1072400008010520FFF79BFF002060602080BDE85B
:10725000F0812DE9FC4105460F469046FBF721F8E9
:107260000026D5F809100C1D2A781146012960D096
:107270000F2933D0352935D0802900F08680812927
:1072800000F08D80822900F08A80852900F08780B7
:10729000862900F08480882900F081808A2900F006
:1072A00086808B2900F09F808C2900F0AB808D298F
:1072B00000F0B380DD2900F0BD80DF2900F0D78029
:1072C000F02918D0F42921D0F62927D0F82945D063
:1072D000F92933D0FF2900F0A5805DE0807D207082
:1072E00001205AE0012007F02EFE304607F02FFE65
:1072F0000120207051E00422DFF8781B2046FDF7C2
:107300000FFB0120FDF7B4F8012046E0042200F154
:1073100010012046FDF704FB01203EE00322214638
:107320003046DFF8543B9B681B6E1B6A9847012070
:1073300033E020460AF076F801202EE0B5F801206F
:10734000B5F80300C010C0EB0011D5F8050000EB44
:1073500081112046FDF7E4FA01201EE03046ADF829
:10736000040001206979012900D10320FCF7E9FA22
:10737000FCF723FBADF80400FCF736FB022201A961
:107380002046FDF7CDFA012007E0D5F80500207072
:107390002146304608F0E2FE3046BDE8F681304630
:1073A0002070214602F07F0008F0D8FEF4E70120AB
:1073B0002070DFF8C40A45683746287F002801D1CD
:1073C0003046EAE7687A002803D1286E4068804793
:1073D00007462046296EC9698847002FDCD0286EF1
:1073E00080688047D8E70120B5F80310C1F3C101D8
:1073F000091D884040F0020020702146012008F05D
:10740000ADFEC9E701782170C17861704179A17042
:107410008079E07001202071BFE720460AF016F85D
:107420000646B9E704F10802211D2046FDF7CEF813
:107430000120B2E76879DFF8401A51F82050687AE5
:10744000002810D0424639462846FFF79FF8DFF85B
:107450002C0A01210170DFF8281A08200AF0B8F878
:107460000120207001E030462070012095E7687906
:10747000DFF8041A51F82050286995F8221090FB83
:10748000F1F0401E0090042200A92046FDF748FAC2
:10749000012082E708400020ECBE00202C6700207D
:1074A000F0B593B00646FAF7FCFE054603F042F944
:1074B000D6F809100C1D3178002208924FF0FF32E7
:1074C000099217460A46312A00F01181322A00F04B
:1074D0001881332A00F02481342A00F02B81A12A5C
:1074E00000F05581A22A00F07481A42A00F07F8167
:1074F000B12A00F0F482B22A00F07684B82A00F0B3
:107500009181C12A00F0B981CD2A00F08080CE2A75
:1075100000F09680D02A37D0D12A2BD0D22A38D06A
:10752000D32A3FD0D42A41D0D62A4DD0D72A4BD007
:10753000D82A51D0D92A4FD0DB2A00F01381DC2A77
:1075400000F01781F12A4FD0F22A00F09280F52A3C
:1075500000F0A680F72A00F0B980FA2A00F06E84C5
:10756000FB2A00F06D84FD2A00F0A580FE2A00F0C1
:107570007684B9E000212846FBF7BEF80020A87306
:10758000FFF732FE0120B0E00020FCF771FF012080
:10759000ABE001212846FBF7AFF801200AF068F8BC
:1075A0000120A2E00020A87201209EE00120A87224
:1075B000002068730120A873E87A002802D1012016
:1075C0000AF056F8012090E0D62901D1012000E010
:1075D0000020E872012088E0D92901D1012000E0D3
:1075E00000202873012080E000210CE00A180B5DC8
:1075F00082F88430022905D10A5D80F887200A5D6F
:1076000080F88820491C0329F0DB01206DE000256B
:1076100012E0DFF86408466806EB4506022204EB38
:10762000450106F15800FDF77BF9B6F95810DFF86F
:107630005408FAF7B8FE6D1C032DEADB012054E074
:10764000002512E0DFF83008066806EB4506022246
:1076500004EB450106F15800FDF762F9B6F9581040
:10766000DFF82408FAF79FFE6D1C032DEADB0120EA
:107670003BE0297C090601D4012036E02178A0F8FE
:107680008A106178A0F88C1002212046DFF8E827E4
:10769000D269126E92699047002825D0012024E01B
:1076A000032221460120DFF8D0379B681B6E1B6A3E
:1076B0009847012019E01B2221460720DFF8B83740
:1076C0009B681B6E1B6A984701200EE0DFF8A80735
:1076D0008669306E80688047002805D001222146E7
:1076E0000520336E1B6A9847002013B0F0BD07F0E9
:1076F00032FC012801D10120F7E7204607F056FBB4
:10770000F2E707F028FC012801D10120EDE720462F
:1077100007F0D1FB20780028E6D007F0FDFBE3E777
:1077200007F019FC012801D10120DEE7207807F0DD
:10773000FAFBD9E707F00FFC012801D10120D4E7BB
:107740004FF480510020FBF710F8012007F07EFA7B
:10775000012007F0FCFB207807F006FC07F0EBFAAD
:107760000120C2E7D6F80510DFF82007FAF71BFE64
:10777000BAE7FDF7EBFB002802D0FDF708FCB3E702
:10778000FDF769FC0028AFD0FDF738FCACE794F9B1
:1077900000500422611C08A8FDF7C2F8B6F80100E9
:1077A000062806DB0422611D09A8FDF7B9F894F943
:1077B0000970042D04D1DFF8C0060069A17A817236
:1077C0000097099B00220899284608F026FD2070A2
:1077D0008AE794F900500422611C08A8FDF7A0F87C
:1077E00000231A460899284608F082FD7DE794F99F
:1077F00000500422611C08A8FDF792F8B6F80100B9
:10780000062806DB0422611D09A8FDF789F894F912
:1078100009700097099B00220899284608F0B8FDD6
:10782000207061E720780146032906D01A2911D07B
:10783000252913D0282915D018E060788DF80A0082
:10784000012805D1A0788DF80B00204600F002FC3D
:1078500001204AE7204600F0FDFBF9E7204600F052
:10786000F9FBF5E7204600F0F5FBF1E794F901108C
:1078700040B209F06AFCC0B237E7207801460E3901
:1078800008D0091F03291CD9091F37D0491E00F051
:107890009B800EE10E208DF8080060788DF80A00BC
:1078A000A1788DF80B10E2788DF80C200023ADF84C
:1078B0000D3052B249B240B2FAF76FFF00F0C1FB8F
:1078C000F7E08DF80800122802D161788DF80A10CF
:1078D000132802D161788DF80B10142802D1617839
:1078E0008DF80C10152802D160788DF80A006278A6
:1078F0002178DFF89C05FAF756FDDAE06078A17888
:10790000090401EB0060E17800EB012021794018C7
:10791000CDF80A006079A179090401EB0060E179F2
:1079200000EB0120217A4018CDF80E00607AA17A90
:10793000090401EB0060E17A00EB0120217B401893
:10794000CDF81200607B8DF81600A07B8DF8170033
:10795000E07B8DF81800207C8DF81900607C8DF894
:107960001A00A07CE17C11EB002000B20146ADF8CA
:107970001B10217D00EB0120617D4018ADF81D003A
:10798000A07D8DF81F00DDF80A00002807D1DDF882
:107990000E00002803D1DDF81200002809D00DF1F7
:1079A0000A0184B068461622FBF742F80FBCFAF7CA
:1079B0009BFF0DF10A0184B068461622FBF738F8E8
:1079C0000FBC00F06BFB74E060788DF809001D2897
:1079D0003ED1A0788DF81300A07801280ED1E07870
:1079E000217911EB0021ADF80A1089B20A469DF801
:1079F00009100FF2A440FAF7D6FC5AE002280BD186
:107A0000E078217911EB0021ADF80C1089B20FF26A
:107A10009840FAF7C8FC4CE003280BD1E0782179B4
:107A200011EB0021ADF8141089B20FF28840FAF77B
:107A3000BAFC3EE004283CD1E078217911EB00212A
:107A4000ADF8161089B20FF27840FAF7ACFC30E0CE
:107A5000262809D1A0788DF80E00A078012828D119
:107A6000E0788DF80D0024E01C2822D1A0788DF854
:107A70000D00A078012807D1E1788DF80A100FF2E7
:107A80004C40FAF790FC14E0022807D1E1788DF819
:107A90000B100FF24C40FAF786FC0AE0032808D0DE
:107AA000052806D1E1788DF80C100FF24840FAF75E
:107AB0007AFC06208DF8280020780B900DF131001B
:107AC00002A91822FAF7B4FF0B208DF8300000202D
:107AD000ADF84A000AA800F007FBC0B205E694F929
:107AE000000008F0DAFD012840F04F8120780146BF
:107AF000032925D0062962D0092928D00C2942D093
:107B00000D294ED0192900F08D801A2964D01B2927
:107B100000F09D801C2900F0D8801D2900F0B08065
:107B20001E2900F0DF80252900F0F880262900F0CA
:107B3000E780272900F0F980282900F01D811FE146
:107B40000322611C0DF10A00FCF7EAFE1DE1072289
:107B5000611C0DF10A00FCF7E3FEBDF80A00010A02
:107B600041EA0020ADF80A00BDF80C00010A41EA24
:107B70000020ADF80C00BDF80E00010A41EA00201B
:107B8000ADF80E0001E10322611C0DF10A00FCF7C3
:107B9000C7FEBDF80B00010A41EA0020ADF80B005A
:107BA000F3E00322611C0DF10A00FCF7B9FEBDF8F9
:107BB0000B00010A41EA0020ADF80B00E5E00122CC
:107BC000611C0DF10A00FCF7ABFE9DF80A100FF2E4
:107BD0003830FAF7E8FBD8E00B22611C0DF10A00FF
:107BE000FCF79EFEDDF80B00010221F0FF11000AF8
:107BF00000F0FF100843CDF80B004FEA3040CDF8FD
:107C00000B00BDF81000010A41EA0020ADF8100099
:107C100000239DF914209DF913109DF91200FAF725
:107C2000BCFDB2E00622611C0DF10A00FCF778FEF3
:107C3000BDF80A00010A41EA0020ADF80A00BDF8CB
:107C40000E00010A41EA0020ADF80E009DE004227A
:107C5000611C0DF10A00FCF763FEBDF80A00010A81
:107C600041EA0020ADF80A00BDF80C00010A41EA23
:107C70000020ADF80C000FF29C20FAF794FB84E092
:107C80000922611C0DF10A00FCF74AFEBDF80A004A
:107C9000010A41EA0020ADF80A00BDF80C00010A13
:107CA00041EA0020ADF80C00BDF80E00010A41EADF
:107CB0000020ADF80E0000239DF912209DF911104F
:107CC0009DF91000FAF769FD5FE060788DF80A0011
:107CD000A0788DF80B00A27861780FF24420FAF7B3
:107CE00062FB52E00322611C0DF10A00FCF718FE52
:107CF000BDF80B00010A41EA0020ADF80B0044E09A
:107D00000522611C0DF10A00FCF70AFEBDF80B000C
:107D1000010A41EA0020ADF80B0036E00922611C9F
:107D20000DF10A00FCF7FCFD2FE00A22611C0DF1A9
:107D30000A00FCF7F5FDBDF90A00C0F3072141EA8E
:107D40000020ADF80A00BDF90C00C0F3072141EA9C
:107D50000020ADF80C00BDF90E00C0F3072141EA88
:107D60000020ADF80E00BDF91000C0F3072141EA74
:107D70000020ADF8100008E060788DF80A0004E0FB
:107D80008DF8080060788DF80900207801460529F3
:107D900007D1404801210170687A00280ED10846B9
:107DA000A3E418290AD18DF8080060788DF809003D
:107DB000A0788DF80A00E0788DF80B0000208DF88F
:107DC000280020780B900DF1310002A91822FAF753
:107DD0002FFE0B208DF830000020ADF84A000AA8D5
:107DE00000F082F9C0B280E42078052804D1294847
:107DF00000210170012078E41A280CD10822611CAE
:107E00000DF10A00FCF78CFDBDF81000010A41EAF3
:107E10000020ADF8100001208DF8280020780B908C
:107E20000DF1310002A91822FAF702FE0B208DF89D
:107E300030000AA800F058F9C0B256E4012054E41A
:107E40002078002802D0052805D006E00FF2E000D7
:107E5000FDF786F801E0FFF7C7F9012045E404F1DA
:107E60000802211D2046FCF769FB01203DE40000CB
:107E7000F4F1002050680020084000200E2F01205F
:107E8000DCA1002094230308A0230308AC230308EB
:107E9000B82303080F2F01204C5420535020256491
:107EA0002C202564000000004C54205750202564ED
:107EB000000000004C5420535220256400000000B4
:107EC0004C54205341522025640000005B41504433
:107ED000525D204E545F5357554E202564000000DC
:107EE0005B415044525D204E545F545755532025FA
:107EF000640000005B415044525D204E545F42419B
:107F0000544348202564000050443A205343202520
:107F1000640000004C5420535320414444000000AE
:107F200041504452204144442025642025640000EF
:107F300041505F52455155455354000069487047C0
:107F4000F8B50C461646012500282BD106EB860015
:107F5000644901EBC007F868E040C00708D5234634
:107F6000FA6831460FF2FC20FAF71DFA0220F2BD42
:107F70004FF0FF30009003462A467968204608F00B
:107F80004CF900280CD02346FA6831460FF2E42061
:107F9000FAF709FAF8682946A1400843F8602CE08E
:107FA0000220F2BD012828D106EB86004D4901EBE5
:107FB000C007F868E040C00708D42346FA68314695
:107FC0000FF2C020FAF7EFF9032516E04FF0FF3368
:107FD0002A467968204608F08BF9002807D0234606
:107FE000FA6831460FF2AC20FAF7DDF900E003251C
:107FF000F8680121A1408843F8602846F2BD09F0E5
:10800000B0B802B58AB00021ADF8221001910A2162
:108010008DF8081000218DF809108DF80A1005213F
:108020008DF80010019004220AA90DF10900FCF757
:1080300077FC0020ADF8220000A800F055F80BB046
:1080400000BD80B50AF0D0F80FF25820BDE802401C
:10805000FAF7A9B938B5447885780078032810D0A4
:108060001A281AD1012C18D101200BF0DBFC0123B6
:1080700022461A210FF2382001B0BDE83040FAF74D
:1080800092B9012C09D128460AF0B9F829460FF215
:108090003020BDE83440FAF786B931BD0FB480B561
:1080A000002805D10846002802D11046002804D037
:1080B0000CF023FAC046C04601E00CF007FA01BC00
:1080C0005DF814FB00222D2809D200EB800305483F
:1080D00000EBC300C068C840C00700D501221046AD
:1080E00070470000ECBE002030B585B00446012585
:1080F00094F90000062800F2A180DFE800F00428CF
:10810000445F76979B0004F1090182B0684618220B
:10811000FAF78EFC0CBC94F90810606840B208F0C5
:1081200059FC02280AD1606800B208F038FE002528
:1081300061680FF29810FAF736F985E0032840F0ED
:10814000838061680FF28C10FAF72DF97CE060688B
:108150001A280AD104F1090009F0AFF8237CE2687B
:10816000E17A0FF27810FAF71EF994F908106068B6
:1081700040B208F02FFD032866D161680FF2741039
:10818000FAF711F960E0618C00A808F022FE9DF971
:10819000040002280AD1009800B208F000FE002571
:1081A00000990FF25810FAF7FEF84DE003284BD172
:1081B00000990FF25010FAF7F6F845E00CF0BAFA11
:1081C00002280AD1606800B208F0E9FD0025616864
:1081D0000FF23810FAF7E7F836E0032834D1616877
:1081E0000FF23010FAF7DFF82EE0606805280CD1A6
:1081F00028460CF066FB02280DD0032824D16168C4
:108200000FF22010FAF7CFF81EE002281CD10CF074
:108210005CFC0228F1D1606800B208F0C0FD0025C6
:1082200061680FF2F800FAF7BEF80DE0204608F09A
:1082300035FE09E0204608F0DFFF05E061680FF237
:10824000EC00FAF7B0F80025284605B030BD012053
:1082500070470FB4022004B070470120704700201F
:1082600070477047534D41432025642025642025E5
:1082700064000000534D41202564202564202564BE
:1082800000000000534D5243202564202564202522
:1082900064000000534D522025642025642025648D
:1082A0000000000050442053657453540000000047
:1082B00041542052492D2564202564202564000066
:1082C00050442055542D256400000000414C4F4679
:1082D00020256400414C4346202564004F4A482035
:1082E000454C203078257820307825782030782546
:1082F00078000000524C434620256400504C4F4605
:1083000020256400504C43462025640050414F46D0
:1083100020256400504143462025640050504F46BC
:108320002025640050504346202564004558204CC9
:108330004D454C20256400005FF0FF0C1CEAD05135
:1083400014BF614506E0C110400721F0E04101F192
:108350006051704779B900F0004100020AD0B0FACC
:1083600080FC00FA0CF001F16051A1EB0C5101EB23
:10837000D0214005704741020CBF40F4E0016FF08E
:1083800000010020704700004FEAF17CBCF1E04C96
:108390002CBFBCF5001F11E05FEA4C0C34BFBCF1F0
:1083A0007F5F2EE05FEA9C0C4FEA0C1C4FEA3C0C0E
:1083B000C10071F100414CEB50707047C90241EAB5
:1083C0005051C00218BF41F0010141F000414FEA95
:1083D0006C50C0F10900212810D240EACC7CCCF1CD
:1083E000200C11FA0CF070F10040CCF1200C21FAB5
:1083F0000CF00CF0004C40EB0C0070474FEACC70D6
:108400007047490011F5001F04D84FEACC10FF3027
:10841000C0057047C81770471FB50CF0B7FB212186
:1084200001601FBDDFF8AC1100220A700A7001283C
:1084300002D0042803D0704701200870704705203F
:108440000870704764490860704710B463494A680F
:1084500002F00C02082A13D10A680B6803F03F03EC
:10846000604CB4FBF3F30A68C2F388125A430B68FA
:10847000C3F301435B1C5B00B2FBF3F2026001E05B
:10848000584A02604A6802F0F003574A1B099B5C95
:10849000046824FA03F343604C6804F4E054A40A2B
:1084A000A45CE3408360496801F46041490B895C46
:1084B000426822FA01F1C16010BC7047484900F4DB
:1084C0004072B2F5407F06D10A6822F4F812474B99
:1084D00003401A430A608A6E000552EA105088660B
:1084E0007047434908607047424908607047424AF4
:1084F0000029116802D008431060704721EA00008B
:10850000106070473D4A0029116802D0084310608E
:10851000704721EA000010607047394A002911684D
:1085200002D008431060704721EA000010607047D5
:10853000344A0029116802D008431060704721EACC
:10854000000010607047304A0029116802D00843CB
:108550001060704721EA0000106070472B4A002924
:10856000116802D008431060704721EA00001060D3
:108570007047274A0029117802D0084310707047CD
:1085800021EA0000107070474109114A012901D108
:10859000116804E0022901D1116F00E0516F00F071
:1085A0001F0021FA00F000F001007047194801682F
:1085B00041F08071016070470021174A1268024241
:1085C00000D0012108467047144908707047000028
:1085D0000038024070380240800E474204380240A2
:1085E000083802400024F40014680020FFFCFF0F4C
:1085F0003C0E4742400E474230380240403802406D
:1086000044380240103802402038024024380240EA
:108610000D380240743802400C3802400E380240D7
:1086200080B52749884209D101210846FFF780FF1C
:1086300000210120BDE80440FFF77ABF21498842AC
:1086400009D101210220FFF773FF00210220BDE8BC
:108650000440FFF76DBF1C49884209D10121042065
:10866000FFF766FF00210420BDE80440FFF760BF6C
:108670001649884209D101210820FFF759FF00213E
:108680000820BDE80440FFF753BF1149884209D1D3
:1086900001211020FFF74CFF00211020BDE804400D
:1086A000FFF746BF0B49884209D101218020FFF71F
:1086B0003FFF00218020BDE80440FFF739BF01BD26
:1086C000000002400004024000080240000C02408A
:1086D00000100240001C0240F0B4002232E00123EE
:1086E00093400C681C409C422BD154000325A540AC
:1086F000ED4306682E40066006680F79A7403E43AA
:1087000006600E79012E01D0022E11D186682E400E
:10871000866086684F79A7403E438660466826EAB1
:108720000303436043688E799640B6B23343436097
:10873000C3682B40C360C368CD7905FA04F42343B2
:10874000C360521C102ACAD3F0BC70474FF6FF71A9
:1087500001600021017141718171C1717047002276
:108760000069084200D0012210467047018370471B
:108770004183704710B4CB1000EB830001F0070178
:108780008900036A0F248C40A3430362036A02FA40
:1087900001F11943016210BC7047000080B54349E4
:1087A00088420BD101214FF40010FFF7CCFE0021CD
:1087B0004FF40010BDE80440FFF7C5BE3C498842B5
:1087C0000BD101214FF48000FFF7BDFE00214FF4D3
:1087D0008000BDE80440FFF7B6BE364988420BD1A1
:1087E00001214FF40000FFF7AEFE00214FF400001E
:1087F000BDE80440FFF7A7BE01BD7FB504460D46A6
:10880000A68800A8FFF721FE02992B48B1FBF0F0E3
:108810004FF6C07232400243A28022884FF6FE73A8
:108820001A4022802A68254B9A420AD25200B1FB94
:10883000F2F10A4692B2042A00DA0421401C208494
:1088400021E0EB884BF6FF76B34204D102EB420203
:10885000B1FBF2F106E019235A43B1FBF2F141F406
:10886000804189B20A0502D141F0010189B241F487
:10887000004180B24FF4967250434FF47A7290FBED
:10888000F2F0401C2084A183208840F00100208069
:1088900020884FF6F5310840A988084369890843C4
:1088A0002080A8892989084320817FBD0054004089
:1088B00000580040005C004040420F00A1860100CB
:1088C0000029018803D041F00101018070474FF673
:1088D000FE721140018070470029018803D041F4E5
:1088E0008071018070474FF6FF6211400180704730
:1088F0000029018803D041F40071018070474FF6D0
:10890000FF52114001807047002A02D041F001015E
:1089100001E001F0FE01018270470029018803D0C7
:1089200041F48061018070474FF6FF3211400180B1
:1089300070470029018803D041F40041018070474D
:108940004904490C0180704782B00246002003466A
:108950000193009300920A0F01920902090A019AF9
:10896000002A03D0009A1432009203E0090C009A06
:1089700018320092009A12680A4200D0012002B018
:108980007047000080B5254988420BD101214FF482
:108990008050FFF7E3FD00214FF48050BDE8044014
:1089A000FFF7DCBD1E4988420BD101214FF4804006
:1089B000FFF7C9FD00214FF48040BDE80440FFF7F8
:1089C000C2BD184988420BD101214FF40040FFF786
:1089D000BAFD00214FF40040BDE80440FFF7B3BDED
:1089E00001BD028802F441520B881A434B881A4396
:1089F0008B881A43CB881A430B891A434B891A4335
:108A00008B891A43CB891A430280828B4FF2FF7302
:108A10001A408283098A01827047000000300140B9
:108A200000380040003C00400029018803D041F09C
:108A30004001018070474FF6BF72114001807047BE
:108A4000002A828802D011438180704722EA010106
:108A50008180704700220089084200D00122104620
:108A60007047000001684908490001600021016069
:108A700041608160C1600161212141616A49884290
:108A800003D16A483D21016070476949884204D199
:108A900066484FF47461016070476649884204D1AA
:108AA00062484FF47411016070476349884204D1F1
:108AB0005E484FF07461016070476049884203D19D
:108AC0005A485F49416070475E49884203D1574820
:108AD0005D49416070475D49884203D153485C4914
:108AE000416070475B49884204D150484FF03D5186
:108AF000416070475849884203D158483D21016080
:108B000070475749884204D154484FF4746101605A
:108B100070475449884204D150484FF474110160A1
:108B200070475149884204D14C484FF0746101604C
:108B300070474E49884203D14848414941607047D7
:108B40004B49884203D145483F49416070474949F4
:108B5000884203D141483E494160704746498842B6
:108B600003D13E484FF03D51416070470268434B8E
:108B70001A400B681A43CB681A434B691A438B6936
:108B80001A43CB691A430B6A1A434B6A1A438B6A1E
:108B90001A434B6B1A438B6B1A4302604269D2082B
:108BA000CB6A53EAC2020B6B1A4342610A69426004
:108BB0004A6882608968C16070470029016803D0F3
:108BC00041F00101016070474908490001607047A8
:108BD000002A01D001617047C1607047006800F051
:108BE0000100704700221C4B984201D2244800E04B
:108BF00024488B0001D5406800E000680840224905
:108C0000084200D0012210467047134A904201D218
:108C10001B4800E01B481C4A0A40890001D5C2607D
:108C20007047826070470000106002400860024098
:108C3000286002404060024058600240706002407C
:108C40003D00002088600240400F0020A0600240EC
:108C500000003D20B86002401064024008640240F9
:108C6000286402404064024058640240706402403C
:108C700088640240A0640240B86402403F801CF057
:108C800000600240006402407D0F7D0F02490860D1
:108C9000704702490860704720000E4224000E42CF
:108CA00070B504460026DFF83854CA20E861532026
:108CB000E86100F018F8002811D0286820F0400082
:108CC00028602868216808432860A068A860A86810
:108CD000616840EA0140A86000F024F80126FF2006
:108CE000E861304670BD81B000200090DFF8F403E9
:108CF0000168490613D44FF0FF310160016801F0AB
:108D00004001009A521C0092009AB2F5803F01D0B7
:108D10000029F3D00068800900F0010000E0012084
:108D200001B07047DFF8BC03016821F080010160E9
:108D3000704781B000200090DFF8A813CA20886136
:108D400053208861086820F0A0000860086800F0DF
:108D50002000009A521C0092009AB2F5003F01D008
:108D60000028F3D00868400900F00100FF228A6162
:108D700001B07047F8B507460E460024DFF85C5393
:108D8000002FA86804D140060AD42046F07007E0FE
:108D9000400603D5307800F0BEF901E02046F070BF
:108DA0003078002F09D07178090241EA0040B1788B
:108DB0000843F17840EA01460FE000F0A1F90746C8
:108DC000707800F09DF9000240EA0747B07800F0A3
:108DD00097F93843F17840EA0146CA206862532087
:108DE0006862FFF780FF00280FD0DFF8FC023040F8
:108DF0002860FFF797FFA868800605D4FFF799FF62
:108E0000002802D0012400E00124FF2068622046EF
:108E1000F2BD10B50C46DFF8C4120968DFF8C822AD
:108E200011400A0C02F03F0323700B0A03F07F038A
:108E3000637001F07F01A17002F04001E170002831
:108E40000BD1207800F067F92070607800F063F9AA
:108E50006070A07800F05FF9A07010BDDFF88C1290
:108E6000486A0968704770B506460D460024002E12
:108E700006D16878C10603D500F0EF000A306870AB
:108E8000002E05D0687800F046F9A87800F043F984
:108E9000E878002E09D06978090241EA0040A978F3
:108EA0000843297840EA41360FE000F029F90646E8
:108EB000687800F025F9000240EA0646A87800F03C
:108EC0001FF93043297840EA4136DFF82052CA20A2
:108ED000286253202862FFF706FF00280FD0DFF832
:108EE000100230402860FFF71DFF6868800605D437
:108EF000FFF71FFF002802D0012400E00124FF201B
:108F00002862204670BD10B50C46DFF8E0110968F4
:108F1000DFF8DC2111400A0CE2700A0A02F01F029D
:108F2000627001F03F02A270490B01F0070121704D
:108F300000280BD1E07800F0EEF8E070607800F0E7
:108F4000EAF86070A07800F0E6F8A07010BDDFF8D5
:108F50009011CA22CA615322CA610A68D208D2009B
:108F60000A600A6810430860FF20C8617047DFF894
:108F70008411CA220A6153220A610860FF20086135
:108F8000704781B000210091DFF85411CA22CA61F4
:108F90005322CA610028086804D040F48060086049
:108FA000012012E020F480600860486800F00400AE
:108FB000009A521C0092009AB2F5803F01D000281E
:108FC000F3D04868800800F00100FF22CA6101B0B8
:108FD000704781B000220092474A0092009A02EB4B
:108FE000800000900098016001B0704781B00021BE
:108FF000009141490091009901EB80000090009898
:10900000006801B0704738B500242246344DCA23A9
:10901000EB615323EB616B681B0701D406E0521C24
:109020006B681B0702D5B2F5805FF8D16A6812073A
:1090300009D42A68D20606D408436862FFF779FE8D
:10904000002800D00124FF20E861204632BD244AD8
:10905000CA23D3615323D36100F0040320F004003A
:109060000029116805D008431060906B1843906385
:1090700005E021EA00001060906B98439063FF20A8
:10908000D06170470021174A12681C4B1A400242F7
:1090900000D001210846704710B40021104A936B9C
:1090A00003F004031468044003EAD03323435268F6
:1090B00002EA101002D0000400D00121084610BCC2
:1090C000704708490003000C40F080000A6802F075
:1090D000800262EA0000086070470000002800403B
:1090E000082800400C2800407F7F7F0004280040B3
:1090F0003FFFFF0014280040502800407F3F010040
:10910000002101E0491C0A38C0B20A28FADA40EA14
:109110000110C0B27047010901EB810200F00F009D
:1091200000EB4200C0B2704730B40168CB43214924
:109130008279002A27D00A461468234013605368B6
:109140000468A34353600379CC18236805682B4354
:10915000236093680468A3439360D3680468A343BF
:10916000D36043790568102B07D19168294391603A
:10917000D16800680843D0600AE051FA83F420689F
:109180002843206004E000790C1820681840206013
:1091900030BC70470021074A1368034052690242FD
:1091A00002D0002B00D00121084670470249086018
:1091B00070470000003C0140143C0140194908433D
:1091C00019490860704770B403781A460121C478C1
:1091D000002C1DD0144B1B6803F4E063C3F5E0635F
:1091E0001B0A4478C3F10405AC4085780F2646FA83
:1091F00003F32B4023431B010C4C13550078421101
:109200000B4B00F01F0001FA00F043F8220006E0CB
:109210005011084A03F01F03994042F8201070BC17
:10922000704700000000FA050CED00E000E400E0EB
:1092300000E100E080E100E030B401F003029200C0
:1092400021F00301054BCC580F259540AC43CC5081
:10925000CC5890402043C85030BC7047083801407B
:1092600080B501214FF48070FFF778F900214FF4A9
:109270008070BDE80440FFF771B942684C4B1A405A
:109280000B7942EA03220B681A4342608268494B19
:109290001A400B691A43CB681A438B681A434B79FF
:1092A00042EA43028260C26A22F47002097D491ECA
:1092B000C9B242EA0151C1627047002101600171E7
:1092C00041718160C16001610121017570473A49B6
:1092D0000A683A4B1A4003681A4343681A43836882
:1092E0001A43C06810430860704700210160416064
:1092F0008160C16070470029816803D041F001019D
:1093000081607047490849008160704770B4072444
:109310000A290BDBC568A1F10A0606EB4606B44034
:1093200025EA0404B3402343C36008E0056901EB68
:109330004106B44025EA0404B340234303611346C5
:109340001F24072B09DA436B521E02EB8202944062
:10935000A34391401943416314E00D2B09DA036BD9
:10936000D21F02EB82029440A34391401943016350
:1093700008E0C36A0D3A02EB82029440A343914095
:109380001943C16270BC7047816841F080418160BF
:1093900070470029816803D041F480618160704783
:1093A00021F4806181607047C06C80B2704700001A
:1093B000FFFEFFFCFDF7FFC004230140E030FCFF8F
:1093C00000220068084200D00122104670470000C9
:1093D00013F0004C03D55B42524263F100039CEA58
:1093E000210C00F0178010B5644603D34942404277
:1093F00061F1000100F00EF8640004D349424042DC
:1094000061F10001244203D55B42524263F1000343
:1094100010BD00001B4213D1094236D12AB1844647
:10942000B0FBF2F002FB10C270470BF0B5BBFCD3EF
:109430000022002370470B0002000021002070472B
:10944000904271EB030CF6D370B5B1FA81F4B3FA24
:1094500083F52C1BA340C4F1200532FA05F63343F3
:10946000A2405FF00046E64002E05B085FEA32029D
:10947000841A71EB030524BF204629467641F4D3B4
:1094800002000B003000002170BD012ACFD970B559
:10949000140C20D0B1FA81F4B2FA82F5C4F12004A0
:1094A0006419B4F12006D6D3B2405FF00044F44012
:1094B000002502E052085FEA3303C61A71EB020E80
:1094C00024BF3046714664416D41F3D302000B0066
:1094D0002000290070BD0C46B1FBF2F102FB1145E2
:1094E0002D0445EA1045B5FBF2F402FB145580B299
:1094F00040EA0545B5FBF2F002FB105240EA044099
:1095000070BD000000B500BF1300964694461039A8
:1095100028BFA0E80C50FAD85FEA417C28BF0CC0F5
:1095200048BF40F8042BC90728BF20F8022B48BFCA
:1095300000F8012B00BD00002DE9F04FA1B08246DC
:1095400002AE002017461D46029170620DF14408DC
:109550000AE017F8011B0298D0470290002800F09B
:10956000DA82706A401C7062387808B9706AD4E296
:109570002528EED10020F06030617061B061F061AB
:10958000306201E040F0010017F8011F2029F9D0F6
:1095900023290DD02B2904D02D2906D030290AD01B
:1095A0000CE040F0020080B2EEE740F00400FAE781
:1095B00040F00800F7E740F01000F4E72A290DD149
:1095C00029680A1D2A600968F162002904D5494208
:1095D00040F00400F16280B27F1C13E00021F162D0
:1095E0000BE0F16A6FF00043994205D001EB810373
:1095F00002EB43013039F1627F1C3A78A2F130016D
:109600000A29EED339782E2903D04FF0FF31B16209
:109610001EE017F8011F2A2906D129680A1D2A60B1
:109620007F1C0968B16213E00021B1620BE0B16AEE
:109630006FF00043994205D001EB810302EB430137
:109640003039B1627F1C3A78A2F130010A29EED399
:1096500030860FF6604039780BF0A0FA08B117F8A1
:10966000010B8DF83A009DF83A00682802BF39785E
:109670006829622005D06C2804BF38786C2803D193
:1096800071208DF83A007F1C11A8B0603978B1F1D3
:10969000250029D01C3800F0C080001F022840F2AD
:1096A000BC80133800F0E480093800F0B680801EDA
:1096B00000F07781401E00F02081401E022840F219
:1096C000AC80001F00F01981401F7BD0401E00F0CD
:1096D000CF80401E22D0C01E0BD0801E00F0C8805C
:1096E000C01E00F0C58064E1F068411CF1602521D6
:1096F00069E12868011D29600068B26A7060002A6B
:1097000002D5FBF76DF807E000210BF053FA0028B3
:109710001ABF7168401AB06A306156E12868011DAD
:10972000296000210068CDE900014FF03C0E11A82E
:109730007060DDE9000111B908B9B26ACAB1020668
:10974000120FA0EB02123032AEF10103D2B29E46EC
:109750003A2AA8BF2732000903F8082040EA01701E
:10976000090908BF002804D0726811AB73449A42FB
:10977000E5D311A971447160CEF13C00B16A30614A
:10978000884207DA081AB0614FF6EF71308E084050
:1097900030861AE1002940F1188196F8301001F066
:1097A0001401102940F01181F16AF268891AB26936
:1097B000891AA1EB000EBEF1010FC0F20681C6F8B6
:1097C00018E002E19DF83A00622818D0682806D017
:1097D0006A280BD06C2819D0712807D016E02868A9
:1097E000011D29600068716A0180EEE02A68101D81
:1097F00028601268706AC117C2E90001E5E02868B4
:10980000011D29600068716A0170DEE02868011D91
:1098100029600068716A0160D7E02868C01D20F0E7
:109820000700286000F108022A60D0E90023CDE992
:109830000023002B04D5F068421CF2602D220DE0BD
:10984000308E820704D5F068421CF2602B2205E0BE
:10985000C00705D5F068421CF260202200F80820FD
:10986000F06811AA8018706000A800F0E3F9ACE07D
:109870009DF83A006C2808BF2A6811D0712808BFEB
:109880002A6802D02A686A280AD1D21D22F007026B
:109890002A60144604F108022A60D4E9002303E098
:1098A000131D2B6000231268CDE90023682808BF30
:1098B00092B207D0622808BFD2B203D0742818BF72
:1098C0007A2802D10023CDE9002396F83000000762
:1098D0005FD5DDE90023002B08BF002A59D041F0F5
:1098E0002000782855D1F068302200F80820401C6C
:1098F000421CF26000F808104BE09DF83A00622824
:109900000CD0682810D06A281AD06C2823D071286F
:1099100016D074281FD07A280CD01CE02868021DAD
:109920002A6090F900201AE02868021D2A60B0F928
:10993000002014E02868021D2A60002302680FE05E
:109940002868C01D20F00700286000F108022A6086
:10995000D0E9002304E02868021D2A600268D317BA
:10996000CDE90023002B04DAF068421CF2602D22BE
:109970000DE0308E820704D5F068421CF2602B2285
:1099800005E0C00705D5F068421CF260202200F80F
:109990000820F06811AA8018706000A800F0C0F8D4
:1099A00013E0F068411CF16029680A1D2A6009680B
:1099B00009E0F068421CF260252200F8082021B17D
:1099C000F068421CF26000F80810F06AF168401A72
:1099D000B169401A3169401AF169401A7169401A37
:1099E000316AA0EB010996F830007F1C400710D4C3
:1099F00020208DF84000002409E0012310AA00A9CE
:109A0000504600F040FC002840F08580641C4C4526
:109A1000F3DBF4680DF1440B0AE01BF8011B02981C
:109A2000D0470290002876D0706A401C7062641E95
:109A3000002CF2D130208DF840004FF0000BB469BB
:109A400009E0012310AA00A9504600F01CFC0028E0
:109A500061D10BF1010BA345F3DB3469D6F804B0F7
:109A60000AE01BF8011B0298D0470290002852D050
:109A7000706A401C7062641E002CF2D130208DF898
:109A800040004FF0000BF46909E0012310AA00A97F
:109A9000504600F0F8FB00283DD10BF1010BA34527
:109AA000F3DB30697168746900EB010B09E01BF8A6
:109AB000011B0298D047029068B3706A401C706224
:109AC000641E002CF3D130208DF840004FF0000BC5
:109AD000346A08E0012310AA00A9504600F0D3FB25
:109AE000C8B90BF1010BA345F4DB96F83000400731
:109AF0007FF53AAD20208DF84000002400E0641C82
:109B00004C45BFF631AD012310AA00A9504600F024
:109B1000BAFB0028F3D04FF0FF3021B0BDE8F08F42
:109B20002DE9FA47064682B035690A466F2A08BF12
:109B3000082705D041F02000782814BF0A271027F5
:109B4000D6E900013C2480468946642A18BF692A68
:109B500005D1002903DAD8F1000869EB4909B9F108
:109B6000000F08BFB8F1000F0CD1306B50B9082FAF
:109B70003BD196F83800000737D530203B2485F8D4
:109B80003B0032E0CDE90089FB17404649463A46A2
:109B9000FFF740FCB846A8FB0023DDE90089A8EBED
:109BA00002023032A4F1010AD2B254463A2A03DB4F
:109BB0009DF80830513B9A180AF8052080465FEA64
:109BC000010908BFB8F1000F03D0F068611988429D
:109BD000D8D3082F09D196F83800000705D5605D65
:109BE000302802D0641E30206055C4F13C00B061C2
:109BF0006119F160316B884207DA081A30624FF65A
:109C0000EF71308F0840308710E000290ED596F8AC
:109C1000381001F01401102908D1716B7269891A8A
:109C2000326A891A081A0128A8BF306204B0BDE858
:109C3000F08700002DE9F24F04468EB0D4E9000110
:109C4000CDE9020104AE9DF8380040F020000090FC
:109C500061280AD0206B002848BF062004D404BF26
:109C60000098672801D1012020636168C1F30A5080
:109C700040F2FF7290421CD1080304BF2068002804
:109C800009D10320A0619DF8380061381A2836D325
:109C90000FF2346108E00320A0619DF838006138BC
:109CA0001A2829D30FF21861E0680322F8F7C0FEE2
:109CB000B5E1012816DA20460AF0A8FF012811DBD9
:109CC000002700200099612920D1E168302201F8A5
:109CD000012B4A1CE2609DF83820612A0CBF7822D3
:109CE00058220FE0626840F2FE3161F31E52471ABB
:109CF00062604FF0FF30E5E70FF2C051D4E70FF29A
:109D0000C451D1E70A706169891C616110B90025ED
:109D100000277BE10098612840F09680206B0028A6
:109D20004CBF2125451CDDE902012DB26E1CD4E992
:109D3000008900220023F9F775F83ABF89F0004046
:109D4000CDE90280CDE902893F1F8DF810200DF189
:109D5000110801E000F20708012E32DBDDE9020103
:109D6000002200230AF074FF2BD21C2102A80AF063
:109D700087FFDDE90201F9F7A1FAF61F8146012EFE
:109D800009DBF9F76BF802460B46DDE90201F8F74B
:109D9000ABFECDE9020108F20700072105E009F05A
:109DA0000F0200F8012D4FEA2919B9F1010F01DB6B
:109DB000491EF4D5491E5CBF002200F8012DF9D5DB
:109DC000C8E70DF11100A8EB00010DF11106A94241
:109DD000B8BF0D462DB228002FD4884206DA04A958
:109DE000411849780829A8BF0F2100DA002104AAE8
:109DF000821800E06D1E12F80139401E8B42F9D026
:109E00000F2904D104A941184A78521C4A7000282D
:109E100002D504AE6D1C3F1D2DB2681E0DD48119F4
:109E20000A783032D2B23A2A03DB9DF838303A3B16
:109E30009A1801F80129401EF2D5206B002840F144
:109E4000E580681E2063E1E0DDE9020100220023D5
:109E5000F8F7E8FF3CBF81F00041CDE902013FB2D5
:109E600047F2975078434849DFF820B190FBF1F76B
:109E70003FB2C7F107069246012E19DBDDE90289E0
:109E8000F00707D552465B4640464946F8F7ECFED8
:109E90008046894676105046594652465B46F8F74A
:109EA000E3FE82468B46002EEAD1CDE9028921E00D
:109EB00076429046DFF8D89012E0F00707D5524678
:109EC0005B4640464946F8F7CFFE80468946761005
:109ED0005046594652465B46F8F7C6FE82468B46C8
:109EE000002EEAD1DDE9020142464B46F9F742F87D
:109EF000CDE90201009866280CBF07F10A00062090
:109F0000216B4518142DA8BF132530208DF81000A3
:109F10000DF11106DFF87C90012D3DDBDDE902013A
:109F2000F9F7E2F906F1080104220A23B0FBF3F382
:109F300003EB8306A0EB4600303001F8010D0A2048
:109F4000B3FBF0F000EB8006A3EB4603303301F8DF
:109F5000013D521EE9D1083D01F10806012DDBDB70
:109F6000DDE90201F9F7C0F9F8F782FF02460B4676
:109F7000DDE90201F8F7B8FD00224B46F8F774FE60
:109F8000CDE90201CAE700BFA0860100000024401D
:109F90000000F03F84D797410DF11100301A0DF108
:109FA000110602E0401E7F1E761C31783029F9D060
:109FB0000099662902D13FB2791C03E065290CBFE4
:109FC00001210021226B8D182DB2A842B8BF054691
:109FD0002DB229001AD4814204DA885D3528A8BF41
:109FE000392000DA30208A19521E00E06D1E12F866
:109FF0000139491E8342F9D0392802D1885D401CBD
:10A000008855002902D5761E6D1C7F1C3FB29DF835
:10A01000381000972BB23246204600F003F80FB0FC
:10A02000BDE8F08F2DE9F043054685B01E46D5F812
:10A03000308089461746012E02DA01260FF28C275E
:10A0400049F02000BDF93040662808BF641C17D0D5
:10A05000672840F0818014F1040FC0F283804445EA
:10A0600080F2808095F83800641C000702D44645D1
:10A07000B8BFB04624B2B8EB040848BF4FF00008A0
:10A08000E868A96924B2012C25DA30234A1C0B5454
:10A09000B8F1010F03DA95F83810090702D52E211F
:10A0A0001154521CAA6118EB040FB8BFC8F1000488
:10A0B00024B26142A0446962B045B8BF464636B298
:10A0C000EE613246AB6939461818F8F7B1FCA8EBD7
:10A0D0000600A862C0E00818A64218DA32463946DF
:10A0E000F8F7A6FCA9697118A961A01B6862B8F10C
:10A0F000010F03DA95F83800000705D5E8682E222D
:10A100000A54E869401CE861C5F82880A4E02246AA
:10A110003946F8F78DFCA8692018361BB8F1010FF5
:10A1200003DA95F83810090703D5E9682E2242545E
:10A13000401C36B2A861B045B8BF4646EB6836B29F
:10A140003246E119C018F8F773FCA8693018A86105
:10A15000A8EB060068627FE0B9F1610F16D14FF0FD
:10A16000700918E0464504DA95F83810090758BF19
:10A17000B046B8F1010848BF4FF00008B9F1670FC9
:10A1800014BF4FF045094FF0650904E0B9F1410FE4
:10A1900008BF4FF05009A969E86817F8013B0B5454
:10A1A0004A1CB8F1010F05DA95F83810090758BFB5
:10A1B000AA6117D52E211154531CAB61B8F1010FC0
:10A1C00010DB761E36B2B045B8BF464636B23246D0
:10A1D00039461818F8F72CFCA8693018A861A8EBC4
:10A1E00006006862A869E9684718200007F8019B23
:10A1F00003D42B2007F8010B03E02D2107F8011BE6
:10A20000644200260DF1080808E00A2200A80AF0BE
:10A21000C1FD019808F8010B761C009C21B20129B0
:10A22000F3DA022E06DA49F02000652804BF302058
:10A2300007F8010B4EB9302007F8010B07E0761E36
:10A2400002A8305C303007F8010B012EF7DAA8695C
:10A25000E9684018381AE86195F8380000F01400F1
:10A2600010280DD16869A9690818696A0818E96990
:10A270000818A96A0818696B8842BCBF081A2862C6
:10A2800005B0BDE8F083F8B504460D4616461F46F6
:10A29000002004E0E86A401CE8627F1E002047B10D
:10A2A00016F8011BA868A047A8600028F2D14FF05B
:10A2B000FF30F2BD686A6C747A4C00006E616E000B
:10A2C0004E414E00696E6600494E46003000000067
:10A2D0000CB41CB5044604A801900A46009401ABD6
:10A2E00000A9074878441830FFF726F900990022A2
:10A2F0000A7000285CBF0098001B16BC5DF80CFBC0
:10A30000538BFFFF01B58B0718D1121F21D351F8D2
:10A31000043BA3F1013C2CEA030C1CF0803C04BF7D
:10A3200040F8043BF1E79CFA8CFCBCFA8CF1C1F1DB
:10A3300018018B40CB4040F8043B13E0042A09D3BA
:10A3400011F8013B521E00F8013B5BB18B07F7D1BE
:10A35000DBE7121D5AB111F8013B521E00F8013B18
:10A3600003B1F8D111001CBF0022F8F7D7FF01BDDF
:10A37000002801D10A48806890F84C10642901D067
:10A38000002000E0806A7047002801D104488068FE
:10A3900090F84C10642901D0002000E0406A70471A
:10A3A0002C6700200248704702480149401A704754
:10A3B00000000020002000204C48C168002903D57F
:10A3C0004B4901604B49016070474B48016841F0BF
:10A3D00000410160704770B50446002600290BD08B
:10A3E000012902D14FF4807606E0022902D14FF410
:10A3F000007601E04FF4407600F082F809281ED183
:10A400003D4D286820F4407028602868304328605B
:10A41000286820F0F8002860286844F0020108430A
:10A420002860286840F48030286000F069F82968C6
:10A4300021F002012960296821F0F801296070BD2E
:10A4400070B504460D4600F05BF8092813D12A4E7A
:10A45000306820F440703060306840F40070306044
:10A46000306840F001003060256000F049F8316844
:10A4700049084900316070BD70B505460E4600F0D0
:10A480003FF8092811D11C4C206820F4407020604E
:10A4900020682060206840F0010020602E7000F0ED
:10A4A0002FF8216849084900216070BD13490860F0
:10A4B0007047092011490A68D20301D5012070476D
:10A4C0000A68D20601D5062070470A68D20501D570
:10A4D000022070470A6812F0EF0F01D00720704782
:10A4E0000968890700D5082070470000043C024035
:10A4F00023016745AB89EFCD103C02400C3C024084
:10A5000080B509208DF80000FFF7D3FF8DF800001B
:10A5100003E0FFF7CEFF8DF800009DF80000012852
:10A52000F7D09DF8000002BD0901002806D500F013
:10A530000F004C4A801800F8041C70474A4A8154A6
:10A54000704710B5401EB0F1807F01D3012010BDCF
:10A55000464C60600F214FF0FF30FFF7E5FF002011
:10A56000A06007202060002010BD38B5404D28783D
:10A57000401C28703F4C2078401C2070FAF7F7FFF1
:10A580000AF010FC2878411E2970002802D198207A
:10A59000FAF742F92078012804D16068002801D038
:10A5A000FAF79DF92078401E207031BD10B5314C6E
:10A5B0006078F021084202D09920FAF72DF9FAF7D5
:10A5C00098F96078401C60700AF046FC2A480068E0
:10A5D0004FF47A71B0FBF1F0FFF7B3FF002800D021
:10A5E000FEE72648264901600E214FF0FF30FFF7B5
:10A5F0009BFF6078F021084202D09920FAF70CF90D
:10A600006078401E6070C0B2002803D1BDE81040E1
:10A61000FAF769B910BD000010B51A4C4FF400519B
:10A6200020464183C04630BF4FF400512046FEF71C
:10A630009DF8F3E710B40F48006A0F4909684FF41A
:10A640007A72B1FBF2F1104A1368CB1A0F4C2468EE
:10A65000640102D512688B1A401C00FB013010BC4B
:10A660007047000018ED00E000E400E010E000E0BA
:10A67000152F01202C670020E067002008ED00E086
:10A68000000000080010024018E000E004ED00E0C7
:10A69000EFF3058000284AF03F84704780B5EFF360
:10A6A000108072B60B49096851F47F01094A1160A4
:10A6B00080F310880848006810F4700F02D1A720BA
:10A6C000FAF7AAF805485FF000710160044800211C
:10A6D000016001BD20ED00E088ED00E03CEF00E00E
:10A6E00034EF00E010B5040010480078002805D1D0
:10A6F0000F480AF050FC0D48012101700C480AF087
:10A7000080FC20000BF050FB040009480AF0ADFC6F
:10A71000200010BD10B5040005480AF072FC2000AE
:10A720000BF09CFC02480AF0A0FC10BD182F012081
:10A73000D42B01200048704728150120BFF34F8F0C
:10A74000DFF8C00C006810F4E060DFF8BC1C0843C0
:10A75000DFF8B01C0860BFF34F8FFEE700B583B091
:10A760000020ADF8040000208DF8060000208DF8D0
:10A770000700012000900DF106037622D021002071
:10A78000F7F7E1FE002801D1002044E076208DF8A3
:10A7900004009DF8060050F020008DF8050002230B
:10A7A00001AAD0210020F7F774FE002801D1002073
:10A7B00031E0012000900DF107034922D021002053
:10A7C000F7F7C1FE002801D1002024E049208DF8D0
:10A7D00004009DF8070050F001008DF805000223E9
:10A7E00001AAD0210020F7F754FE002801D1002053
:10A7F00011E076208DF804009DF806008DF8050024
:10A80000022301AAD0210020F7F743FE002801D13E
:10A81000002000E001200EBD38B50400F7F741FD2F
:10A820000500DFF8100D0078401CDFF8081D0870E7
:10A83000DFF8000D4078F021084202D09920F9F7A6
:10A84000EBFFFAF756F8DFF8EC0C4078401CDFF825
:10A85000E41C4870210089B22800F7F70FFFDFF8E9
:10A86000D40C4078F021084202D09920F9F7D4FFA7
:10A87000DFF8C00C4078401EDFF8B81C4870C0B24A
:10A88000002801D1FAF72FF8FAF78DFE31BD10B587
:10A8900082B00020ADF80000F7F703FD04006B2044
:10A8A0008DF8000080208DF80100022300AAD0213D
:10A8B0000020F7F7EEFD002801D1002094E064218C
:10A8C0002000F7F7DBFEFFF749FF002801D1002049
:10A8D0008AE06B208DF8000000208DF80100022333
:10A8E00000AAD0210020F7F7D4FD002801D10020D4
:10A8F0007AE028212000F7F7C1FE19208DF800002A
:10A9000004208DF80100022300AAD0210020F7F7CF
:10A91000C0FD002801D1002066E01A208DF800005B
:10A9200003208DF80100022300AAD0210020F7F7B0
:10A93000B0FD002801D1002056E01B208DF800005A
:10A9400018208DF80100022300AAD0210020F7F77B
:10A95000A0FD002801D1002046E01D208DF8000058
:10A9600003208DF80100022300AAD0210020F7F770
:10A9700090FD002801D1002036E06A208DF800000B
:10A9800000208DF80100022300AAD0210020F7F753
:10A9900080FD002801D1002026E06C208DF8000009
:10A9A0003F208DF801009DF80110DFF85C0DF7F7EE
:10A9B000FAFC022300AAD0210020F7F76AFD002844
:10A9C00001D1002010E06B208DF8000040208DF8B0
:10A9D0000100022300AAD0210020F7F75AFD002829
:10A9E00001D1002000E0012016BD0178407850EA36
:10A9F000012000B2704780B502200090DFF80C3DC6
:10AA00006B22D0210020F7F79EFD002801D1002005
:10AA10005BE001200090DFF8F83C1A22D0210020F2
:10AA2000F7F791FD002801D100204EE001200090B1
:10AA3000DFF8E03C1B22D0210020F7F784FD00283E
:10AA400001D1002041E001200090DFF8CC3C1C2225
:10AA5000D0210020F7F777FD002801D1002034E055
:10AA600001200090DFF8B43C1D22D0210020F7F730
:10AA70006AFD002801D1002027E001200090DFF8C6
:10AA8000A03C6A22D0210020F7F75DFD002801D10B
:10AA900000201AE001200090DFF8883C3822D02105
:10AAA0000020F7F750FD002801D100200DE0012023
:10AAB0000090DFF8743C1922D0210020F7F743FD05
:10AAC000002801D1002000E0012002BD80B5002057
:10AAD000ADF800001A208DF80000DFF8300C007986
:10AAE0008DF80100022300AAD0210020F7F7D1FC45
:10AAF000002801D1002090E01B208DF80000DFF835
:10AB00000C0C40798DF80100022300AAD02100200E
:10AB1000F7F7BFFC002801D100207EE01C208DF853
:10AB20000000DFF8E80B80798DF80100022300AA0D
:10AB3000D0210020F7F7ADFC002801D100206CE007
:10AB40001D208DF80000DFF8C40BC0798DF80100DE
:10AB5000022300AAD0210020F7F79BFC002801D196
:10AB600000205AE06A208DF80000DFF8A00BC078C2
:10AB70008DF80100022300AAD0210020F7F789FCFC
:10AB8000002801D1002048E019208DF80000DFF8EE
:10AB90007C0B80788DF80100022300AAD0210020D0
:10ABA000F7F777FC002801D1002036E038208DF837
:10ABB0000000DFF8580B007A8DF80100022300AA8C
:10ABC000D0210020F7F765FC002801D1002024E007
:10ABD0006B208DF80000DFF8340B00788DF8010051
:10ABE000022300AAD0210020F7F753FC002801D14E
:10ABF000002012E06C208DF80000DFF8100B407888
:10AC00008DF80100022300AAD0210020F7F741FCB3
:10AC1000002801D1002000E0012002BD10B582B063
:10AC20000020ADF80000DFF8E40A0078400612D5F5
:10AC30006B208DF8000000208DF80100022300AA8F
:10AC4000D0210020F7F725FC002801D10020C9E021
:10AC50003220FFF7E1FD6C208DF80000DFF8AC0A30
:10AC6000407810F0F8008DF80100022300AAD021EE
:10AC70000020F7F70EFC002801D10020B2E06A2086
:10AC80008DF8000000208DF80100022300AAD021D9
:10AC90000020F7F7FEFB002801D10020A2E00024ED
:10ACA00000E0641C062C10DA14F113008DF800008B
:10ACB00000208DF80100022300AAD0210020F7F720
:10ACC000E8FB0028EDD100208CE019208DF8000071
:10ACD00000208DF80100022300AAD0210020F7F700
:10ACE000D8FB002801D100207CE01A208DF800005C
:10ACF00003208DF801004FF4FA642000FA281DD0DB
:10AD0000B0F5FA7F13D0B0F57A7F09D0B0F5FA6FBD
:10AD100019D19DF8010050F018008DF8010016E0DF
:10AD20009DF8010050F010008DF801000FE09DF833
:10AD3000010050F008008DF8010008E09DF80100C6
:10AD40008DF8010003E09DF801008DF80100022359
:10AD500000AAD0210020F7F79CFB002801D1002099
:10AD600040E0FA2C14D0B4F5FA7F0DD0B4F57A7F18
:10AD700006D0B4F5FA6F0FD103208DF801000EE074
:10AD800002208DF801000AE001208DF8010006E0A4
:10AD900000208DF8010002E000208DF801001B204A
:10ADA0008DF800009DF80100C0008DF8010002231D
:10ADB00000AAD0210020F7F76CFB002801D1002069
:10ADC00010E038208DF8000000208DF801000223EB
:10ADD00000AAD0210020F7F75CFB002801D1002059
:10ADE00000E0012016BD00B583B00020ADF80600DC
:10ADF00000208DF804006B208DF8060001208DF8EE
:10AE0000070002230DF10602D0210120F7F741FBD4
:10AE1000002801D1002023E02820FFF7FDFC0120BD
:10AE2000009001AB6C22D0210120F7F78CFB0028A9
:10AE300001D1002014E06C208DF806009DF804007C
:10AE400010F0C0008DF8070002230DF10602D0219A
:10AE50000120F7F71EFB002801D1002000E00120AF
:10AE60000EBD2DE9F04F85B080460C0015001E0088
:10AE70000020ADF8040002A80021002206C0083816
:10AE8000062738208DF8040000208DF805000223E5
:10AE900001AAD0210120F7F7FCFA002802D15FF0C7
:10AEA000FF3079E123208DF8040000208DF80500A3
:10AEB000022301AAD0210120F7F7EBFA002802D1E2
:10AEC0005FF0FF3068E16A208DF8040000208DF803
:10AED0000500022301AAD0210120F7F7DAFA0028A1
:10AEE00002D15FF0FF3057E16A208DF804000420A2
:10AEF0008DF80500022301AAD0210120F7F7C9FA35
:10AF0000002802D15FF0FF3046E11A208DF80400DE
:10AF100001208DF80500022301AAD0210120F7F7B6
:10AF2000B8FA002802D15FF0FF3035E119208DF822
:10AF3000040000208DF80500022301AAD021012081
:10AF4000F7F7A7FA002802D15FF0FF3024E11B20B9
:10AF50008DF804008DF80580022301AAD02101207C
:10AF6000F7F797FA002802D15FF0FF3014E1F6B24C
:10AF7000002E0FD01C208DF804008DF805800223D0
:10AF800001AAD0210120F7F784FA002802D15FF04E
:10AF9000FF3001E14FFA88F8B8F1000F02D0C82065
:10AFA000FFF73AFC6A208DF8040044208DF8050074
:10AFB000022301AAD0210120F7F76BFA002802D161
:10AFC0005FF0FF30E8E023208DF80400F6B2002E99
:10AFD00003D008208DF8050002E070208DF80500F0
:10AFE000022301AAD0210120F7F753FA002802D149
:10AFF0005FF0FF30D0E00A20FFF70EFC5FF0000AA0
:10B000000BE05FFA8AFA002044F82A005FFA8AFA15
:10B01000002045F82A001AF1010A5FFA8AFABAF10B
:10B02000030FEEDB5FF00009B9F1320F6FDA0A208F
:10B03000FFF7F2FB0220009002AB7222D021012028
:10B04000F7F781FA002802D15FF0FF30A4E002A8F0
:10B05000FFF7CBFCFFB290FBF7F8B8F1070F02DA6D
:10B060007FF0010098E05FF0000A1BE05FFA8BFBC5
:10B0700002A810EB4B00FFF7B8FC5FFA8BFB54F80B
:10B080002B1001FA80F05FFA8BFB44F82B001BF1C8
:10B09000010B5FFA8BFBBBF1030FE7DB19F1010931
:10B0A0001AF1010A5FFA8AFAC245BDDAB9F1320F24
:10B0B000BADAFFB2009702AB7422D0210120F7F771
:10B0C00042FA002802D15FF0FF3065E0F6B2002EB0
:10B0D0001AD05FF0000B5FFA8BFBBBF1030FDDDAD8
:10B0E0005FFA8BFB02A810EB4B00FFF77EFC5FFAC8
:10B0F0008BFB55F82B1001FA80F05FFA8BFB45F8BB
:10B100002B001BF1010BE6E75FF0000BC1E72320EA
:10B110008DF8040000208DF80500022301AAD0213B
:10B120000120F7F7B6F9002802D15FF0FF3033E0D5
:10B130005FF0000B0FE05FFA8BFB54F82B004FF42D
:10B140007A714843322190FBF1F05FFA8BFB44F8AF
:10B150002B001BF1010B5FFA8BFBBBF1030FEADB4A
:10B16000F6B2002E17D05FF0000B0FE05FFA8BFBFA
:10B1700055F82B004FF47A714843322190FBF1F0DF
:10B180005FFA8BFB45F82B001BF1010B5FFA8BFB81
:10B19000BBF1030FEADB012005B0BDE8F08F2DE91C
:10B1A000F04389B004000D00160000275FF001088D
:10B1B00001A8002101605FF000090320009001ABAD
:10B1C0000D22D0210120F7F7BEF9002801D15FF050
:10B1D000FF385FF0000905E005A8002140F82910BC
:10B1E00019F10109B9F1030F11DA01A819F80000EA
:10B1F0000028F1D001A819F80000DFF87C1A11EB43
:10B20000400030F8020C05A941F82900E8E75FF09A
:10B2100000091FE002A850F82900DFF8601A8842F0
:10B2200007DADFF85C0AF7F7BEF8012010FA09F038
:10B23000074302A850F82900DFF8481A884207DBC4
:10B24000DFF8440AF7F7AFF8012010FA09F00743D6
:10B2500019F10109B9F1030F2ADA55F8290056F856
:10B260002910401A0BF088F902A941F8290005A815
:10B2700050F829000028CDD002A850F8290005A9CF
:10B2800051F8291090FBF1F0B0F57A700BF074F9D9
:10B2900024F8190034F91900B0F5FA7FD8DDDFF889
:10B2A000EC09F7F780F8012010FA09F00743CFE71F
:10B2B000B4F904000090B4F90230B4F90020390068
:10B2C000DFF8CC09F7F76FF8002F05D0DFF8C409D5
:10B2D000F7F769F87FF00208404640B209B0BDE8D0
:10B2E000F08338B505000020ADF800000020ADF86F
:10B2F0000200F6F7D6FF040038208DF80000002089
:10B300008DF80100022300AAD0210020F7F7C1F830
:10B31000002801D1002074E000F026FB002801D1B4
:10B3200000206EE01F208DF800004B208DF80100FA
:10B33000022300AAD0210020F7F7ABF8002801D1A2
:10B3400000205EE01E208DF8000006208DF8010030
:10B35000022300AAD0210020F7F79BF8002801D192
:10B3600000204EE069208DF80000C0208DF801001B
:10B37000022300AAD0210020F7F78BF8002801D182
:10B3800000203EE0012201210320F7F7FEF9002012
:10B39000F7F7FDF938208DF8000040208DF8010006
:10B3A000022300AAD0210020F7F773F8002801D16A
:10B3B000002026E0012028702000407DC0460128A2
:10B3C00010D001212000F7F759F9BDF80200401C08
:10B3D000ADF80200BDF802003228EDDBDFF8B80856
:10B3E000F6F7E1FF012200210320F7F7CEF9002054
:10B3F000F7F7CDF900F0AEFB002801D1002000E006
:10B40000012032BD0CED00E00400FA0570B58EB0ED
:10B41000040000A80021002206C0083801250026EB
:10B420000BA80021002200230EC00C3808A8002120
:10B43000002200230EC00C3805A8002100220023A2
:10B440000EC00C3802A80021002200230EC00C38C8
:10B45000FFF7D1FA002801D1002056E0FFF7DEFB0C
:10B46000002806D00126FFF7BEFC002803D10020EB
:10B470004BE0002049E0012302AA08A90020FFF7C1
:10B48000F0FC05006DB2012D04D0DFF80808F6F7D6
:10B490008AFF1CE0012305AA0BA97FF01F00FFF71C
:10B4A000E0FC05006DB2012D04D0DFF8E007F6F7EF
:10B4B0007AFF0CE005AA02A900A8FFF770FE0500BC
:10B4C0006DB2012D03D0DFF8B807F6F76CFF2670D8
:10B4D000BDF800006070BDF900000012A070BDF85A
:10B4E0000200E070BDF9020000122071BDF80400F6
:10B4F0006071BDF904000012A071E571FFF7E6FA72
:10B50000002801D1002000E001200EB070BD80B500
:10B51000DFF888070078002809D1FFF7B8F900287C
:10B5200001D1002004E0DFF874070121017001203F
:10B5300002BD00002C6700201CB500208DF806001D
:10B540000020ADF80400F6F7ACFE040001200090E6
:10B550000DF106036B22D0210020F6F7F4FF00283E
:10B5600001D1002088E09DF806006021084216D035
:10B570006B208DF804009DF8060010F09F008DF8F8
:10B580000500022301AAD0210020F6F782FF00283F
:10B5900001D1002070E014212000F7F76FF801209E
:10B5A00000900DF106036C22D0210020F6F7CBFFAE
:10B5B000002801D100205FE06C208DF804009DF888
:10B5C000060010F0C7008DF80500022301AAD02163
:10B5D0000020F6F75EFF002801D100204CE00A2190
:10B5E0002000F7F74BF81D208DF8040043208DF85C
:10B5F0000500022301AAD0210020F6F74AFF002807
:10B6000001D1002038E01C208DF8040000208DF8C6
:10B610000500022301AAD0210020F6F73AFF0028F6
:10B6200001D1002028E020208DF8040080208DF832
:10B630000500022301AAD0210020F6F72AFF0028E6
:10B6400001D1002018E01F208DF8040080208DF823
:10B650000500022301AAD0210020F6F71AFF0028D6
:10B6600001D1002008E0DFF83806007850F0010032
:10B67000DFF82C160870012016BD00B583B000203D
:10B680008DF806000020ADF80400012000900DF1B7
:10B6900006036C22D0210020F6F755FF002801D1C7
:10B6A000002030E06C208DF804009DF8060050F07A
:10B6B00038008DF80500022301AAD0210020F6F7FA
:10B6C000E8FE002801D100201DE0DFF8D405007855
:10B6D00080070FD46B208DF8040040208DF8050002
:10B6E000022301AAD0210020F6F7D3FE002801D1C1
:10B6F000002008E0DFF8A805007810F0FE00DFF871
:10B70000A015087001200EBD28250308AC2C0120CF
:10B71000B02C0120B12C0120B22C0120B32C01202F
:10B72000AF2C0120B42C0120AE2C012000B583B039
:10B7300000208DF804000020ADF8060001200090E4
:10B7400001AB6C22D0210020F6F7FDFE002801D1CC
:10B75000002014E06C208DF806009DF8040050F0E5
:10B7600038008DF8070002230DF10602D0210020D9
:10B77000F6F78FFE002801D1002000E001200EBD69
:10B780002DE9F04186B004000D0004A8002100223C
:10B7900006C008380020ADF80C000126DFF80405CB
:10B7A0000768F6F77EFD8046DFF8FC040068401C61
:10B7B000DFF8F41408600120009004AB6B22D02164
:10B7C0000020F6F7C0FE002801D10020C9E09DF856
:10B7D000100040061AD56B208DF80C009DF8100063
:10B7E00010F0BF008DF80D00022303AAD021002025
:10B7F000F6F74FFE002801D10020B2E014214046A8
:10B80000F6F73CFFDFF8A404F6F7CDFD0120009029
:10B8100004AB6C22D0210020F6F795FE002801D160
:10B8200000209EE09DF81000382108421ED06C20B8
:10B830008DF80C009DF8100010F0C7008DF80D0079
:10B84000022303AAD0210020F6F723FE002801D10D
:10B85000002086E005214046F6F710FFDFF850048F
:10B86000F6F7A1FDDFF84C0401210160EDB200956F
:10B8700004AB3B22D0210020F6F765FE002805D15D
:10B88000DFF83404F6F78FFD00206AE09DF8110020
:10B8900020709DF8100060709DF81300A0709DF856
:10B8A0001200E0709DF8150020719DF81400607181
:10B8B000002000E0401C062806D2015DDFF8FC23D2
:10B8C000825C9142F6D00026F6B2012E18D1DFF844
:10B8D000F0030068401CDFF8E8130860DFF8E003BD
:10B8E0000068132804D1DFF8DC03F6F75CFD0BE0F9
:10B8F000DFF8CC030068142806D1FEF71FFF03E031
:10B90000DFF8BC030021016006222100DFF8AC0350
:10B91000F9F706F8DFF890030068C82190FBF1F210
:10B9200001FB120000281BD1F86AC0680290F86A77
:10B9300080680190B4F904000090B4F90230B4F9C1
:10B940000020DC480168DFF88003F6F72CFDD648BC
:10B950000068DFF87813884202DBD34800210160D9
:10B96000012006B0BDE8F08130B583B0012400208D
:10B97000ADF8060000208DF80400F6F792FC0500F3
:10B980000120009001AB6B22D0210020F6F7DBFDF7
:10B99000002801D100208BE09DF8040040061AD554
:10B9A0006B208DF806009DF8040010F0BF008DF8A4
:10B9B000070002230DF10602D0210020F6F769FDF1
:10B9C000002801D1002073E014212800F6F756FE6C
:10B9D000BF48F6F7E8FC1D208DF8060008208DF81A
:10B9E000070002230DF10602D0210020F6F751FDD9
:10B9F000002801D100205BE00120009001AB6C2207
:10BA0000D0210020F6F79FFD002801D100204FE053
:10BA10006C208DF806009DF8040050F080008DF831
:10BA200004009DF8040050F007008DF804009DF814
:10BA3000040010F0C7008DF804009DF804008DF894
:10BA4000070002230DF10602D0210020F6F721FDA8
:10BA5000002801D100202BE00120009001AB6B22D7
:10BA6000D0210020F6F76FFD002801D100201FE053
:10BA70006B208DF806009DF8040010F0BF008DF8D3
:10BA800004009DF8040050F020008DF804009DF89B
:10BA900004008DF8070002230DF10602D0210020DA
:10BAA000F6F7F7FC002801D1002001E02000C0B229
:10BAB0003EBD80B50020ADF80000FFF755FF00281F
:10BAC00001D1002045E01F208DF800004B208DF8AB
:10BAD0000100022300AAD0210020F6F7DAFC00289A
:10BAE00001D1002035E01E208DF8000006208DF8E1
:10BAF0000100022300AAD0210020F6F7CAFC00288A
:10BB000001D1002025E069208DF80000C0208DF8CB
:10BB10000100022300AAD0210020F6F7BAFC002879
:10BB200001D1002015E0012201210320F6F72DFEAE
:10BB300038208DF8000040208DF80100022300AA73
:10BB4000D0210020F6F7A5FC002801D1002000E05C
:10BB5000012002BD80B50020ADF8000001220021C7
:10BB60000320F6F712FE38208DF8000000208DF833
:10BB70000100022300AAD0210020F6F78AFC002849
:10BB800001D1002058E06B208DF8000000208DF8D6
:10BB90000100022300AAD0210020F6F77AFC002839
:10BBA00001D1002048E01D208DF8000000208DF814
:10BBB0000100022300AAD0210020F6F76AFC002829
:10BBC00001D1002038E06C208DF800003448007866
:10BBD000032803D100208DF8010012E030480078DE
:10BBE000022803D138208DF801000AE02C480078A3
:10BBF000012803D107208DF8010002E03F208DF8D5
:10BC00000100022300AAD0210020F6F742FC002800
:10BC100001D1002010E069208DF8000000208DF88F
:10BC20000100022300AAD0210020F6F732FC0028F0
:10BC300001D1002000E0012002BD80B5017801297A
:10BC400005D1FFF74EFB00280AD1002009E001785A
:10BC5000022905D1FFF7DAFB002801D1002000E01E
:10BC6000012002BD80B51B490020FAF781F81A496E
:10BC70000B20FAF77DF801BD900C0308003E490047
:10BC8000B825030801EFE700C0250308B025030825
:10BC9000A4240308C8250308D0250308FB2B012092
:10BCA000EC2E012008400020B42D0120D8250308E7
:10BCB000E0250308042E0120E8250308E42D0120D7
:10BCC000702E01208425030840250308A186010069
:10BCD000F0250308F02303081424030810B50024FA
:10BCE000DFF8500C007800280AD1FEF7D0FD0028BC
:10BCF00001D1002007E0DFF83C0C0121017000E0D9
:10BD000001242000C0B210BD1CB500208DF8060033
:10BD10000020ADF80400F6F7C4FA040001200090FA
:10BD20000DF106036B22D0210120F6F70CFC002850
:10BD300001D1002068E09DF806006021084216D07D
:10BD40006B208DF804009DF8060010F09F008DF820
:10BD50000500022301AAD0210120F6F79AFB002852
:10BD600001D1002050E01E212000F6F787FC0120C1
:10BD700000900DF106036C22D0210120F6F7E3FBC1
:10BD8000002801D100203FE06C208DF804009DF8D0
:10BD9000060010F0F8008DF80500022301AAD0215A
:10BDA0000120F6F776FB002801D100202CE00A21C3
:10BDB0002000F6F763FC1B208DF8040018208DF896
:10BDC0000500022301AAD0210120F6F762FB00281A
:10BDD00001D1002018E01A208DF8040003208DF80E
:10BDE0000500022301AAD0210120F6F752FB00280A
:10BDF00001D1002008E0DFF8400B007850F002008D
:10BE0000DFF8341B0870012016BD00B583B0002098
:10BE10008DF806000020ADF80400012000900DF11F
:10BE200006036C22D0210120F6F78DFB002801D1FA
:10BE3000002030E06C208DF804009DF8060050F0E2
:10BE400007008DF80500022301AAD0210120F6F792
:10BE500020FB002801D100201DE0DFF8DC0A00787B
:10BE6000C0070FD46B208DF8040040208DF805002A
:10BE7000022301AAD0210120F6F70BFB002801D1F3
:10BE8000002008E0DFF8B00A007810F0FD00DFF8CD
:10BE9000A81A087001200EBD00B583B000208DF8EF
:10BEA00004000020ADF806000120009001AB6C22D8
:10BEB000D0210120F6F747FB002801D1002014E033
:10BEC0006C208DF806009DF8040050F007008DF8F6
:10BED000070002230DF10602D0210120F6F7D9FA5E
:10BEE000002801D1002000E001200EBD7FB5040034
:10BEF00002A80021002206C0083800260020ADF864
:10BF00000400F6F7CEF905000120009002AB6B2289
:10BF1000D0210120F6F717FB002801D1002083E093
:10BF20009DF80800400625D56B208DF804009DF88B
:10BF3000080010F0BF008DF80500022301AAD021EF
:10BF40000120F6F7A6FA002801D100206CE032218A
:10BF50002800F6F793FBDFF8E409F6F724FA002649
:10BF600003E0F6B200203055761CF6B2062EF8DB60
:10BF7000012059E00120009002AB6C22D021012069
:10BF8000F6F7E1FA002801D100204DE09DF8080005
:10BF90000721084225D06C208DF804009DF8080088
:10BFA00010F0F8008DF80500022301AAD02101202D
:10BFB000F6F76FFA002801D1002035E00A212800A9
:10BFC000F6F75CFBDFF87809F6F7EDF9002603E0F9
:10BFD000F6B200203055761CF6B2062EF8DB0120B2
:10BFE00022E00620009002AB4322D0210120F6F788
:10BFF000AAFA002805D1DFF84C09F6F7D4F9002099
:10C0000012E09DF8090020709DF8080060709DF80E
:10C010000B00A0709DF80A00E0709DF80D002071E3
:10C020009DF80C006071012004B070BD2DE9F64F41
:10C03000ADF63C6D05000020ADF8080003A8142102
:10C04000F8F7ACFB002608A80021002200230EC050
:10C050000C385FF0000940F68C1068444FF496618C
:10C06000F8F79CFBFFA8E0304FF49661F8F796FBD9
:10C070000BA84FF49661F8F791FB5FF000080027DA
:10C0800000240020070000E07F1C032F80F2BA800C
:10C090006B208DF80800781C8DF80900022302AA95
:10C0A000D0210120F6F7F5F9002801D1002099E10F
:10C0B0003220FEF7B1FB6A208DF8080044208DF88D
:10C0C0000900022302AAD0210120F6F7E2F9002894
:10C0D00001D1002086E1012409E019EB060608A839
:10C0E00050F8270019EB000008A941F827002000AC
:10C0F000441E012875DB23208DF8080070208DF880
:10C100000900022302AAD0210120F6F7C2F9002873
:10C1100001D1002066E14B20FEF77EFB23208DF845
:10C12000080000208DF80900022302AAD021012076
:10C13000F6F7AFF9002801D1002053E1022000906A
:10C1400003AB7222D0210120F6F7FDF9002801D1BE
:10C15000002047E103A8FEF748FC00EE100AB8EE05
:10C16000C00A10EE100AFCF7E7F8DFF8DC27DFF86A
:10C17000DC37F6F779FDF7F7A1F88146B9F1480009
:10C180000128B4DB5FF000081DE003A8FEF72DFCDA
:10C1900018EB060140F68C126A4422F811000DF1EA
:10C1A0000E00FEF722FC18EB0601FFAAE03222F88F
:10C1B000110004A8FEF719FC18EB06010BAA22F8DF
:10C1C000110018F10108C84587DA0620009003AB7A
:10C1D0007422D0210120F6F7B6F90028D5D100202D
:10C1E00000E123208DF8080000208DF809000223CB
:10C1F00002AAD0210120F6F74CF900287FF444AFC1
:10C200000020EFE0002E01D0340000E001245FF0B8
:10C21000000800200021C5E9000100200021C5E937
:10C22000020100200021C5E9040122E0D5E9000156
:10C2300040F68C126A4432F91820D31780185941FD
:10C24000C5E90001D5E90201FFAAE03232F9182060
:10C25000D31780185941C5E90201D5E904010BAA99
:10C2600032F91820D31780185941C5E9040118F193
:10C270000108B045DADBD5E900012200E317FDF73C
:10C28000A7F8C5E90001D5E902012200E317FDF78F
:10C290009FF8C5E90201D5E904012200E317FDF783
:10C2A00097F8C5E904015FF00008DDF83C0E0022B4
:10C2B0000023C0E90023DDF83C0E00220023C0E982
:10C2C0000223DDF83C0E00220023C0E9042382E0B3
:10C2D000DDF83C2ED2E90001CDE9000140F68C10DA
:10C2E000684430F91800C117D5E90023801A994134
:10C2F00040F68C126A4432F918A05FEAEA7BD5E96D
:10C300000023BAEB02027BEB0303A2FB00AB02FBB0
:10C3100001BB03FB00BBDDE9000110EB0A0051EBA0
:10C320000B01DDF83C2EC2E90001DDF83C2ED2E91C
:10C330000201CDE90001FFA8E03030F91800C11773
:10C34000D5E90223801A9941FFAAE03232F918A0F8
:10C350005FEAEA7BD5E90223BAEB02027BEB030337
:10C36000A2FB00AB02FB01BB03FB00BBDDE900014C
:10C3700010EB0A0051EB0B01DDF83C2EC2E9020183
:10C38000DDF83C2ED2E90401CDE900010BA830F91B
:10C390001800C117D5E90423801A99410BAA32F974
:10C3A00018A05FEAEA7BD5E90423BAEB02027BEB33
:10C3B0000303A2FB00AB02FB01BB03FB00BBDDE9F7
:10C3C000000110EB0A0051EB0B01DDF83C2EC2E935
:10C3D000040118F10108B045FFF67AAFDDF8400E10
:10C3E000066001200DF6446DBDE8F08F2DE9F043A5
:10C3F00089B004000D00160001275FF0000801A8B5
:10C40000002101600320009001AB0022D021012017
:10C41000F6F799F8002801D15FF0FF375FF00009C7
:10C4200007E04FFA89F905A8002140F8291019F111
:10C4300001094FFA89F9B9F1030F17DA4FFA89F9AF
:10C4400001A819F800000028EBD04FFA89F901A8DB
:10C4500019F80000DFF8F81411EB400030F8020C76
:10C460004FFA89F905A941F82900E0E75FF00009D2
:10C4700025E04FFA89F902A850F82900DFF8D41412
:10C48000884208DADFF8D004F5F78DFF012010FAB2
:10C4900009F050EA08084FFA89F902A850F8290073
:10C4A000DFF8B814884208DBDFF8B404F5F77BFF47
:10C4B000012010FA09F050EA080819F101094FFAB1
:10C4C00089F9B9F1030F3BDA4FFA89F955F82900D8
:10C4D0004FFA89F956F82910401A0AF04DF84FFA28
:10C4E00089F902A941F829004FFA89F905A850F8FD
:10C4F00029000028BDD04FFA89F902A850F8290078
:10C500004FFA89F905A951F8291090FBF1F0B0F51F
:10C510007A700AF031F84FFA89F924F819004FFAC5
:10C5200089F934F91900B0F5FA7FC6DDDFF8340473
:10C53000F5F739FF012010FA09F050EA0808BCE7C6
:10C540004FFA88F8B8F1000F05D0DFF81C04F5F7B2
:10C550002AFF7FF00207380040B209B0BDE8F0833F
:10C560002DE9F0479CB004005FF0010801250CA8FC
:10C570001821F8F713F906A81821F8F70FF902A8FF
:10C580000021016000A80021002206C008385FF0E9
:10C59000000A18A80021002200230EC00C3815A89C
:10C5A0000021002200230EC00C3812A80021002216
:10C5B00000230EC00C3803A80021002200230EC067
:10C5C0000C380026DFF8A403D0F80490FEF713FA25
:10C5D000002801D1002049E1FEF720FB80465FFAE8
:10C5E00088F8B8F1010F0AD15FF0010A02AA06A982
:10C5F0000CA8FFF71BFD002805D1002036E1FEF74F
:10C6000065FA002032E1FEF7EEFB002801D10020A0
:10C610002CE1002303AA15A90020FEF722FC050047
:10C620006DB2012D03D0761CD148F5F7BCFE002376
:10C6300012AA18A97FF01F00FEF713FC05006DB2C7
:10C64000012D03D0B61CCB48F5F7ADFE18AA15A9ED
:10C6500000A8FFF7CBFE05006DB2012D03D0361DFB
:10C66000C548F5F7A0FEDDE90601002901D1002843
:10C670000BD0DDE90801002901D1002805D0DDE952
:10C680000A01002905D1002803D1BC48F5F78BFE2B
:10C69000083600273AE0FFB20CA810EBC700D0E93B
:10C6A000002340F2411000218B420FDB01DC82426B
:10C6B0000CD31036FFB20CA810EBC702D2E9000170
:10C6C0000200FFB23900AE48F5F76DFEFFB206A8D2
:10C6D00010EBC702D2E90001029AD317FCF778FEEB
:10C6E000002912DB02DCB0F5C85F0ED34036FFB282
:10C6F00006A810EBC702D2E90001029990FBF1F203
:10C70000FFB239009F48F5F74EFE7F1CFFB2032FA2
:10C71000C1DB36B2002E1AD100220CE0D2B219EBE6
:10C720004203D2B20CA810EBC206D6E90001800089
:10C73000A3F85800521CD2B2032AEFDBB9F95C30DF
:10C74000B9F95A20B9F958108F48F5F72CFE84F83A
:10C7500000A0BDF800006070BDF900000012A070DC
:10C76000BDF80200E070BDF9020000122071BDF8B2
:10C7700004006071BDF904000012A071E571029817
:10C78000207202980012607202980014A07202983F
:10C790000016E072DDE90C012073DDE90C0100B246
:10C7A00000126073DDE90C010014A073DDE90C01D7
:10C7B0000016E073DDE90E012074DDE90E0100B220
:10C7C00000126074DDE90E010014A074DDE90E01B1
:10C7D0000016E074DDE910012075DDE9100100B2FA
:10C7E00000126075DDE910010014A075DDE910018B
:10C7F0000016E075DDE906012076DDE9060100B2EC
:10C8000000126076DDE906010014A076DDE906017C
:10C810000016E076DDE908012077DDE9080100B2C5
:10C8200000126077DDE908010014A077DDE9080156
:10C830000016E077DDE90A0184F82000DDE90A014D
:10C8400000B2001284F82100DDE90A01001484F826
:10C850002200DDE90A01001684F82300FEF736F90C
:10C86000002801D1002001E04046C0B21CB0BDE864
:10C87000F08730B583B004000020ADF8040000203C
:10C880003A494D68697A002907D1286E4068804787
:10C89000F5F707FD0A21F5F7F1FE0220009001AB44
:10C8A0004122D0210120F5F74EFE002801D10020C1
:10C8B00017E09DF805009DF8041050EA01200321BF
:10C8C00010FB01F04FF47A7190FBF1F015302070FD
:10C8D00000206070687A002802D1286E8068804746
:10C8E00001203EBD80B50178002905D1FFF738FE53
:10C8F00000280AD1002009E00178012905D1FFF7BD
:10C90000B8FF002801D1002000E0012002BD80B561
:10C91000C0B2062806D10800FFF7ABFF002801D1FE
:10C92000002000E0012002BD80B518490120F9F780
:10C930001FFA01BDFB2B0120EC2E0120F825030876
:10C9400000260308082603082D211FF46C56C53F56
:10C95000900E030830FD13001826030879E2D10079
:10C960002026030810260308282603080840002074
:10C9700030260308382603084026030894250308B8
:10C98000C424030858250308702503083824030825
:10C99000DFF88005704730B583B00020ADF80600A1
:10C9A0008DF804000120009001AB00221821022024
:10C9B000F5F7C9FD04469DF8040048281FD1312031
:10C9C0008DF806000DF106050120687002230DF1B7
:10C9D000060218211846F5F75CFD00280DD031201D
:10C9E0008DF806000020687002230DF10602182160
:10C9F0001846F5F74EFD002802D100203EBD002468
:10CA000018220021DFF80C05F5F728FC20463EBD72
:10CA100070B582B00020ADF8000009F0B6FD044604
:10CA2000DFF8F4048168497AC268527A51180069C3
:10CA3000407A0818012801DB012076BDDFF8DC54BC
:10CA4000687801281CD032208DF8000000AE01204B
:10CA50007070022300AA18211846F5F71AFD002865
:10CA60000CD031208DF8000001207070022300AA44
:10CA700018211846F5F70DFD002803D1002076BDDA
:10CA800001202870281D61698847012076BD38B5CE
:10CA90000020ADF8000009F078FD0446DFF87804C6
:10CAA0008168497AC268527A51180069407A081838
:10CAB000022801DB012032BDDFF86054287801280C
:10CAC00012D031208DF8000000208DF801000223E3
:10CAD00000AA18211846F5F7DCFC002801D1002037
:10CAE00032BD0020687001E000202870281D2169F7
:10CAF0008847012032BD80B50020ADF8000031200C
:10CB00008DF8000000208DF80100022300AA1821F2
:10CB10001846F5F7BEFC002801D1002002BD012017
:10CB200002BD7CB504460020ADF806008DF8040077
:10CB30000120009001AB002218210220F5F703FD2F
:10CB400005469DF80400482829D131208DF80600BB
:10CB50000DF106061F20707002230DF10602182148
:10CB60001846F5F796FC002817D0032000902346BE
:10CB7000602218210220F5F7E6FC00280DD03120B4
:10CB80008DF806000020707002230DF106021821B6
:10CB90001846F5F77EFC002802D1002076BD00255E
:10CBA000284676BD0021DE4A02E00B5C8B54491C0E
:10CBB0001B29FADBDB48C0F8D423012070472DE99C
:10CBC000F04387B004460D4616461F464FF0000856
:10CBD0004046ADF8040002A841460A460B460EC086
:10CBE0004FF0050906C00120009002AB1022182169
:10CBF0000220F5F7A8FC9DF80810C9070ED50128FA
:10CC00000CD1082000900DF10903112218210220F7
:10CC1000F5F799FC002807D140467BE04846A0F193
:10CC2000010980B20028DED1BF489DF808100170CC
:10CC300002A90A7A4270CA7982704A78C2708A78E8
:10CC40000271CA7842710A7982714A79C27189790E
:10CC500001720AE002A800EB48008178407810EBEE
:10CC6000012024F8180008F10108B8F1030FF1DBE6
:10CC7000A948D0F80C8008F10C0999F81520214634
:10CC8000D9F80C00D8F80C30C018F7F749FE404628
:10CC900003F00AF999F81520D9F80C00D8F80C100F
:10CCA00041182046F7F73CFEDFF8788205AA2146B6
:10CCB000404609F0BFFE98F9F4023860B8F8EE007B
:10CCC000288008F2EE00418869808188A9808189E6
:10CCD0002180C1896180008AA08020882988401A2B
:10CCE000308060886988401A7080A088A988401ABE
:10CCF000B08031208DF8040001208DF8050002235A
:10CD000001AA18211846F5F7C4FB002801D100201C
:10CD100000E0012007B0BDE8F08330B585B00446DF
:10CD20000020ADF8040002A800210A460B460EC000
:10CD300005250120009002AB102218210220F5F7F2
:10CD400002FC9DF80810C9070ED501280CD1082057
:10CD500000900DF10903112218210220F5F7F3FBD1
:10CD6000002806D1002029E02846451E80B2002870
:10CD7000DFD16D489DF80810017002A90A7A42704F
:10CD80004878207088786070C878A0700879E07062
:10CD9000487920719DF80E00607131208DF80400F3
:10CDA00001208DF80500022301AA18211846F5F785
:10CDB00070FB002801D1002000E0012005B030BD4B
:10CDC0002DE9F04104460025FDF7B4FC0746FFF7C6
:10CDD000DFFD06465048D0F81080F86E40070BD4AF
:10CDE00006F1140306F10C02B11D3046FFF7E7FE11
:10CDF000002801D1284651E098F80A00012848D1BE
:10CE000049480178217041786170C178A170017939
:10CE1000E1704179217181796171C179A171007AE3
:10CE2000E0714048818D2172B0F92C1009126172B5
:10CE300000F12C014A88A272B1F902201212E272AA
:10CE40008A882273B1F9041009126173B0F8F410E2
:10CE5000A173B0F9F4100912E173F4304188217420
:10CE6000B0F90210091261748188A174B0F904004C
:10CE70000012E074284620750FE006EB4500C188DB
:10CE800004F8151004EB4501B0F9060000124870D3
:10CE90006D1C032DF1DB7069A0710120BDE8F081EC
:10CEA000F8B504460025FDF745FC0746FFF770FD81
:10CEB0000646F86E000705D52046FFF72EFF00282E
:10CEC00026D109E006F1140306F10C02B11D30462B
:10CED000FFF775FE002814D12846F2BD36F815007C
:10CEE00004F8150004EB450036F9151009124170DD
:10CEF00006EB45018A898271B1F90C100912C171E2
:10CF00006D1C032DEADB182231460248F7F708FDB5
:10CF10000120F2BDA42A012008400020982B012006
:10CF2000502A0120B0D60020D02C01207CB5044628
:10CF30000020ADF806008DF80400F5F7B2F90546BB
:10CF40000120009001AB002218210220F5F7FBFA26
:10CF50009DF80410482932D131208DF806000DF1DA
:10CF600006061F20707002230DF1060218211846D4
:10CF7000F5F78FFA00281BD031208DF8060000202D
:10CF8000707002230DF1060218211846F5F781FA98
:10CF900000280DD001212846F5F770FB01200090F4
:10CFA00001AB312218210220F5F7CDFA002801D17A
:10CFB000002076BD9DF804002070012076BDFF2181
:10CFC000217076BD2DE9F04387B0044604A8002106
:10CFD0000A460B460EC00846ADF80C004FF0050996
:10CFE000F5F75FF905460220009004AB00221821F6
:10CFF000F5F7A9FA06469DF81000482840F00B8185
:10D000009DF81000207004AF7878607031208DF8A2
:10D010000C000DF10C081F2088F80100022303AA60
:10D0200018211846F5F735FA002800F0F58003209E
:10D03000009004AB602218210220F5F784FA002842
:10D0400000F0EA809DF81000A0707878E070B87861
:10D05000207131208DF80C00002088F80100022397
:10D0600003AA18211846F5F714FA002800F0D48016
:10D070000120009004AB312218210220F5F763FA59
:10D08000002800F0C9809DF81000607531208DF8EF
:10D090000C00012088F80100022303AA1821184679
:10D0A000F5F7F7F9002800F0B7801E212846F5F7BC
:10D0B000E5FA0120009004AB102218210220F5F7B8
:10D0C00042FA06469DF81000C0070DD5012E0BD17F
:10D0D000082000900DF11103112218210220F5F70C
:10D0E00032FA002806D160E04846A0F1010980B27A
:10D0F0000028DED1B87902907879019038790090D3
:10D10000FB78BA7879780FF26C10F5F74CF9B878AB
:10D11000797811EB00203979FA7812EB0121BA798C
:10D120007B7913EB022203461BB21B126371A071C1
:10D13000084600B20012E0712172104600B20012DF
:10D140006072A2729DF81000E072387A207331206C
:10D150008DF80C00102088F80100022303AA182182
:10D160001846F5F796F9002856D01E212846F5F7FF
:10D1700085FA4FF005090120009004AB1022182118
:10D180000220F5F7E0F906469DF81000C0070ED51D
:10D19000012E0CD1082000900DF11103112218214D
:10D1A0000220F5F7D0F9002807D1002035E04846E5
:10D1B000A0F1010980B20028DDD1B8790290787918
:10D1C000019038790090FB78BA7879780FF2C00036
:10D1D000F5F7E9F8B878797811EB00203979FA7821
:10D1E00012EB0121BA797B7913EB022203461BB2C1
:10D1F0001B126373A073084600B20012E07321741F
:10D20000104600B200126074A2749DF81000E07421
:10D21000387A207500E00026304607B0BDE8F0837C
:10D2200018B404460B4611460020032C04D0042CED
:10D2300005D0072C06D008E0184614BC71E4184647
:10D2400012BC73E6184612BCACE412BC704710B5B1
:10D250000FF2580421460220F8F78AFD0FF2700100
:10D260000420F8F785FD21460320BDE81040F8F7BB
:10D270007FBD0000474D53312D25642C2025642CA3
:10D280002025642C2025642C2025642C2025640076
:10D29000474D53322D25642C2025642C2025642CE9
:10D2A0002025642C2025642C2025640097C90008C3
:10D2B00011CA00088FCA0008F7CA00080000000061
:10D2C000A1CE000800000000C5CF000821D2000850
:10D2D00097C9000811CA00088FCA0008F7CA0008D9
:10D2E00000000000C1CD000800000000C5CF00080C
:10D2F00021D2000838B50020ADF800000446F4F74C
:10D30000D0FF05464FF480512046F5F72EFA0A214A
:10D310002846F5F7B3F900E0641C062C12D2DFF8BA
:10D32000080D215C8DF800102018007A8DF801009E
:10D33000022300AA72210720F5F7ABF80028EBD1F1
:10D34000002032BD012032BD2DE9FC410746884650
:10D35000FDF7F0F904460020ADF80400DFF8CC5CDE
:10D36000288C0646B8F1000F02D03843288401E02B
:10D37000B8432884012000900DF10603AB227221EE
:10D380000620F5F7E0F8002801D10020C5E1288C3F
:10D390000E2800F2A681DFE810F00F00A4011C00A7
:10D3A000A4013F00A4013F00A401B700A401B700FD
:10D3B000A401B700A401B70080208DF8040000206C
:10D3C0008DF805009DF8060000F0FD008DF80600C0
:10D3D00087E116F00C0F01D00120687581208DF8CF
:10D3E000040001AEEE207070022301AA7221092010
:10D3F000F5F74FF8002801D100208EE17078E87031
:10D4000080208DF80400032070709DF8060000F065
:10D41000FD008DF8060064E13046000701D4022EBD
:10D4200001D1012068759D208DF8040001AE0C200B
:10D430007070022301AA72210920F5F72AF800284A
:10D4400001D1002069E19E208DF804000C2070704D
:10D45000022301AA72210920F5F71BF8002801D147
:10D4600000205AE181208DF80400FD207070022315
:10D4700001AA72210920F5F70CF8002801D100203B
:10D480004BE17078E8708E208DF80400287A00282F
:10D4900012D00C218F2009F0E8FD04218F2009F023
:10D4A000BAFD3021902009F0E0FD3021902009F0F4
:10D4B000B2FD4520707011E00C218F2009F0D5FDE0
:10D4C00008218F2009F0A7FD3021902009F0CDFD23
:10D4D0001021902009F09FFD82207070022301AA84
:10D4E00072210920F4F7D5FF002801D1002014E1B2
:10D4F00080208DF80400272070709DF8060000F051
:10D50000FD008DF80600ECE016F0080701AE4FD1E3
:10D5100009F0B4FE01206875A4208DF804000020F5
:10D520007070DFF88C0D00210170022301AA7221B6
:10D530000920F4F7AEFF002801D10020EDE0A5207E
:10D540008DF8040000207070DFF8680D0021017074
:10D55000022301AA72210920F4F79BFF002801D1C0
:10D560000020DAE0A7208DF8040000207070DFF8BA
:10D57000480D00210170022301AA72210920F4F74D
:10D5800088FF002801D10020C7E0A9208DF8040001
:10D5900000207070DFF8980D00210170022301AAAD
:10D5A00072210920F4F775FF002801D10020B4E0B2
:10D5B00081208DF80400FE207070022301AA7221E0
:10D5C0000920F4F766FF002801D10020A5E070785B
:10D5D000E8708E208DF80400287A002812D00C21E3
:10D5E0008F2009F042FD04218F2009F014FD302125
:10D5F000902009F03AFD3021902009F00CFD4F20D9
:10D60000707011E00C218F2009F02FFD08218F2070
:10D6100009F001FD3021902009F027FD2121902003
:10D6200009F0F9FC84207070022301AA72210920FC
:10D63000F4F72FFF002801D100206EE0002F20D149
:10D64000B4F88A00B4F88C10401AE883B4F88A1051
:10D650008900A98389B2FF2901DBFE21A98380B259
:10D660008100652902DB6420E88301E08000E88313
:10D67000A98BE88B0A1AEA8392B20FF2A400F4F79E
:10D6800092FEA6208DF80400287A00280AD0602196
:10D69000A32009F0EAFC4121A32009F0BCFC57209B
:10D6A000707009E06021A32009F0DFFC4121A32074
:10D6B00009F0B1FC8B207070022301AA72210920AD
:10D6C000F4F7E7FE002801D1002026E080208DF845
:10D6D0000400672070709DF8060040F002008DF88D
:10D6E0000600022301AA72210920F4F7D2FE0028C5
:10D6F00001D1002011E0AB208DF804009DF8060058
:10D700008DF80500022301AA72210920F4F7C1FE59
:10D71000002801D1002000E00120BDE8F6810000D2
:10D72000233E6755703D25642C674C6F3D25640092
:10D7300010B534220021DFF8A00CF4F78FFDDFF8DC
:10D74000EC480120A0710AF02BF909F0B9FC012086
:10D750002073DFF8D00D0021017010BD10B582B02C
:10D760000FF25C00F4F71FFE0020ADF800008020EF
:10D770008DF8000000AC03206070022300AA722123
:10D780000620F4F786FE002818D0DFF8A008817A7A
:10D7900000290DD08C218DF800100021617081705E
:10D7A000022300AA72210620F4F773FE002805D098
:10D7B000FFF7BEFF01210020FFF7C6FD13BD0000EB
:10D7C000233E484C5300000010B582B00FF24000D9
:10D7D000F4F7E9FD0020ADF80000044600E0641C09
:10D7E000052C12D2DFF8700D215C8DF80010201886
:10D7F000007A8DF80100022300AA72210720F4F7B5
:10D8000048FE0028EBD1002016BD012016BD000007
:10D81000233E50525000000030B583B00FF2880014
:10D82000F4F7C1FD0020ADF804008DF80600DFF824
:10D83000FC47607180208DF8040001AD0320687002
:10D84000022301AA72210720F4F723FE002801D148
:10D8500000203EBD8C208DF8040000206870A07070
:10D86000022301AA72210720F4F713FE002801D138
:10D8700000203EBD0120607201460420FFF764FDD8
:10D88000002801D100203EBD012000900DF10603CB
:10D89000E52272210720F4F756FE002801D100206E
:10D8A0003EBD01203EBD0000233E50524F0000000F
:10D8B00000B583B00FF26400F4F775FD0020ADF8F9
:10D8C00006008DF8040080208DF8060003208DF8F6
:10D8D000070002230DF1060272210720F4F7D9FD9B
:10D8E000002801D100200EBDDFF840070021417261
:10D8F0000420FFF729FD002801D100200EBD0120E2
:10D90000009001ABE52272210720F4F71CFE0028ED
:10D9100001D100200EBD01200EBD0000233E50525B
:10D92000430000000120704730B583B0044600205A
:10D93000ADF80400DFF8F456A87B00282CD1A87AB3
:10D94000002802D0287C207031E0012000900DF1E9
:10D950000503932272210720F4F7F5FD00280DD06E
:10D960009DF80500800722D50120009001AB9C2284
:10D9700072210720F4F7E7FD002801D100203EBD09
:10D980009DF80400697951FA80F080B24008207057
:10D990009DF8040068710AE0012808D1DFF8380A10
:10D9A00041696A79891849102170406968710120BC
:10D9B0003EBD2DE9F04391B00446FCF7BBFE0546A1
:10D9C000F4F76FFC06460020ADF80800ADF80C0037
:10D9D0008DF80A00012000900DF10A0393227221B4
:10D9E0000720F4F7B0FD002801D1002025E2022035
:10D9F000009003AB942272210720F4F7A4FD0028C5
:10DA000001D1002019E2DFF824769DF80D009DF881
:10DA10000C1041EA0020DFF8181D4843F978C1F5E1
:10DA200080713A79DFF80C3DD25C12FB01F140F2D3
:10DA30004232514390FBF1F0797B002902D0B97A50
:10DA4000002901D1B86208E0B86AF97D4A1CFA756C
:10DA5000062902DB00217973F975397A00290CD186
:10DA600041F6593188422DDB01213972F8620020DC
:10DA70003876FFF773FE0120DFE1F96A411A44F6B8
:10DA80002162914215DA40F6B831884218DA9DF8E1
:10DA90000A20920614D53A7E531C3B76C92A04DA32
:10DAA000BA7A002A0ED188420CDA884201DA0021C3
:10DAB0003972F86200203876FFF750FE0120BCE191
:10DAC000002038769DF80A00800640F1B5810020DC
:10DAD000B873012000900DF10A03932272210720F0
:10DAE000F4F731FD002801D10020A6E19DF80A00DD
:10DAF00080071BD50120009003AB9C2272210720D8
:10DB0000F4F721FD002801D1002096E19DF80C00DA
:10DB1000797951FA80F080B2400860709DF80C006D
:10DB2000F8739DF80C00787160783874387B0028A1
:10DB300002D00020387371E1DFF81C8D607888F81E
:10DB40000000B87900280AD009F0C4FA002806D1EC
:10DB5000B87A002803D0607809F0CEFA7AE0787AB3
:10DB6000002839D0B87AB978084335D1002030750B
:10DB70008C208DF808000DF10809202089F801009B
:10DB8000B870022302AA72210720F4F782FC002851
:10DB900001D1002051E189208DF80800002089F88A
:10DBA0000100022302AA72210720F4F772FC002868
:10DBB00001D1002041E18B208DF80800B5F88A00E2
:10DBC00089F80100022302AA72210720F4F761FC00
:10DBD000002801D1002030E1B87A00280ED105F1EB
:10DBE0008A004288B5F88A100FF25420F4F7DBFB64
:10DBF00061780FF25C20F4F7D6FB2BE0414684B04D
:10DC000068461822F4F724FF0FBC09F0DAFE04A8D6
:10DC100009F03DFFDFF8C49C484604A93422F4F71C
:10DC200017FF99F81C00002807D034224946DFF876
:10DC3000A807F6F775FE0120787009F11C00417DF8
:10DC400088F81410817D88F81510007D002801D017
:10DC5000FFF76EFD787A002800F0E080B87A00289F
:10DC600040F0DC806078B5F88A10884231D3307D8E
:10DC700000282ED10120F87120702078307589207D
:10DC80008DF808000DF1080905F18A00408889F82F
:10DC90000100022302AA72210720F4F7FAFB0028F0
:10DCA00001D10020C9E08B208DF80800FF2089F801
:10DCB0000100022302AA72210720F4F7EAFB0028E0
:10DCC00001D10020B9E061780FF29010F4F76BFBFE
:10DCD000A4E005F28A0041886278914231D3317D17
:10DCE00001292ED10120F871002020702078307594
:10DCF00089208DF808000DF10809002089F801003D
:10DD0000022302AA72210720F4F7C3FB002801D1E5
:10DD1000002092E08B208DF80800B5F88A0089F881
:10DD20000100022302AA72210720F4F7B2FB0028A7
:10DD300001D1002081E061780FF22810F4F733FB65
:10DD40006CE0B5F88A106278914235D3317D0029B4
:10DD500032D1797C01292FD10120F8710020207067
:10DD6000207830750020787489208DF808000DF136
:10DD70000809002089F80100022302AA7221072065
:10DD8000F4F787FB002801D1002056E08B208DF8A6
:10DD90000800B5F88A0089F80100022302AA72215E
:10DDA0000720F4F776FB002801D1002045E00FF2B0
:10DDB000BC00F4F7F8FA31E06178428891422DD343
:10DDC000317D01292AD1797C012927D1002179745B
:10DDD00089218DF808100DF10809408889F80100A3
:10DDE000022302AA72210720F4F753FB002801D175
:10DDF000002022E08B208DF80800FF2089F8010028
:10DE0000022302AA72210720F4F743FB002801D164
:10DE1000002012E00FF25C00F4F7C5FA0120009038
:10DE200003ABE52272210720F4F78DFB002801D116
:10DE3000002002E0012000E0002011B0BDE8F083E6
:10DE4000233E55703D25642C4C6F3D256400000039
:10DE5000233E50524157202564000000233E50319C
:10DE600020256400233E503220256400233E526565
:10DE700054483100233E5265544832002DE9F8439E
:10DE800004460D46694EB07C002805D000F01EFF08
:10DE90000020F0743075C5E0FCF74CFC804600278C
:10DEA0003846ADF800002078072823D16078FF2895
:10DEB00020D12946601CFFF737FD6078B8F88A103A
:10DEC000884208D301202070627821780FF2601018
:10DED000F4F769FA0CE0B8F88C006178884207D34F
:10DEE00038462070627821780FF24410F4F75BFA1C
:10DEF000012097E00020F074307529462046FFF796
:10DF000058FD00280DD0707A00280AD0F07900283A
:10DF100007D00FF23010F4F746FA0020F07101201C
:10DF20003075B07A002877D0DFF8648DD8F8189073
:10DF300009F10C00417DC068D9F80C20801800F070
:10DF40004DFA002868D0DFF8DC050078411E8941D1
:10DF5000C90FF1747078002801D000207070707AB9
:10DF6000002857D0D9F80C0040780DF1000989F845
:10DF70000100B18B814218D2F4F793F9007D00289B
:10DF800013D1707E401C7076C0B202282DD10020C3
:10DF900070760127F4F785F93946017599F8011073
:10DFA0000FF2A800F4F7FFF91FE099F80100F18BD8
:10DFB000884218D2F4F775F9007D012813D1707EDC
:10DFC000401C7076C0B202280FD100207076012765
:10DFD000F4F767F90021017599F801100FF2780044
:10DFE000F4F7E1F901E000207076002F12D0D8F8A4
:10DFF0001C80F4F756F9007D8DF8000008F10C0044
:10E00000427D00A9C068D8F80C30C018F6F788FC2B
:10E010000120307500203070F6F722FA00283FF416
:10E0200069AF307DBDE8F283E4670020FC66002024
:10E03000233E536C656570204144432025642025B0
:10E0400064000000233E505550000000233E6775D9
:10E050007031202564000000233E67757032202552
:10E0600064000000F8B507460020ADF80000FCF79A
:10E0700061FB0546DFF8304D012060743878A5F863
:10E080008A0005F28A0678787080B5F88A00002840
:10E0900002D07088002808D10FF29400F4F783F9B9
:10E0A0007820A5F88A000020708089208DF8000073
:10E0B00000AF70887870022300AA72210720F4F75D
:10E0C000E8F900280DD08B208DF80000B5F88A0003
:10E0D0007870022300AA72210720F4F7DAF90028E9
:10E0E00001D10020F2BD7288B5F88A100FF2480005
:10E0F000F4F759F9B5F88A007188401AE083B5F849
:10E100008A108900A18389B2FF2901DBFE21A18346
:10E1100080B28100652902DB6420E08301E0800099
:10E12000E083A08BE18B401AE0830120F2BD000068
:10E13000233E5054483D3000233E5448534554201C
:10E14000256420256400000080B50FF21801072027
:10E15000F7F70EFE0FF230010A20BDE80440F7F792
:10E1600007BE0000C9D7000819D80008B1D80008B8
:10E1700025D90008000000007DDE000865E00008E9
:10E180000000000000000000C9D7000819D80008EE
:10E19000B1D8000825D900080000000029D90008DE
:10E1A00065E00008000000000000000010B582B02B
:10E1B0000FF25400F4F7F7F80020ADF80000FFF775
:10E1C00099F8002803D10FF24800F4F7ECF8002486
:10E1D00000E0641C0B2C12D2DFF8840D2118097B9F
:10E1E0008DF80010205C8DF80100022300AA722136
:10E1F0000620F4F74EF90028EBD1002016BDF5F704
:10E2000063FB012016BD0000233E4745500000007F
:10E21000233E47504641494C0000000038B50FF2FC
:10E220009C00F4F7C0F80020ADF8000080208DF8C5
:10E23000000000AC03206070022300AA72210620B7
:10E24000F4F727F9002801D1002032BD8C208DF889
:10E25000000000206070DFF8505BA870022300AA65
:10E2600072210620F4F715F9002801D1002032BDF3
:10E27000A3208DF80000DFF8E80CC078607002235E
:10E2800000AA72210620F4F704F9002801D1002029
:10E2900032BD0120A872FFF74BFA01210820FFF7D9
:10E2A00053F8002801D1002032BD012032BD00000A
:10E2B0007F2B0120802B0120812B0120233E47450D
:10E2C0004F00000010B582B00FF26800F4F76BF851
:10E2D0000020ADF8000080208DF8000000AC032085
:10E2E0006070022300AA72210620F4F7D2F80028F9
:10E2F00001D1002016BDDFF86C0C002181720820CE
:10E30000FFF722F8002801D1002016BD9F208DF8CC
:10E31000000000206070022300AA72210620F4F79A
:10E32000B8F8002801D1002016BD012016BD00005C
:10E33000822B0120233E4745430000000120704707
:10E3400030B58DB0DFF8605AA879002814D008F0F5
:10E35000C1FE002810D0DFF80045201D0FC808F0CE
:10E36000B5FF08F0C0FE002832D00020A8710120BF
:10E3700060752075A0752BE0A879002828D1DFF8FA
:10E38000D844214684B068461822F4F761FB0FBCDC
:10E3900009F04AFB00A809F07AFBDFF8405528464F
:10E3A00000A93422F4F754FB05F11C00417D2175CE
:10E3B000817D6175007D002801D0FFF7B9F9287FC4
:10E3C000002805D034222946DFF81C0DF6F7A8FAFC
:10E3D00001200DB030BD00004428012010B584B0EC
:10E3E000044602A8002101600846ADF8040001209F
:10E3F000009001AB932272210620F4F7A4F80028C4
:10E4000000F088809DF8040010F0040004D1DFF8CB
:10E410009819497800297DD0002806D0DFF88809AE
:10E420004178002901D101218173012000900DF173
:10E430000503AE2272210620F4F785F8002869D082
:10E440009DF80500002817D00420009002ABFC22A4
:10E4500072210620F4F777F800285BD0DFF8F80384
:10E460009DF80810416002A94A7882608A78C260EB
:10E47000C9780161FFF764FFDFF86C1C0A78DFF8E8
:10E4800028094378002B227007D000226270A27006
:10E49000E27022716271A2710BE04A6962708A694E
:10E4A000A2704A68E2708A682271CA6862710A6959
:10E4B000A2710A6AE2714A6A22728A6A6272CA6A3E
:10E4C000A2724A7FE272DFF8242C12782273DFF8FE
:10E4D000202C12786273DFF81C2C1278A273DFF8FC
:10E4E000182C1278E273DFF8142C12782274DFF8FB
:10E4F000102C12786274DFF80C2C1278A274C27B94
:10E50000E274002202700878042801D110460870D5
:10E51000012000E0002004B010BDDFF8480AC07CF4
:10E52000704700008C25012080B5052802D10846DF
:10E5300000F002F8012002BD80B5017841F04103EE
:10E54000DFF8C41BCB70027801780FF6DC30F3F7EC
:10E550002AFF012002BD0000F467002070B584B0DE
:10E5600004460020019002A8002101600E460FF62B
:10E57000CC30F3F718FF01210820FEF7E5FEA020BC
:10E580008DF8040001AD30466870022301AA7221A3
:10E590000620F3F77EFF002801D13046C5E0A12018
:10E5A0008DF80400FF206870022301AA7221062062
:10E5B000F3F76FFF002801D13046B6E0AB208DF8AD
:10E5C000040001206870022301AA72210620F3F7DB
:10E5D00060FF002801D13046A7E0012000900DF136
:10E5E0000603802272210620F3F7ADFF002801D137
:10E5F00030469AE080208DF804009DF8060040F037
:10E6000045006870022301AA72210620F3F741FF3A
:10E61000002801D1304688E0A3208DF80400DFF8FF
:10E620004009C0786870022301AA72210620F3F71E
:10E6300030FF002801D1304677E0012000900DF135
:10E640000703AF2272210620F3F77DFF002801D1D6
:10E6500000206AE09DF80700C0070BD50420009059
:10E6600002ABFC2272210620F3F76DFF00280CD1CB
:10E6700000205AE03046461CB0F57A7FDDDB0FF60D
:10E68000C420F3F790FE00204FE09DF808002070B2
:10E6900002A8417861708178A170C078E070012093
:10E6A00000900DF10603802272210620F3F74BFF44
:10E6B000002801D1002038E080208DF80400DFF828
:10E6C000A408417A002905D09DF8060000F0BF009B
:10E6D00068700CE09DF8061001F0BB016970C07A0B
:10E6E000002804D19DF8060000F0BA0068700223EB
:10E6F00001AA72210620F3F7CCFE002801D10020E8
:10E7000013E0AB208DF8040000206870022301AAFA
:10E7100072210620F3F7BDFE002801D1002004E09D
:10E7200000210820FEF710FE012004B070BD00009B
:10E73000D8D00100E0F100080FF6A8210620F7F775
:10E7400017BB1CB50FF60820F3F72DFE00208DF83F
:10E750000400ADF80600044600E0641C052C13DA42
:10E76000DFF8A809215C8DF806102018007A8DF8D2
:10E77000070002230DF1060272210920F3F789FE3A
:10E780000028EAD1002016BD0120009001ABD6225E
:10E7900072210620F3F7D7FE002801D1002016BD14
:10E7A0009DF804100FF6B010F3F7FDFDDFF8B40785
:10E7B0009DF80410C9098176012016BD30B583B0DB
:10E7C000DFF8A047A07E002804D00FF69C10F3F7D6
:10E7D000EAFD03E00FF69810F3F7E5FD0020ADF831
:10E7E000040080208DF8040001AD0320687002232E
:10E7F00001AA72210920F3F74CFE002801D1002064
:10E800003EBD8F208DF804000B206870022301AA02
:10E8100072210920F3F73DFE002801D100203EBD02
:10E82000032020710120A075E07201460220FEF74E
:10E830008BFD002801D100203EBD012000900DF18C
:10E840000603E62272210920F3F77DFE002801D19C
:10E8500000203EBD01203EBDD42A012000B583B07A
:10E860000FF61410F3F79FFD0020ADF8060080208E
:10E870008DF8060003208DF8070002230DF1060233
:10E8800072210920F3F705FE002801D100200EBDFA
:10E890000120009001AB8F2272210920F3F753FE73
:10E8A000002801D100200EBDDFF8B8060021C1729A
:10E8B0000220FEF749FD002801D100200EBD0120F5
:10E8C000009001ABE62272210920F3F73CFE0028FC
:10E8D00001D100200EBD01200EBD0000A82701209F
:10E8E000012070472DE9F04184B004460020ADF8C6
:10E8F00004000290DFF89803456A002085F85E0066
:10E90000DFF86066B07D012803D0707D002840F0FC
:10E9100090800220009001AB942272210920F3F72D
:10E9200012FE00282DD09DF80400A07101AF787868
:10E93000E0710220009001AB962272210920F3F7CA
:10E9400002FE00281DD09DF80400207078786070C9
:10E950000220009001AB982272210920F3F7F3FD09
:10E9600000280ED09DF80400A0707878E070022096
:10E97000009001AB9A2272210920F3F7E4FD0028F0
:10E9800001D1002097E09DF8040020717878607133
:10E99000F0782072307960726078217841EA002046
:10E9A000E178A27842EA01216279237943EA0222DE
:10E9B000E379A77947EA032302AF009700F0CCF888
:10E9C00000281BD1B07D012834D10020B075DFF8BC
:10E9D00040075B2101700021417085218170002179
:10E9E000C170AE210171002141717021817101213D
:10E9F000C171EE210172002141721BE00020B0754F
:10EA0000DFF80C072178017061784170A17881707E
:10EA1000E178C1702179017161794171A1798171C8
:10EA2000E179C171217A0172617A41720298706252
:10EA300038E037D0DFF8D80601782170417861706E
:10EA40008178A170C178E17001792171417961719A
:10EA50008179A171C179E171017A2172407A607284
:10EA6000002070756078217841EA0020E178A27872
:10EA700042EA01216279237943EA0222E379A77904
:10EA800047EA0323F77894F808C086F803C096F89D
:10EA90000480647A347102AC009400F05DF8F77081
:10EAA00086F80480029840F68451884202D1012001
:10EAB00085F85E00012004B0BDE8F0811CB5044675
:10EAC0000020ADF806008DF804000120009001AB95
:10EAD0008F2272210920F3F736FD002801D1002092
:10EAE00016BD9DF8040000F0FC008DF80400012C18
:10EAF0000AD0042C04D0102C1FD0402C22D026E0A9
:10EB000040F001008DF804008F208DF806009DF87C
:10EB100004008DF80700DFF84C449DF8040000F075
:10EB20000300207102230DF1060272210920F3F780
:10EB3000B0FC00280DD1002016BD40F002008DF879
:10EB40000400E1E740F003008DF80400DCE700205A
:10EB500016BD0120607316BD2DE9F0419C46144698
:10EB60000D460646A8192018A0EB0C00401C4710C3
:10EB70003FB2002F00D50027DFF8E81308790FF225
:10EB80006062805CC978C1F5807110FB01F240F6CB
:10EB9000DC2E0EFB02F88902B1F5803F01D34FF65F
:10EBA000FF71C9000A22B1FBF2F110282DD18B426E
:10EBB0002BD30120FFF782FF002840D1E91B0698E4
:10EBC000B74206DA0268F31B4FF4B47606FB032261
:10EBD0000260AF4205DA02684FF47A7303FB012149
:10EBE0000160A74201DA016801600168002901D5CE
:10EBF0000021016040F2A641B8FBF1F10268B2FBCE
:10EC0000F1F101600120BDE8F081102808D1BCF1CC
:10EC1000640F05DA4020FFF751FF00280FD1CDE740
:10EC2000402802D164398B4204D20128C6D1BCF1FC
:10EC3000640FC3DA1020FFF741FF0028BED0002088
:10EC4000E1E70FF2C4510920F7F792B8C54988747B
:10EC50000120704710B5DFF8BC4420202070002050
:10EC600060700A20A0700020E0700A20207100204F
:10EC700060713220A0710020E07207222146DFF887
:10EC80009804F5F74DFE00206072012010BD0000D1
:10EC90000840002000B583B000A800210A4606C045
:10ECA0000722DFF870140DF10100F5F739FEA020FE
:10ECB0008DF80000082300AA72210720F3F7E9FB72
:10ECC000002801D100200EBD01200EBD00B583B08B
:10ECD00000208DF80400DFF83C04417B012903D1BA
:10ECE00000F0B0F901200EBD418AFF290CD00029A7
:10ECF0000DD0C27A521CC272491E4182417AD2B2F0
:10ED0000914201D20021C17200F015F805E0818A1C
:10ED100041820021C17200F00EF80120009001AB89
:10ED2000E32272210720F3F70EFC002801D1002016
:10ED30000EBD01200EBD38B50020ADF80000DFF893
:10ED4000D443608A002801D1A07A60720722E07A59
:10ED5000C0EBC000DFF8C01341182046F5F7E0FD16
:10ED6000FFF798FF80208DF8000000AD81206870CB
:10ED7000022300AA72210720F3F78BFB002801D1A0
:10ED8000002032BDA7208DF80000208A6870022381
:10ED900000AA72210720F3F77CFB002801D1002094
:10EDA00032BD012032BD0000FC66002030B585B0C8
:10EDB000044600208DF80C00ADF80E00607902903A
:10EDC00020790190E0780090A378627821780FF2A2
:10EDD000B030F3F7E8FA0120009003AB80227221F3
:10EDE0000720F3F7B0FB002801D1002061E0C94DF6
:10EDF0009DF80C0028720120009003AB8F22722135
:10EE00000720F3F7A0FB002801D1002051E09DF876
:10EE10000C00A8730120009003AB90227221072000
:10EE2000F3F791FB002801D1002042E09DF80C008F
:10EE3000E87300F0A6F88F208DF80E000DF10E0596
:10EE40000B20687002230DF10E0272210720F3F7E8
:10EE500020FB002801D100202BE090208DF80E002F
:10EE60000120687002230DF10E0272210720F3F7D2
:10EE700010FB002801D100201BE0A84D8122FF21BA
:10EE80002846F3F7EBF980222146681CF5F748FD88
:10EE90000020287081232A4672210720F3F7F9FA0F
:10EEA000002805D10FF2F020F3F77DFA002000E0F2
:10EEB000012005B030BD80B501780F2904DA954AEC
:10EEC000527A521C8A4205DA0FF2D820F3F76BFA15
:10EED000002002BD4278202A01DB2022427000225D
:10EEE000C2704271C1EBC1018B4A20238B54891837
:10EEF00000224A704278002A01D1002201E052002B
:10EF0000521E8A7182788A70C278CA7002790A7138
:10EF100040794871012002BD7E48417A491C417206
:10EF200081720120704738B504467A4D6C82FFF734
:10EF300091FE002C00D0AC8221460FF27820F3F72E
:10EF400032FA012032BD7349487301207047744979
:10EF50000870012070477248007870470000000078
:10EF60007C670020FC66002080B56A4908730A7B34
:10EF700052000A8201460FF24C20F3F714FA0120E6
:10EF800002BD00B583B00020ADF806008DF8040086
:10EF900080208DF8060001208DF8070002230DF176
:10EFA000060272210720F3F774FA002801D100202D
:10EFB0000EBD102000905B4BA02272210720F3F7BA
:10EFC000C2FA002801D100200EBD0120009001AB43
:10EFD000802272210720F3F7B6FA002801D1002021
:10EFE0000EBD01200EBD00B587B00020ADF80000B9
:10EFF00001A81421F5F7D2FB80208DF80000012034
:10F000008DF80100022300AA72210720F3F741FACC
:10F01000002801D1002013E0102242490DF1050023
:10F02000F5F77EFCA0208DF80400112301AA7221BF
:10F030000720F3F72EFA002801D1002000E001207C
:10F0400007B000BD30B583B00020ADF804008DF8E6
:10F050000600304C217A0FF27C10F3F7A4F900205F
:10F06000FFF7F4FD002060736072FFF7BCFF8F2094
:10F070008DF8040001ADA07B6870022301AA722103
:10F080000720F3F706FA002801D100203EBD9020AA
:10F090008DF80400E07B6870022301AA722107202A
:10F0A000F3F7F7F9002801D100203EBD80208DF84C
:10F0B0000400207A6870022301AA72210720F3F766
:10F0C000E8F9002801D100203EBD012000900DF19B
:10F0D0000603E32272210720F3F735FA002801D155
:10F0E00000203EBD01203EBD44280120F82B012018
:10F0F0007F2B0120802B0120812B0120822B0120DE
:10F10000F92B0120FA2B01207C67002004680020E5
:10F11000DC2C0120642B0120241C0120DC160120A2
:10F12000ED2E01204C2C0120233E47452043552045
:10F13000257820257820257800000000233E4753BD
:10F14000454C4600233E47535445525200000000B0
:10F15000233E4C4947500000233E4C434849502031
:10F160003078257800000000233E3E4C49474F0090
:10F17000233E4C49474F0000233E4C494743000083
:10F180004D424420256420256420256420256420E8
:10F1900025642025640000004D6F6265616D205775
:10F1A000460000004D6F6265616D20486F7020461B
:10F1B00061696C004D4220486F70436F756E74201A
:10F1C000256400004D6F6265616D204C656E3D25C4
:10F1D000640000004D4220436C6F7365202564007D
:10F1E00001041040ADE100081DE20008C5E200087E
:10F1F0003DE30008000000001BE5000800000000DF
:10F200005DE5000829E5000843E70008BDE70008C0
:10F210005DE80008E1E8000800000000E5E80008FB
:10F220000000000000000000000000007CB5002489
:10F230002046ADF80400F3F734F8054620208DF899
:10F24000040001AE20467070022301AABA210520F5
:10F25000F3F71FF9002801D1204676BD0121284689
:10F26000F3F70CFA641C0120009001AB2122BA21B3
:10F270000520F3F768F9002801D1002076BDA4B27B
:10F28000B4F5FA7F05DD0FF21C20F3F78CF80020AF
:10F2900076BD9DF804000006E0D420208DF804001F
:10F2A00002207070034601AABA210520F3F7F1F895
:10F2B000002801D1002076BD012076BD1CB5044692
:10F2C0000020ADF804000120009001AB0F22BA210C
:10F2D0000520F3F738F9002801D1002016BD9DF86C
:10F2E0000400BD2834D100F035F8002801D10020F9
:10F2F00016BD032001E0401E40B2002807D40FF2E3
:10F30000BC1151F830108C4201D20028F3D12020DA
:10F310008DF8040001ACA4206070022301AABA2178
:10F320000520F3F7B6F8002801D1002016BD102003
:10F330008DF804007F206070022301AABA21052005
:10F34000F3F7A7F8002801D1002016BD012016BD53
:10F35000002016BD80B50020ADF8000020208DF8FB
:10F36000000000208DF80100022300AABA21052028
:10F37000F3F78FF8002805D10FF23010F3F713F8E8
:10F38000002002BD012002BD80B58F20FFF796FF4F
:10F39000002801D1002002BD012002BD80B5FFF789
:10F3A00045FF002805D10FF20C10F2F7FCFF0020FA
:10F3B00002BD012002BD80B5FFF7E6FF002801D1A4
:10F3C000002002BD012002BD80B5FFF7C3FF002869
:10F3D00001D1002002BD012002BD012070470120A3
:10F3E00070471FB5044601A800210A460B460EC00F
:10F3F0000120009001AB0F22BA210520F3F7A3F8FA
:10F40000002821D09DF80400BD281DD105200090C2
:10F4100001ABA822BA21F3F796F8002801D1002009
:10F4200013E09DF80400207001A841786170817894
:10F43000A1700021E170C178217100796071E01C38
:10F4400000F006F8012000E0002004B010BD00002C
:10F450004178007840EA01204FF4F07190FBF1F020
:10F4600000EE100AB8EEC00ADFED070A30EE200AFF
:10F47000BDEEC00A10EE100A80B204490870000AFE
:10F48000487001207047000000002A42E82E012049
:10F4900001207047012070470FF240010520F6F768
:10F4A00067BC000042522D524600000042522D43DC
:10F4B0004600000042522D50460000002800000087
:10F4C0007000000050000000600000008F0000008D
:10F4D00050000000E8030000100000009DF3000849
:10F4E000B7F30008C9F30008DBF30008DFF30008F6
:10F4F000E3F300080000000091F4000895F4000810
:10F5000000207047012070470120704738B504463D
:10F510000D46F2F7C6FE0521F3F7B0F800201049BA
:10F5200004E00A680255521C0A60401CA842F8DB3D
:10F53000012032BD01207047012070470948026850
:10F540000A704A70511C01600120704706490A6820
:10F5500002704270501C08600120704700000000DB
:10F560004C680020782E01207C2E01200FF23401FF
:10F570000820F6F7FDBB10B50FF228042146122033
:10F58000F6F7F6FB21461320F6F7F2FB214614208E
:10F59000BDE81040F6F7ECBB0FF208011520F6F7B6
:10F5A000E7BB000001F5000805F5000809F50008B3
:10F5B00009F5000839F500080DF5000835F50008D3
:10F5C0004DF500083DF5000810B50024F2F769FE7E
:10F5D000007CC00700D50124204610BD00B589B0CD
:10F5E00000A82421F5F7DAF80020ADF822000A205F
:10F5F0008DF8080000208DF809008DF80A008DF8BC
:10F6000000001F20019000A8F8F76EFD012009B04E
:10F6100000BD00B589B000A82421F5F7BFF800208F
:10F62000ADF822000A208DF8080000208DF80900AE
:10F630008DF80A0001208DF800001F20019000A81D
:10F64000F8F752FD012009B000BD00B589B000A84F
:10F650002421F5F7A3F80020ADF822000A208DF848
:10F66000080000208DF809008DF80A0001208DF8AF
:10F6700000001F20019000A8F8F736FD012009B016
:10F6800000BD0120704710B50024F2F70AFE007C8F
:10F69000C00700D50124204610BD00B589B000A8E0
:10F6A0002421F5F77BF80020ADF822000A208DF820
:10F6B000080000208DF809008DF80A008DF8000080
:10F6C0002020019000A8F8F70FFD012009B000BD2F
:10F6D00000B589B000A82421F5F760F80020ADF846
:10F6E00022000A208DF8080000208DF809008DF80E
:10F6F0000A0001208DF800002020019000A8F8F7F2
:10F70000F3FC012009B000BD00B589B000A8242198
:10F71000F5F744F80020ADF822000A208DF8080023
:10F7200000208DF809008DF80A0001208DF80000F6
:10F730002020019000A8F8F7D7FC012009B000BDF7
:10F740000120704710B50024F2F7ABFD007C800764
:10F7500000D50124204610BD00B589B000A82421A1
:10F76000F5F71CF80020ADF822000A208DF80800FB
:10F7700000208DF809008DF80A008DF80000212086
:10F78000019000A8F8F7B0FC012009B000BD00B559
:10F7900089B000A82421F5F701F80020ADF8220077
:10F7A0000A208DF8080000208DF809008DF80A0065
:10F7B00001208DF800002120019000A8F8F794FCAA
:10F7C000012009B000BD00B589B000A82421F4F7DC
:10F7D000E5FF0020ADF822000A208DF80800002087
:10F7E0008DF809008DF80A0001208DF80000212015
:10F7F000019000A8F8F778FC012009B000BD0120B5
:10F80000704710B50024F2F74CFD007C00F00300B7
:10F81000032800D10124204610BD00B589B000A8FE
:10F820002421F4F7BBFFDFF86C03017841F00201FB
:10F8300001700020ADF822000A208DF80800012098
:10F840008DF809008DF80A1000208DF800002220A4
:10F85000019000A8F8F748FC012009B000BD00B5F0
:10F8600089B000A82421F4F799FFDFF8281308785D
:10F8700010F0FD00087014D10020ADF822000A201D
:10F880008DF8080001208DF8090000208DF80A008D
:10F8900001208DF800002220019000A8F8F724FC38
:10F8A00002E040B208F08EFE012009B000BD012048
:10F8B00070470120704710B50024F2F7F2FC007C7D
:10F8C00000F00700072800D10124204610BD00B534
:10F8D00089B000A82421F4F761FFAE49087840F010
:10F8E00001000870032805D140B208F06BFE08F053
:10F8F00085FE12E00021ADF822100A218DF80810D3
:10F9000000218DF809108DF80A0008468DF80000D6
:10F910002220019000A8F8F7E7FB012009B000BD04
:10F9200000B589B000A82421F4F738FF9949087878
:10F9300010F0FE00087013D10020ADF822000A205C
:10F940008DF8080000208DF809008DF80A000120CC
:10F950008DF800002220019000A8F8F7C5FB04E014
:10F9600040B208F02FFE08F04EFE012009B000BDA5
:10F97000012070470120704710B50024F2F791FC78
:10F98000007CC00700D50124204610BD30B58BB0E7
:10F9900001A82421F4F702FF002000907E48446C67
:10F9A0000020ADF826000A208DF80C0000208DF80C
:10F9B0000D008DF80E008DF804002320029001A8A0
:10F9C000F8F792FB0020009004F10C056A7D00A975
:10F9D000E868E368C018F4F7A3FF0120A8740020CA
:10F9E00008F0C7FE02F06DFB01200BB030BD00B582
:10F9F00089B000A82421F4F7D1FE0020ADF8220040
:10FA00000A208DF8080000208DF809008DF80A0002
:10FA100001208DF800002320019000A8F8F764FB76
:10FA2000012009B000BD00B589B000A82421F4F779
:10FA3000B5FE0020ADF822000A208DF80800002055
:10FA40008DF809008DF80A0001208DF800002320B0
:10FA5000019000A8F8F748FB012009B000BD012083
:10FA60007047000070B58AB004460E46F8F766FA93
:10FA70000546002000900422214600A8F4F750FF1C
:10FA800001A82421F4F78AFE009A31460FF2C01033
:10FA9000F2F789FC30460C3809284ED8DFE800F030
:10FAA000051118253C0C4D4D4D481420C5F8DC04BB
:10FAB000207001200AB070BD1420C5F87C052070AC
:10FAC000F7E705F2DC403C21816208462070F0E750
:10FAD00005F2DC4021783C2904D13C2121702178B9
:10FAE0000165E6E700990165E3E72A480078C10768
:10FAF00012D50021ADF826100A218DF80C10002136
:10FB00008DF80D108DF80E0001208DF804002220D4
:10FB1000029001A8F8F7E8FA0099304640B200F0E8
:10FB200012F80090206005F2DC4000998167C0E780
:10FB30001420C5F8BC062070BBE70FF22410F2F7C2
:10FB400032FC0020B6E710B4134AD36B126C114C90
:10FB50002478002C1AD00F2802D010280BD015E0E2
:10FB6000507A002812D0906B806800280ED488420A
:10FB70000DDD08460BE0587A002807D0986B8068A6
:10FB8000002803D4884202DD084600E0084610BC85
:10FB900070470000EE2E01200840002012B589B009
:10FBA00001460C3909292CD8DFE801F0051F212373
:10FBB000231D2B2B2B291F240020ADF822000190A0
:10FBC0000A208DF8080005208DF800000194042219
:10FBD00009A90DF10900F4F7A3FE00A8F8F784FACB
:10FBE00001200AB010BD2324E6E72024E4E7212405
:10FBF000E2E722240999FFF7A6FF0990DCE72B240E
:10FC0000DAE70FF26400F2F7CEFB0020E9E780B5F7
:10FC10000FF25C010C20F6F7ABF80FF2780111201F
:10FC2000F6F7A6F80FF290010D20F6F7A1F80FF203
:10FC3000AC010E20F6F79CF80FF2C4010F20F6F786
:10FC400097F80FF2E0011020BDE80440F6F790B8F5
:10FC50004D52322044523D25642C256400000000A2
:10FC60004D523220534446004D52322052434600FA
:10FC7000C9F50008DDF5000813F600084BF600088A
:10FC80000000000083F6000865FA0008000000008C
:10FC90000000000079F900088DF90008EFF900086C
:10FCA00027FA0008000000005FFA000865FA000863
:10FCB000000000000000000087F600089BF6000826
:10FCC000D1F6000809F700080000000041F700081D
:10FCD00065FA0008000000000000000045F7000879
:10FCE00059F700088FF70008C7F700080000000068
:10FCF000FFF7000865FA000800000000000000009F
:10FD000003F800081BF800085FF80008AFF80008C7
:10FD100000000000B3F8000865FA000800000000C9
:10FD200000000000B7F80008CFF8000821F900082B
:10FD300071F900080000000075F9000865FA000874
:10FD4000000000000000000080B5FAF7F3FCDFF8C7
:10FD500034180860012002BD80B5F4F7ABFCDFF871
:10FD60002818D1E90023801A02BDF8B50446A0691D
:10FD7000E1684518B5F90000B5F90270B5F90460FD
:10FD8000B4F9581094F90820012A2AD1B5EE000AD6
:10FD900000EE901AF8EEE00A60EE800AFDEEE00A4E
:10FDA00010EE901A411A2980B4F95A1000EE901AF8
:10FDB000F8EEE00A60EE800AFDEEE00A10EE901A1E
:10FDC000791A6980B4F95C1000EE901AF8EEE00A36
:10FDD00020EE800ABDEEC00A10EE101A711AA9803A
:10FDE00009E0411A2980B4F85A10791A6980B4F8E8
:10FDF0005C10711AA980B5F90010C913B1EBE03F8E
:10FE000013D0B4F95810C913B1EBE03F0DD00FF285
:10FE10009470F2F7C8FAB5F90000012802DBDFF8A8
:10FE20006C0701E047F6FF702880B5F90210C9138E
:10FE3000B1EBE73F13D0B4F95A10C913B1EBE73F68
:10FE40000DD00FF26C70F2F7AEFAB5F9020001288E
:10FE500002DBDFF8380701E047F6FF706880B5F98C
:10FE60000410C913B1EBE63F13D0B4F95C10C91309
:10FE7000B1EBE63F0DD00FF24470F2F794FAB5F90A
:10FE80000400012802DBDFF8040701E047F6FF70F9
:10FE9000A88094F90800002804D1002000E0401C4C
:10FEA0000328FCDBF1BD0000FEB5044600A80021DC
:10FEB0000A460B460EC0A069E1684518174694F93A
:10FEC0000860052E80F09A80012E02D12046FFF7AF
:10FED0004CFF3046012802D9C01E40F08A80002E17
:10FEE00001D14FF6FF77DFF89C060068301890F8D4
:10FEF0008400401E06285ED8DFE800F004101D29AB
:10FF000036424F00B5F90200009000A8B5F9001084
:10FF1000791A4160B5F90410816056E0B5F9000026
:10FF2000381A009000A8B5F90210791A4160B5F9A5
:10FF30000410816049E0B5F90200381A009000A869
:10FF4000B5F900104160B5F9041081603DE0B5F9E4
:10FF50000000381A009000A8B5F902104160B5F908
:10FF60000410791A816030E0B5F90200009000A811
:10FF7000B5F900104160B5F90410791A816024E0E8
:10FF8000B5F90000009000A8B5F90210791A416097
:10FF9000B5F90410791A816017E0B5F90200381A32
:10FFA000009000A8B5F90010791A4160B5F9041065
:10FFB000791A816009E0B5F90000009000A8B5F950
:10FFC00002104160B5F904108160012E0AD10021B0
:10FFD00006E050F8212002F30F0240F82120491CCE
:10FFE0000329F6DB0098288000A8416869808068B2
:10FFF000A880002E02D12046FFF7B7FE0120FEBDEB
:020000021000EC
:1000000070B52DED028B82B08169C2688A1890F9B3
:10001000081008460A2800F29880DFE800F0062B56
:1000200073969665969696808E00B2F90240B2F964
:100030000450DFF8500500689FEDAC0AB2F90010DB
:1000400000EE901AF8EEE00A60EE800AC0ED000AB9
:1000500000EE904AF8EEE00A60EE800AC0ED010A78
:1000600000EE905AF8EEE00A20EE800A001D80EDC6
:10007000010A6EE0B2F90240B2F90450DFF804055B
:100080000068061D9FEDC08BB2F9000000EE100A5B
:10009000B8EEC00A10EE100AF8F74EF953EC182B20
:1000A000F2F7E2FDF8F770F9B06000EE104AB8EE32
:1000B000C00A10EE100AF8F73FF953EC182BF2F7CC
:1000C000D3FDF8F761F9F06000EE105AB8EEC00AFF
:1000D00010EE100AF8F730F953EC182BF2F7C4FDC4
:1000E000F8F752F9306134E0002000901068009079
:1000F0009DED000ABAEECA0ADFF88804006880EDB8
:100100000C0A26E0DFF87C0400681188A0F85A1079
:1001100000F25A00518841809188818019E0DFF80F
:100120006404006800F25A001188C180518801817E
:1001300091884181D18881810BE0DFF84804006813
:1001400092F9001080F8681003E00FF27C40F2F79B
:100150002AF9012002B0BDEC028B70BD70B50D46CE
:10016000DFF82C1451F820400026207F002801D110
:10017000304670BD607A002803D0206E80688047CA
:1001800006462846216EC96988470546002E02D0DA
:10019000206E40688047284670BD01207047F0B44B
:1001A000002A10D400F11004A57C066992FBF1F737
:1001B0006F43B74202DAA263E26304E096FBF5F212
:1001C0005143A163E163002B03D4990701D510309B
:1001D0000374F0BC7047002903D40021816441619D
:1001E00081617047042817D101F10C008A7A012A35
:1001F00009D0072242750B228275DFF89823CA6066
:100200000B21416070471522427519228275DFF873
:100210008823CA601921416070472DE9F243804666
:1002200014461A46C146B9F1160F46D24546DFF8C4
:10023000600350F825600227307F00283DD0084633
:10024000C82802D1B420009003E0422801D13C200C
:1002500000909DF92030002B06D4D80704D50099D2
:100260003046FFF79AFF3FE000993046FFF797FFCF
:10027000A9F10C00062805D24146C9B200A8326E89
:100280009269904731464046FFF7ACFF707A0028EC
:100290001BD1214649B23046726E12689047002841
:1002A0000DD0306E40688047002804D139464F1E7B
:1002B000C9B20029F5D1002801D1002014E021465F
:1002C00049B23046726E52689047707A401C707224
:1002D0000D2D08D0224652B200993046736E1B692C
:1002E000984700F0B7F80120BDE8F28360F61C3AA9
:1002F0002DE9F04106460C4615461946162E07D242
:10030000A34850F826704FF00208387F002801D12A
:10031000002036E0C82C01D1B42402E0422C00D1E8
:100320003C243846FFF757FF787A012818D1294630
:1003300049B238467A6E9268904700280AD0386EE3
:1003400080688047002805D14046A0F10108C0B26E
:100350000028F4D1294649B238467A6ED2689047CF
:10036000787A002801D0401E78720D2E08D02A46D7
:1003700052B2214638467B6E5B69984700F06AF8B6
:100380000120BDE8F081000089AD84FA0A74513F74
:100390002DE9F84304460D4616461A462746162F01
:1003A00026D27B4951F8208098F81C1000291FD0D4
:1003B000C82D01D1B42502E0422D00D13C250D28E5
:1003C00001D1012044E09DF92030002B07D4D8074B
:1003D00005D52946404601B0BDE8F043DDE606EB11
:1003E000460008EB8009D9F838008068002801D55C
:1003F00000202DE029464046FFF7D1FED9F838000D
:100400008068854217D0012D15DB0FF2C810F1F777
:10041000CAFF324652B2D9F8380081684046D8F84F
:1004200064305B699847324652B229464046D8F854
:1004300064301B699847A7F10C00062805D22946AD
:100440002046FFF7ABFB012002E000F003F801209B
:10045000BDE8F28370B56FF0004634464F4801683E
:1004600004E08A68A24200DA144609688142F8D1A1
:100470004B4D2878401C28706878F021084202D043
:100480009920F4F7C9F9F4F734FA6878401C6870D9
:10049000B44200D100243B4E3068C467D0F88020BD
:1004A00021468A4212D0002901D0002A0BD1C0F87F
:1004B00080100FF23010F1F776FF3068D0F880002E
:1004C000F1F74DFF02E0012008F09CF96878F02177
:1004D000084202D09920F4F79FF96878401E6870AE
:1004E000C0B2002801D1F4F7FEF9F5F75CF801205D
:1004F00070BD38B505462A4C2078401C20706078C5
:10050000F021084202D09920F4F786F9F4F7F1F9C6
:100510006078401C607029460FF2DC00F1F743FF61
:1005200018480068C0F880501C48016805E08A68D7
:10053000B2FBF5F26A43CA6009688142F7D160787C
:10054000F021084202D09920F4F766F96078401E45
:100550006070C0B2002801D1F4F7C5F9BDE83140A0
:10056000F5F721B80D490A6808E01369012B01DA93
:10057000D368136113691B1A136112688A42F4D19C
:10058000704700008C2E0120082E01200080FFFF04
:10059000084000208C500020882A0120784000204C
:1005A0002C67002058206973206F76657200000068
:1005B00059206973206F7665720000005A206973B4
:1005C000206F766572000000554353542825642936
:1005D0004E5300006368616E676520726174653216
:1005E00000000000675F707453682D3E6354696DAE
:1005F0006572203D202564006374696D6572203D3D
:100600002025640038B504000D0014480078401C13
:100610001249087012480078002802D0A120F4F78F
:10062000FBF8F4F77FFF607E662802D08220F4F7A3
:10063000F3F8F4F75EF905E03821200008F0E8F857
:10064000F4F757F9E06821698842F5D029002000C5
:1006500008F000F9F4F7A7FF31BD00BF2C670020B8
:10066000162F01204FF0FF31801E012812D9C01E25
:1006700004280FD9801F05280CD908380AD0801EFD
:10068000042807D9401F03D0401E102802D902E0D9
:10069000072100E001210846704780B5014600208F
:1006A000C91E18D0C91E16D0C91E14D0C91E0129D2
:1006B00011D90D3903290ED9091F05D0491E0AD0B9
:1006C000C91F032907D902BD1D210FF21000F1F740
:1006D0006AFE012002BD012002BD000050443A2004
:1006E0004C4C53202564000038B504464FF0FF35CC
:1006F000F7F724FC2B2C35D8DFE804F02F34332F08
:100700002F332F2F3333342F183316162F3434331F
:10071000342F2F2F182F332F332F2F1B1E22262A33
:100720002D33333333333133B4251BE04FF47A7533
:1007300018E0D0F8DC5415E000F2DC40856A11E0E6
:1007400000F2DC40056D0DE000F2DC40856F09E051
:10075000D0F87C5506E00A2504E03C2502E005259A
:1007600000E01425284632BD38B5DFF8004AF9F715
:10077000E1FFE06208F0D6F8F7F7E0FB2063002520
:1007800012E0DFF8EC190161DFF8E8194161DFF8E8
:10079000E8298261DFF8E429C261DFF8E429026216
:1007A0004162406A80476D1C2D2D80F21181216BC2
:1007B00005EB8500C00000224254401842704FF003
:1007C000FF32426000220272C2604272032D04D1E5
:1007D0007431DFF8B0298A62E3E7022D03D1DFF834
:1007E000A8294A67DDE7002DCBD0042D04D1743150
:1007F000DFF898290A65D4E7052D04D17431DFF8B4
:1008000090298A67CDE7062D04D1DFF88829C1F841
:100810001421C6E7072D05D101F58A71DFF8782983
:100820008A62BEE7082D05D101F58A71DFF86C29CF
:100830000A65B6E7092D05D101F58A71DFF860294F
:100840008A67AEE70A2D9CD00B2D9AD0012D98D047
:100850000C2D04D1DFF84C29C1F80422A1E70D2D9D
:1008600005D101F50171DFF840298A6299E70E2D63
:1008700005D101F50171DFF834290A6591E70F2DE3
:1008800005D101F50171DFF828298A6789E7102D64
:1008900004D1DFF82029C1F8A42282E7122D3FF409
:1008A00070AF142D3FF46DAF132D3FF46AAF162DCA
:1008B0003FF467AF2B2D3FF464AF152D04D1DFF863
:1008C000082AC1F86C236CE7172D05D101F55B717F
:1008D000DFF8F8290A6564E7182D05D101F55B7189
:1008E000DFF8EC298A675CE71A2D05D101F20C418B
:1008F000DFF8E0298A6254E71E2D05D101F2AC41F0
:10090000DFF8D4298A624CE7192D04D1DFF8CC290D
:10091000C1F80C2445E71F2D05D101F2AC41DFF8E9
:10092000C0290A653DE7202D05D101F2AC41DFF871
:10093000B4298A6735E7212D04D1DFF8AC29C1F845
:100940004C252EE7222D05D101F24C51DFF89C29D0
:100950008A6226E7232D05D101F24C51DFF8902958
:100960000A651EE71B2D05D101F20C41DFF8842931
:100970000A6516E71C2D05D101F20C41DFF8782934
:100980008A670EE71D2D04D1DFF87029C1F8AC2469
:1009900007E7262D04D1DFF86829C1F8142600E7FF
:1009A000272D05D101F21461DFF858298A62F8E693
:1009B000292D05D101F21461DFF84C298A67F0E690
:1009C0002A2D7FF4DEAEDFF84429C1F8B426E8E62C
:1009D000012032BD0CB42DE9FF47054688460124AD
:1009E00047462E461A2E48D006EB86004FEAC0082E
:1009F000DFF878970B2F20D1D9F8300008EB000AE8
:100A00009AF80100002818D02846FFF72BFE01288D
:100A100013DB2846FFF726FE9AF8011081420CDB13
:100A2000284600F086F90446D9F8300040440021F9
:100A300041700FF6E400F1F7B6FCD9F8300018F871
:100A40000010002947D108EB00014A78002A42D162
:100A5000002208F80020104648700CA983B06846B0
:100A60001822F1F7F5FF0EBC284600F07CF80228AA
:100A70002CD003282FD103242DE00B2F16D1FFF704
:100A8000F1FD012812DB2846FFF7ECFD06EB86019D
:100A9000DFF8D826126B02EBC1014978814205DBF1
:100AA0000FF67C00F1F77FFC022057E04046C0B211
:100AB00002F080F80CA983B068461822F1F7C8FF4D
:100AC0000EBC284600F04FF8022801D1022045E074
:100AD000032800D103240A2F0DD1DFF89096D9F80E
:100AE000300006EB86014FEAC10818F80010491CD7
:100AF00008F8001017E00B2F15D1DFF87096032EC1
:100B000007D1D9F8300090F87900002801D101F020
:100B1000B2FA06EB86004FEAC008D9F8300040442C
:100B20004178491C4170DFF84496D9F83000D9F873
:100B30002C1006EB86024FEAC208D1E91C23CDE94E
:100B40000223C96E009108EB00014B7818F80020D1
:100B500031460FF2D870F1F726FC204604B0BDE80C
:100B6000F0075DF80CFB0EB42DE9F04183B00546AB
:100B70000124C0B2FFF7B8FDDFF8F06505EB850191
:100B8000326B02EBC107786000203872F86009A967
:100B900084B068461822F1F75BFF0FBC3F69B84785
:100BA000022801D1022011E0032801D103240CE026
:100BB000D6F82C80D8E91C67204600212A4607F089
:100BC00055FF30433943C8E91C012046BDE8FE010A
:100BD0005DF810FB2DE9FF4704460D460126274628
:100BE00007EB87004FEAC008DFF88095D9F830009E
:100BF0001A2F57D008EB000A9AF80100022814DBDC
:100C00002046FFF72FFD01280FDB2046FFF72AFDC6
:100C10009AF80110814208DB2046FFF723FD8AF88D
:100C200001000FF21C70F1F7BEFBD9F8300018F884
:100C30000010002904D108EB00025278002A60D08D
:100C40002A460A2A09D1002903D0491E08F80010B3
:100C500017E0002108F8001013E00B2A11D108EB6F
:100C600000014A78002A02D0521E4A7001E0002298
:100C70004A70032F05D190F87900002801D101F0C6
:100C800009FAD9F8300018F80010002939D1404489
:100C90004078002835D1204600F04BF8032830D1A9
:100CA00003262EE018F80010002904D108EB0002FA
:100CB0005278002A25D02A460A2A09D1002903D0D1
:100CC000491E08F8001012E0002108F800100EE09C
:100CD0000B2A0CD108EB000A9AF80100002803D077
:100CE000401E8AF8010002E000208AF80100284630
:100CF000C0B201F05FFF204600F01BF8032800D1CE
:100D00000326D9F83000D9F82C10D1E91C23CDE9FD
:100D10000223C96E009108EB00014B7818F80020FF
:100D200039460FF22460F1F73EFB304604B0BDE8CF
:100D3000F0872DE9F0410746012607EB8700C50043
:100D4000DFF82844206B281840698047032800D129
:100D50000326384640B200F080F9032800D103266C
:100D6000206B295C002917D128184178002913D15C
:100D70004FF0FF31416000210172C160D4F82C8036
:100D8000D8E91C4501203A4607F070FE24EA00002D
:100D900025EA0101C8E91C013046BDE8F08138B5FB
:100DA000044604EB8400C000DFF8C053296B002226
:100DB00042544018114641702046FFF7BAFFE86AD6
:100DC000D0E91C2321460FF29450F1F7ECFA0120F0
:100DD00032BD2DE9F041B6B004460E46B6B2012050
:100DE0008DF86400DFF884531AA8E96A6C22F1F7E1
:100DF0002FFE17951AA984B068466C22F1F728FED9
:100E00000FBC00F0D9F900270BE0032803D1189795
:100E100003208DF86400286B4044002101727F1C80
:100E20007FB22D2F2ADAEA6AD2E91C013A4600F095
:100E3000CBFA00F0010011F0000101D10028EED042
:100E400007EB87004FEAC008286B4044416800293F
:100E5000E5D4027A521C0272D2B2724389B28A423B
:100E6000DDDB806980470228CFD1189702208DF8FA
:100E70006400DDE91801C4E9000103E0DDE91801BF
:100E8000C4E9000136B0BDE8F08100210A3842F221
:100E90000772904200D20121084670472DE9F043C5
:100EA00083B0044600200190042204F1090101A846
:100EB000F3F736FD6168DFF8B462376B282505FB70
:100EC00001704068019A904204D10FF2A040F1F7FE
:100ED0006AFA68E01046FFF7D8FF002809D1616878
:100EE000019B05FB017042680FF28C40F1F75BFA41
:100EF00059E0DFF81C743868D0F8008025E090F9DC
:100F000008906068316B05FB0010C06820FA09F09A
:100F1000C00717D54FF0FF3000900346012201991A
:100F20004846FFF77AF940B200280BD16168019872
:100F30000090306B05FB010043684A460FF24C40BD
:100F4000F1F731FA4046D0F80080B842D7D138687E
:100F5000D0F800801FE090F90890C86820FA09F0E6
:100F6000C00715D54FF0FF33012249684846FFF707
:100F7000BFF940B200280BD1616801980090306B36
:100F800005FB010043684A460FF21840F1F70BFADF
:100F90004046D0F800806168326B05FB0121B84201
:100FA000D9D101984860BDE8F7832DE9F84381461F
:100FB000002425466D4F21E005EB8500C600386B07
:100FC00006EB0008002088F80900FA6AD2E91C0143
:100FD0002A4600F0F9F900F0010011F0000101D1FA
:100FE00000280AD04846D8F81C108847002804D0AA
:100FF000386B3018012141720C466D1C2D2DDBDB46
:101000002046BDE8F2835948C16AD1E91C23002B70
:1010100001D1002A0DD0002107E002EB8203026B10
:1010200002EBC30200235372491C49B20A462D2A1F
:10103000F3DB704700B502464C48C36AD3E91C0194
:1010400000F0C2F900F0010011F0000101D1002808
:1010500001D0012000BD084600BD2DE9F0478146C2
:10106000012409EB8900C500404E306B2818C06888
:10107000002829D0DFF898723868D0F8008003E0A3
:1010800003244046D0F80080B8421DD090F908A053
:10109000306B2818C168012202FA0AF2114021FAC5
:1010A0000AF149B20129ECD14FF0FF330122416826
:1010B0005046FFF71DF90028E2D0524649460FF28C
:1010C000FC20F1F770F9DCE72046BDE8F08710B5A9
:1010D0008AB004460020ADF8220001900A208DF865
:1010E000080000208DF809008DF80A00ADF82200F4
:1010F000600719D50520FFF79DFF002807D00420C1
:101100008DF800000520019000A8F6F7EDFF022001
:10111000FFF790FF002807D004208DF80000022080
:10112000019000A8F6F7E0FFE0060CD50820FFF7D5
:1011300081FF002807D003208DF8000008200190CF
:1011400000A8F6F7D1FF0AB010BD02460020092A18
:1011500000D0704780B5012902D107F049FD012078
:1011600002BD02492C22F1F773BC0000782801204F
:10117000538200084F8200085B8200085F820008EB
:10118000638200083D1A01089D4A0108E91301081D
:10119000614801082B0B0308E51C03089946010868
:1011A0003F8B0108FD160108D9090308C9FE020892
:1011B000151403089B1A03080FB41B9800990160CB
:1011C00001994160029981600399C16004990161AC
:1011D00005994161BDF85A100183BDF85C10418347
:1011E000BDF85E1081830C990162139941621499D4
:1011F000816204B0704700004168122903D1C17AAE
:10120000002000F0FABF132903D1017B012000F078
:10121000F4BF142903D1417B022000F0EEBF152951
:1012200002D1C07A00F0FABF172945D1817A1B2973
:1012300006D01C2930D01D290FD0262926D0704772
:10124000C17B012903D1B0F80B0003F043B9022997
:1012500032D1B0F80D0003F03BB9017D012903D173
:10126000B0F80B0007F0A8BF022903D1B0F80D00B9
:1012700007F096BF042903D1B0F8170007F0A8BF04
:10128000032919D1B0F8150007F0AEBFC17B0129C1
:1012900012D1807B08F0E9B8817B012902D1C07AA4
:1012A00008F0EFBA022902D1007B08F0F4BA052950
:1012B00002D1407B08F0CFBA7047164908607047EA
:1012C0001448006870470000FD1D03082D20030826
:1012D000F1120308B137010833070308ED160308BC
:1012E00033AD0108CF1B03088B1103086785010884
:1012F0003387010875440108D19601083F91010820
:10130000B193010813E80208211F0308ADE90208A0
:1013100074490020902E0120414C204558000000C7
:10132000414C2045582D415400000000414C25649B
:1013300020256420256420256420256C6C75000020
:10134000524C204558000000524C25642025642052
:10135000256420256420256C6C7500005445524D91
:1013600020256420256C6C75000000004558204C39
:101370004D435231202564004558204C4D43523294
:101380002025642025642025640000004558204C59
:101390004D43523320256420256420256420256494
:1013A000000000004558204C4D4352342025642055
:1013B000256420256420256400000000534D52411F
:1013C0002025642025640000D2B2203A22BF21FAF1
:1013D00002F0002170472032D141D0404840914076
:1013E000D14048407047000038B5F6F7A7FD0446E5
:1013F000104DF9F79FF9286005F0C2F805F0C5F81F
:10140000686005F0FDF90C48C4F8B00004F1B000C4
:101410000A4941600A4981600A49C1600A4901617B
:10142000012032BD0349496889680847014840687E
:1014300000680047302E0120538200084F820008C8
:101440005B8200085F820008638200082DE9F04794
:1014500086B0044601A81421F3F7A0F9F0F721FFA4
:1014600005464FF00208002601E0761C76B20A2EEF
:1014700080F29E80022EF8D0032EF6D0062EF4D0F5
:10148000524850F82670787A002806D107F10C00EF
:10149000406D406880470028E7D008F8046008F1F4
:1014A00001084FFA88F8304609284FD8DFE800F0E5
:1014B000050A4E4E10204E154E49C8212846F1F718
:1014C000DDF843E04FF448712846F1F7D7F83DE0E6
:1014D00032212846F1F7D2F838E007208DF80400D1
:1014E000FF208DF8050032212846F1F7C7F82DE0DE
:1014F0003C212846F1F7C2F84FF0000A07F10C0929
:10150000BAF1030F22DA0020D9F85410096988478C
:1015100014212846F1F7B2F80120D9F854100969CE
:10152000884714212846F1F7A9F8BAF1020F05DA25
:10153000062101A8D9F85420526990470AF1010AFE
:10154000DEE74FF416712846F1F798F807F10C0919
:1015500099F8151001A8D9F854205269904700282D
:1015600019D0D9F80C00F96800EB010A99F8152098
:1015700001A95046F3F7D4F93846FEF795FC99F8DF
:101580001520514608EB0400F3F7CAF999F9150044
:1015900080444FFA88F8787A00287FF466AFD9F84B
:1015A00054008068804700287FF45FAF002009E086
:1015B000A8F10200ADF80000022200A92046F3F7CE
:1015C000AFF9002006B0BDE8F08700000840002019
:1015D00038B505000C0094F84C00642802D0802037
:1015E000F3F71AF9F3F776FFF3F783F96069284305
:1015F0006061207C10F0F800082806D1A0696169BC
:10160000084202D02000F4F70AF807484078F02199
:10161000084202D09920F3F7FFF8034840780028E9
:1016200001D1F3F760F931BD2C6700200FB480B50C
:10163000BDF80B0064494880022802DB801E088048
:1016400001E0002008800C229DF90A100020F6F726
:1016500077FC032801D1022000E0012002BC5DF8E4
:1016600014FB59480121418000210180012070476D
:10167000564908707047000030B58DB002A8F6F7E3
:10168000BEFC514C2088401C2080618880B288427A
:1016900031D300202080054627E06068D0F8EC01B7
:1016A000E840C00720D5284607F08EF900281BD453
:1016B00000EB80009FED430ADDED0B0A60EE800A2F
:1016C000FDEEE00A10EE901A00AA8152DDED0C0A40
:1016D00020EE800ABDEEC00A10EE101A821851806A
:1016E00000A94018012101716D1C172DD5DBDDE922
:1016F000000107F072F901200DB030BD80B5F6F79A
:101700001DFC314948603249C0F8F01100F5F8700D
:1017100030494160304981600FF20D01C1600FF224
:1017200025010161012002BD10B50024274890F970
:101730000000002804D107F070F9002800D001242F
:10174000204610BDF8B504460D4640F22116287813
:1017500016FB004001210170287816FB0040417003
:10176000287816FB00400C218170287816FB004079
:10177000164991F90010002902D00221C17001E040
:101780000121C170287816FB0040012101712878E1
:1017900016FB0040C180287816FB0047002007F0A8
:1017A000DDF83881287816FB0044002007F0DBF8CC
:1017B00060812878401C28700C20BDE8F24007F0BA
:1017C000EBB800000000C84244680020F72E01205A
:1017D0002D16010863160108791601080FB410B51B
:1017E000032200210846F6F7ABFB022801D10220B4
:1017F0001CE00FF24000F0F7D6FDDFF8444C00206B
:101800006073608260629DF80C209DF80B109DF85B
:101810000A0008F0C9FD58220021DFF8B80CF0F7E3
:101820001DFD00202074A0732063012010BC5DF812
:1018300014FB000050443A20537461727450656484
:101840006F2D30323235000080B503220021012097
:10185000F6F776FB032801D1032002BD012002BD6B
:1018600030B58BB000A8F6F7CAFB05210320F6F7C8
:1018700029FC002802D1DFF8600C0890DFF8C04B8B
:10188000E069C56F08F026FD207294F9080002286F
:1018900006D13C2D04D114210320F6F7B2FB07E05A
:1018A000012805D1142D03D13C210320F6F7A9FB13
:1018B000284680B2DDED081A00A991EC030A08F071
:1018C000D6FB206A2818206201200BB030BD10B56D
:1018D000DFF86C4B94F9000000283AD494F90A0020
:1018E00094F90110814228D1217B0818A07240B2DE
:1018F0003D2801DB3C38A07294F90A100FF26C000D
:10190000F0F751FD00202062DFF8D00B90F90100C4
:1019100010F1010F01D1012010BD94F90110081A36
:10192000F1F79CFA21F00041F1F7C8FC40B2012820
:1019300001DB012010BD002010BDDFF8A40B90F9E1
:101940000120914203D0D4E90023C0E90023002004
:1019500010BD206ADFF88C1B884205DB0FF21800EF
:10196000F0F721FD012010BD002010BD50443A20A9
:101970004E5420256400000050443A204E6F5469B4
:101980006D650000F8B52DED028B0024DFF8B05A2C
:1019900007E0BA19AA7252B221460FF26C00F0F7B2
:1019A00002FD95F90A60002C1FD46878841B64B28C
:1019B00095F90C70002CECD52046F1F74FFA21F088
:1019C000004141EC180B3846F1F748FA53EC182B5C
:1019D000F1F728FAE5D2F21BAA72002452B221468E
:1019E0000FF23800F0F7DFFCDBE73C2E02DBA6F15C
:1019F0003C00A87295F90A100FF23400BDEC028B7E
:101A0000BDE8F440F0F7CFBC50443A20636F6D70EE
:101A1000312025642C2025640000000050443A2029
:101A2000636F6D70322025642C2025640000000057
:101A300050443A20435554202564000010B5DFF887
:101A4000004A0020A07301202072002060724FF035
:101A5000FF3020700F20E07214202073002060738C
:101A60006082606260746063A06328220146DFF8D0
:101A70007C0AF0F7F3FBF6F761FAE061F0F711FC8E
:101A8000A061E069DFF8681AC0F888108830DFF8D4
:101A9000641A4160DFF8601A81600FF28D21C16025
:101AA0000FF659210161012010BD10B582B04FF42D
:101AB0006163C1EB0114A40013FB0043D3184FF47E
:101AC0007A746343DFF8244A2360DFF874391B7C9F
:101AD000009313460A4601460FF20800F0F763FC34
:101AE00013BD00005044204254202564202564206A
:101AF00025642025640000002DE9F0412DED028BC6
:101B0000AAB0DFF8D069314684B068465822F0F7B1
:101B10009FFF0FBC00F096FC10EE100AF6F70CFCCD
:101B200041EC100B9FED7E8BDFF8C049656853ECEC
:101B3000102B51EC180BF1F797F8F1F7BFFB15FAE2
:101B400080F060604FF6FF75A84200D365603146B3
:101B500084B068465822F0F77BFF0FBC00F028FCE9
:101B600010EE100AF6F7E8FB41EC100BA76853ECF7
:101B7000102B51EC180BF1F777F8F1F79FFB17FAE0
:101B800080F0A060A84200D3A5600020139002203E
:101B90001290314684B068465822F0F759FF0FBCC6
:101BA00000F09AFAA1894018A08180B2FF2801DBD9
:101BB000FF20A0810020139003201290314684B0B2
:101BC00068465822F0F744FF0FBC00F085FA2169FF
:101BD00040182061A84200D3256100201390062000
:101BE0001290314684B068465822F0F731FF0FBC9E
:101BF00000F072FAA18A4018A08280B2FF2801DBAF
:101C0000FF20A0820020139007201290314684B05C
